:020000040804EE
:1000000000000824E18D05082D8E05089DCC04080C
:10001000A3CC0408A9CC0408AFCC0408000000005D
:10002000000000000000000000000000914D0408E6
:100030002D8E0508000000002B4E04083B4E0408DE
:100040002D8E05082D8E05082D8E05082D8E050890
:100050002D8E05082D8E05082D8E05082D8E050880
:100060002D8E05082D8E05082D8E05082D8E050870
:100070002D8E05082D8E05082D8E05082D8E050860
:100080002D8E05082D8E05082D8E0508D99C050896
:10009000E99C0508E59C0508F59C05082D8E0508DA
:1000A0002D8E05082D8E05082D8E05082D8E050830
:1000B0002D8E05082D8E05082D8E05082D8E050820
:1000C0002D8E05082D8E05082D8E05082D8E050810
:1000D0002D8E05082D8E05082D8E05082D8E050800
:1000E0002D8E05082D8E0508000000002D8E0508B8
:1000F0002D8E05082D8E05082D8E05082D8E0508E0
:100100002D8E0508FD8A05082D8E05082D8E050803
:100110002D8E05082D8E05082D8E05082D8E0508BF
:100120002D8E05082D8E05082D8E05082D8E0508AF
:100130002D8E0508437C04082D8E05082D8E05089C
:100140002D8E05082D8E050800000000000000001F
:100150002D8E05082D8E05082D8E05082D8E05087F
:100160002D8E05082D8E05082D8E05082D8E05086F
:100170002D8E05082D8E05082D8E05080000000027
:100180002D8E05082D8E05082D8E05082D8E05084F
:100190002D8E05082D8E05082D8E05082D8E05083F
:1001A0002D8E05082D8E05082D8E05082D8E05082F
:1001B0002D8E05082D8E05082D8E05082D8E05081F
:1001C0002D8E05082D8E05082D8E05082D8E05080F
:1001D0002D8E05082D8E05082D8E05082D8E0508FF
:1001E0002D8E05082D8E05082D8E05082D8E0508EF
:1001F0002D8E05082D8E05082D8E05082D8E0508DF
:100200002D8E05082D8E05082D8E05082D8E0508CE
:100210002D8E05082D8E05082D8E05082D8E0508BE
:100220002D8E05082D8E05082D8E05082D8E0508AE
:100230002D8E0508DD8D05082D8E05082D8E0508EF
:100240002D8E05082D8E05082D8E05082D8E05088E
:100250002D8E05082D8E05082D8E05082D8E05087E
:100260002D8E05082D8E05082D8E05082D8E05086E
:100270002D8E05082D8E05082D8E05082D8E05085E
:100280002D8E05082D8E05082D8E05080000000016
:100290002D8E05082D8E050810B5054C237833B931
:1002A000044B13B10448AFF300800123237010BD49
:1002B000C0180024000000004CCC060808B5034B11
:1002C0001BB103490348AFF3008008BD00000000E4
:1002D000C41800244CCC0608154B002B08BF134B48
:1002E0009D46A3F5803A00218B460F461348144AD9
:1002F000121A21F0A5FC0F4B002B00D098470E4B93
:10030000002B00D098470020002104000D000D486C
:10031000002802D00C480DF077FB20F08FFF200062
:10032000290006F025FF0DF081FD00BF0000080048
:100330000000082400000000CD700408C01800244C
:100340009817012409DA0408000000002DE9F043A1
:10035000234C91B0234F04AD234E94E80F0085E861
:100360000F0004F1100308AD20340FCB85E80F0017
:1003700094E80F0010AC1D4D04E90F001C4BFA214E
:1003800040F213121B4CC3E90012DDE90C89DDE9D0
:100390000801DDE90423C6E90001C7E90023C5E936
:1003A0000089CDE90001CDE90289204600F07CF802
:1003B000DDE90A01DDE90623C6E90201C7E90223F6
:1003C000DDE90E67C5E90267CDE9000104F17800B7
:1003D000CDE9026700F068F811B0BDE8F08300BF16
:1003E00038700608280000241800002408000024A3
:1003F00048000024081B0024FFF7A8BF38B590F878
:100400007050044615B90025284638BD04F066FB37
:10041000236CA26DC31A9A42F5D8636B93ED002B3F
:10042000E36B93ED005B94ED087B94ED126B35EE7E
:10043000425BA7EE056B94ED1A7BB4EEC76B84EDBF
:10044000126BF1EE10FA23DD84ED127B94ED063B86
:1004500094ED126B94ED0A4BA3EE056B94ED145BD7
:1004600032EE455BA4EE456BB4EEC67BF1EE10FABE
:1004700007D494ED187BB4EEC67BF1EE10FA37FE8C
:10048000067BA36B83ED007B84ED142B2064BBE71C
:1004900094ED184BB4EEC46BF1EE10FAD6D584EDA2
:1004A000124BD3E7000000009FED215B43EC162BBD
:1004B0009DED007BB4EEC56B9DED024BF1EE10FAA5
:1004C00033D4B4EEC57BF1EE10FA2ED4B4EEC54BA6
:1004D000F1EE10FA29D4D0ED163AC0E90023164BFC
:1004E000B8EE632B93ED003A036BB8EEC33B012BE0
:1004F00082EE031B80ED027B80ED044B80ED066BEA
:1005000084EE013B27EE017B80ED087B80ED0A3B0A
:100510000BD135EE466B35EE477B35EE435B80ED18
:10052000066B80ED087B80ED0A5B7047AFF30080BF
:100530000000000000000000040000249DED006B9E
:1005400043EC172BB4EEC67BF1EE10FA2BDAC0E9C0
:10055000182390F8703080ED1A6B23B3836B93ED02
:10056000005BB4EEC56BF1EE10FA0DD583ED006BB8
:1005700090ED126B90ED1A7BB4EEC76BF1EE10FAB2
:100580000ADD80ED127B0EE0B4EEC57BF1EE10FAD1
:10059000EEDD83ED007BEBE790ED187BB4EEC76BEF
:1005A000F1EE10FAEDD47047836B90ED1A6B93ED7A
:1005B000007B436BB4EEC67B80ED127BF1EE10FA4C
:1005C000D3E90023C0E9142302DD80ED126B06E0BD
:1005D00090ED186BB4EEC67BF1EE10FAF5D47047CF
:1005E0004B1E5942594190F8703083F001038B4201
:1005F00010B5044601D1FFF7D7FF84F8701010BD85
:1006000090F87030B3B1036B8B4213D09FED0A7B2F
:1006100090ED066B37EE466B80ED066B90ED086B48
:1006200037EE466B80ED086B90ED0A6B37EE467B3C
:1006300080ED0A7B016370470000000000000000AD
:100640001FB5C3630023044680F870300023C0E95F
:100650000D1200220C99C0E918230FA3D3E900233F
:10066000C0E91A234FF4FA738365FFF7C9FFDDE988
:100670000A23CDE90223DDE90823CDE90023DDE9E2
:100680000623FFF711FF04F029FAA36DC01A2064B6
:10069000204604B010BD00BF0000000000E06F4025
:1006A000D0E900017047D0E902017047D0E90401A8
:1006B000704708B5002000F0C7F90120BDE80840E8
:1006C00000F0C2B9012307B50022009300200323E4
:1006D000024900F0E1FA03B05DF804FB0000694054
:1006E0000149024804F0B4B87FBF060890330024E3
:1006F0002DE9F04114490026144804F08CF8144800
:1007000000F0C6FDDFF850800546104C114FB5B122
:1007100001364146204604F07EF80A223146204642
:1007200004F0DFF83946204604F075F829462046E3
:1007300004F08EF8064800F0ABFD0546E7E7BDE89B
:10074000F041FFF7CDBF00BF817006089033002451
:10075000DC180024097106087670060808B50449FB
:10076000044804F058F8BDE80840FFF7B9BF00BFDF
:100770008D7006089033002408B50449044804F03D
:100780004AF8BDE80840FFF7ABBF00BF9A70060803
:1007900090330024014800F015BE00BFDC1800248F
:1007A000014800F057BD00BFDC18002437B5104CDD
:1007B0004FF496410F4D204602F06EFC0E4B28463A
:1007C0000E4A01930E4B0F4900930F4B00F00CFEA5
:1007D000002328460D4A0E49CDE9003300F004FEFF
:1007E0000C49204603B0BDE8304004F027B800BFF4
:1007F00090330024DC18002479070408B3060408A9
:100800005D07040868700608F1060408C5060408B8
:100810006B7006087070060807EE902AF5EEC07A35
:10082000F1EE10FA48BFDFED147A032923D8DFE890
:1008300001F0020A121AB2EE057AC7EE877A17EEB5
:10084000901A08F087BBB2EE057A2430C7EE877A9B
:1008500017EE901AF5E7B2EE057A4830C7EE877AC0
:1008600017EE901AEDE7B2EE057A6C30C7EE877A94
:1008700017EE901AE5E7704700000000F8B52DED7F
:10088000028B02F0CFF803781C4CB52B1C4F33D1F0
:10089000C18841F6030399420CBF02210021194B84
:1008A00000224FF44075D4F89400B842FBD1914235
:1008B000D86902F1010203F11C030EBF9E68000417
:1008C000DE68032A30606561EDD1962004F024F9DA
:1008D00000210D4801F01CFA08EE100A00210A4818
:1008E00001F06CFAB7EEC88A084B83ED008B83EDFC
:1008F000028BBDEC028BF8BD0021D0E700640258EA
:1009000000030080BC1C0024C41C0024F81B00242D
:1009100010B5164C1648FFF771FD94ED007BBDEE47
:10092000C77B17EE103A002B08DC00200021114B8A
:10093000C3E9000100210E48FFF752FE0E48FFF701
:100940005DFD94ED027BBDEEC77B17EE103A002BE8
:100950000ADC00200021074BBDE81040C3E902017A
:1009600000210548FFF73CBE10BD00BF3800002441
:10097000081B0024081C0024801B00242DE9F843D8
:1009800004F0ACF8134D0646134F00244FF0000955
:10099000DFF84C806B6821464046F31AB3F5FA7FC6
:1009A00088BF6E6055F8043FF31A07EE903AB7EC33
:1009B000026BB8EE677BB4EEC76BF1EE10FACCBFFA
:1009C000064A4A46FFF728FF0CB1BDE8F883012428
:1009D000E0E700BF141C0024081C0024000028418C
:1009E0002C1C00242DE9F843124E4FF00008124F42
:1009F0004FF000090025114C1149124803F028FF5F
:100A000030460021C7E90089FFF7EAFD2A46204663
:100A10000021FFF701FF06F178000021C7E90289F4
:100A2000FFF7DEFD2A4601212046FFF7F5FEBDE86F
:100A3000F88300BF081B0024380000242C1C00246D
:100A40009471060890330024F7B5334C05463349BA
:100A500078272046022603F0DAFE0A22294620469D
:100A600003F03FFF2E49204603F0D1FE2D4B07FB3C
:100A70000537ED003846FFF713FE009602460B4699
:100A8000204603F0D1FF2849204603F0C0FE384637
:100A9000FFF709FE009602460B46204603F0C4FF0E
:100AA0002249204603F0B3FE3846FFF7FFFD0096CB
:100AB00002460B46204603F0B7FF1D49204603F0CF
:100AC000A6FE1C4B009620462B44D3E9002303F0DE
:100AD000ABFF1949204603F09AFE184B00962046BA
:100AE0002B44D3E9002303F09FFF1549204603F070
:100AF0008EFE144B009620461D44D5E9002303F0DA
:100B000093FF1149204603F082FE204603B0BDE862
:100B1000F04003F08DBE00BF903300247F700608C4
:100B200074710608081B0024B0700608B770060828
:100B3000BE70060838000024C5700608F81B0024A3
:100B4000CC700608081C0024D370060837B521486D
:100B500001F02DF8204A214BD2F894109942FBD194
:100B60001F4B802000241F4DD96F1B6F1B040B608F
:100B70004FF440730021536104F0DCF8012106209A
:100B800004F0D8F81849194808F0E4F9164918484B
:100B900008F0E0F900211748FFF722FD00220023AA
:100BA0001448CDE90045FFF7C9FC0020FFF74CFFD2
:100BB00000211148FFF714FD002200230E48CDE963
:100BC0000045FFF7BBFC012003B0BDE83040FFF754
:100BD0003BBF00BFC41C0024006402580003008017
:100BE000BC1C002400407F403DCF733F2C1C0024E0
:100BF000501C0024081B0024801B002407EE901AC0
:100C0000084B00294FF07802B8EEE77B03EBC003F6
:100C1000D4BF0021012183ED007B034B02FB003098
:100C2000FFF7DEBC38000024081B002408B403686A
:100C30008B4277B50446164623DBC36821EAE1758B
:100C400013B1294680689847237953B10F4BA068A8
:100C50002B4413F8011C03F0E2FD0D49A06803F0DA
:100C6000DAFD08AA07992046019201F083FD236965
:100C700013B12946A06898471EB10649A06803F041
:100C8000CAFD03B0BDE8704001B07047A970060806
:100C900009710608D78E06082DE9F04F2DED108B4F
:100CA0008FB092464FF0010808934FEACA0541EC15
:100CB0001D0B03F013FF064603F010FFB249B348C3
:100CC000B14603F0C5FDB346FFF78CFEB049B14B0A
:100CD0000022481907919FEDA0ABC0E90023CDE9A0
:100CE0000A230020AC4BB0EE4ABBB0EE4ACB2B44FB
:100CF000B0EE4A9B0746069009939FED998B9FEDB6
:100D00009AFB03F0EBFE0446FFF7B8FD099B93ED59
:100D100000EBB4EE4EABF1EE10FAB4EE4E8B48BFE2
:100D2000B0EE4EABF1EE10FA3EFE088BB8F1000FBC
:100D300017D0B4EECDEBF1EE10FA40F3CA8009F50E
:100D40009C530833A34280F0C480079BB0EE4DABA8
:100D500026462B449FED807B83ED007BA4EB0903AB
:100D60000693B4EECDEBF1EE10FA02D44FF000088A
:100D7000AFE006F59C530833A342F7D2002F40F3AF
:100D80009C8086494FF00208804803F040FD0A220B
:100D9000FA217E4803F083FD7C4803F049FD804939
:100DA0007A4803F034FD0A22FA21784803F077FDEF
:100DB000764803F03DFD7B49744803F028FDCDF8EB
:100DC0000080724853EC182B03F02EFE6F4803F09E
:100DD0002FFD75496D4803F01AFDCDF800806B4872
:100DE00053EC1A2B03F020FE684803F021FD474521
:100DF00063DD3AEE488B069AB6EE006BA31B6B4997
:100E000028EE0F8B134461489FED597B9FED5A9B51
:100E100028EE068B9FED5A5B87EE086B08EE103AC2
:100E2000B8EEC88B28EE058B26EE099B8DED0C6B7A
:100E300039EE095B28EE09BB85EE08CBB4EE005B0A
:100E40002BEE05BB03F0E3FCCDF800804F489DED91
:100E50000C6B53EC162B03F0E9FD55494B4803F09E
:100E6000D6FCCDF80080494853EC182B03F0DEFD8A
:100E70005049464803F0E2FC4F49444803F0C7FCA0
:100E8000CDF80080414853EC192B03F0CFFD4B49BE
:100E90003E4803F0BCFCCDF800803C4853EC1C2BD2
:100EA00003F0C4FD4649394803F0B1FCCDF8008099
:100EB000364853EC1B2B03F0B9FD079BB0EE4D8B6E
:100EC0000137A1462B444FF001089DED0A7B83EDCD
:100ED000007BB3EE046B3DEE066BB4EECE6BF1EE31
:100EE00010FA08D5374929480FB0BDEC108BBDE882
:100EF000F04F03F0A3BC0BF5FA63A34223D23249AF
:100F00004FF0020B214803F086FC0A2251461F488D
:100F100003F0E7FC2D491D4803F07DFCCDF800B03F
:100F20001A4853EC1E2B03F07FFD2949174803F0A4
:100F300072FC079BCDF800B0A3462B441348D3E9BD
:100F4000002303F073FD09EB0603C3EB4404214BBC
:100F50009C4243D92049C6E7000000000000000081
:100F6000000000000088C340182D4454FB210940B4
:100F70000000000000408F40333333333333E33F0E
:100F8000FCA9F1D24D62503F6870060890330024EE
:100F9000081C002400406F40F81B0024DA7006088B
:100FA000FB700608E0700608E5700608EA7006089F
:100FB000EE700608D88E0608F2700608F67006086D
:100FC000FA700608FE7006086970060809710608BE
:100FD00007710608808D5B000C710608089B9F4214
:100FE0004EDD02242849294803F028FC28492748D7
:100FF00003F011FC0094254853EC192B03F016FD67
:101000002449224803F007FC0094204853EC1C2B91
:1010100003F00CFD20491D4803F0FDFB00941B4824
:1010200053EC1B2B03F002FD1C4B1D4978202B4475
:1010300000FB0A1083ED009B1A4B2B4483ED00CB81
:10104000194B1D4453EC192B85ED00BB8DED02BBF4
:101050008DED00CBFFF728FA144B0122062114482E
:101060008DED049B8DED02CB8DED00BBFFF7DEFD1A
:1010700050460FB0BDEC108BBDE8F04FFFF7E4BC5D
:10108000FFF77CFC3DE600BF147106089033002496
:101090001C7106083A7106085871060828000024D9
:1010A000081B00241800002408000024767106089C
:1010B000782D00242DE9F04FDFF884A089B0DFF807
:1010C00084904FF0000BDFF88080194F194E1A4DB5
:1010D0001A4C2946CDF818B02046DAE90023CDE9AC
:1010E0000423D9E90023CDE90223D8E90023CDE97F
:1010F00000233B463246FFF7A3FA05F10801CDF87D
:1011000018B004F17800DAE90223CDE90423D9E923
:101110000223CDE90223D8E90223CDE9002307F118
:10112000080306F10802FFF78BFA09B0BDE8F08F5B
:1011300038000024081C0024F81B0024081B00248D
:1011400008000024180000242800002408B501200D
:10115000FFF752F9FFF7FAFCBDE80840FFF726BB9E
:10116000F7B503F0BBFC204A04461368C31A642B8E
:101170001CD91E4E1060FFF781FBFFF7C9FB3578C5
:10118000A5B91B4F28463968FFF738FD396801209B
:101190000127FFF733FD2846FFF756FC009702238F
:1011A0002A4600201349FFF777FD3770124DFFF7ED
:1011B000E5FB124A2B681268E31A93420CD90C4ED5
:1011C00000203168FFF71AFD31680120FFF716FD96
:1011D0000020FFF739FC2C60FFF7DCFA642003B035
:1011E000BDE8F04003F098BC281C0024201C00241B
:1011F0005000002400006940241C002454000024F6
:1012000000207047406910B103681B691847704798
:10121000406910B103685B6918477047406910B1B5
:1012200003689B6918477047406910B10368DB6821
:10123000184770470020704700F11C034FF40072FC
:10124000002110B50446184620F0FAFCC4F81C0230
:1012500010BD000000234FF47A7210B5C0E90132CE
:10126000054A044680F824320260C0E90433FFF7DF
:10127000E3FF204610BD00BFBC71060810B503692E
:10128000044603B198472046BDE81040FFF7D4BF9D
:1012900000F508720149002021F05CBD9E7106082E
:1012A0002DE9F04300F11C04ADF5017D06464FF435
:1012B00000722146684620F0C5FB204606F50872FC
:1012C000214921F047FD0446B0B396F82482002757
:1012D0004FF40479B8452FDDB5694FF4007220460C
:1012E00009FB0755294621F019FA50BB204621F089
:1012F000A7F9022204461549684421F00FFA28B9DB
:10130000D5F8003203B19847012016E01DF80430EB
:101310003F2B08D1D5F80432002BF4D1D5F80C427C
:1013200034B1A047F0E73D2BF8D1D5F80832F3E708
:101330000749304603F08CFA00200DF5017DBDE829
:10134000F0830137C6E700BF9E710608A771060843
:10135000AA71060870B500F11C05D0F81C320446CD
:101360000E465B1BB3F5FF7F01DDFFF787FFD4F867
:101370001C325A1CC4F81C2200221E70D4F81C32E5
:101380001A70D4F81C325B1BB3F5FF7F16DD2846BC
:1013900021F056F902380A49284420F0D5FF68B9EF
:1013A0002046FFF77DFF20B12046BDE87040FFF7E3
:1013B00043BF2046BDE87040FFF760BF70BD00BF6F
:1013C000A471060810B50446236820461B69984797
:1013D000002808DD236820465B699847C1B2204693
:1013E000FFF7B8FFF0E710BD2DE9F0414FF40475A9
:1013F000884690F8241204468069174601FB05517F
:101400001E4620F0D3FC94F82432A0614FF4007201
:1014100005FB0300414621F0CDF994F82422A3698D
:1014200005FB0232C2F8007294F82422A36905FB7E
:101430000232C2F8046294F82432A26905FB032345
:10144000069AC3F8082294F82432A26905FB032502
:10145000079BC5F80C3294F82432013384F8243207
:10146000BDE8F081704710B504461C300AF01EFC40
:10147000204610BD10B504460AF018FC204610BDE9
:1014800010B504466C3007F0B6FD04F1480007F0D3
:10149000B2FD04F1240007F0AEFD204607F0ABFDDD
:1014A000204610BD38B504460D461C22002120F010
:1014B000C7FB204629460AF078FC204638BD0000CC
:1014C00038B504463421FFF7EDFF352104F11C0047
:1014D000254DFFF7E7FF432104F13800FFF7E2FF56
:1014E000632104F15400FFF7DDFF372104F17000A0
:1014F000FFF7D8FF762104F18C00FFF7D3FF972187
:1015000004F1A800FFF7CEFF7F2104F1C400FFF72C
:10151000C9FF7A2104F1E000FFF7C4FF042104F1C0
:10152000FC00FFF7BFFF082104F58C70FFF7BAFF3E
:10153000262104F59A70FFF7B5FF2A4640F62301ED
:1015400004F5A87007F0C6F92A4640F6220104F512
:10155000E07007F0BFF92A4640F6010104F50C706F
:1015600007F0B8F9204638BD0000C07F10B504462A
:101570001221FFF797FF862104F11C00FFF792FF6D
:10158000792104F13800FFF78DFF992104F154000F
:10159000FFF788FF422104F17000FFF783FF8321EA
:1015A00004F18C00FFF77EFF822104F1A800FFF711
:1015B00079FF332104F1C400FFF774FF0E2104F119
:1015C000E000FFF76FFF204610BD10B50446A430C1
:1015D00007F054FC04F1540007F050FC201D07F004
:1015E0004DFC204610BD10B5044600F58470FFF791
:1015F000ECFF2046FFF7E9FF204610BD10B504467A
:1016000000F59E7007F000FA204610BD2DE9F34169
:101610004FF47A73002504464FF48072C561294661
:1016200004F59E76058404F52777C0E90153224B23
:1016300003602023C0E905358923283020F8063CC3
:101640004FF6FF7320F8043C20F8023C20F0F8FA33
:10165000C4F8285184F838517D22C4F82C5118213F
:10166000C4F83051304607F071F9284603F008FA03
:1016700005468D2003F004FA80468A2003F000FA24
:10168000009043462A462146384600F009FD04F5FD
:1016900034731C220021184620F0D2FA00220D21BA
:1016A0000AF07FFB04E0304607F0AEF91CF0D0FFF3
:1016B000204602B0BDE8F0813C77060813B506214C
:1016C0004F4800F0D7F84F4A07214F4800F028FA5A
:1016D00036214E48FFF7E6FE84214D48FFF7E2FE33
:1016E0006A214C48FFF7DEFE2F214B48FFF7DAFE58
:1016F0004A48FFF78BFF4A4A4A4948480CF082F9AA
:101700004948FFF7DDFE464A484947480CF07AF958
:101710009B21474807F051FCA121464807F04DFCAA
:101720006721454807F049FC2721444807F045FC5C
:1017300000243B4A42493E480CF064F97B237C225A
:1017400098214048CDE9004400F046F99A238722C9
:101750002D213D48CDE9004400F03EF90CE036482B
:1017600007F049FC334807F046FC314807F043FCDA
:101770001CF06EFFF6E7F8E7294A344931480CF0CF
:1017800041F93348FFF7F2FE324800F035FB3248AA
:1017900000F032FB7E213148FFF784FE304800F034
:1017A000BDF91C2200212E4820F04AFA01221921FD
:1017B0002B480AF0F4FA1A4A2A4929480CF022F96F
:1017C0001C220021284820F03BFA00221E21264836
:1017D0000AF0E7FA1C220021244820F031FA1F21E8
:1017E00022480AF0D9FA0E4A21491F4802B0BDE842
:1017F00010400CF007B91348FFF7E7FEB8E700BF49
:10180000BC1C002478260024C41C0024D81C0024FE
:10181000F41C0024101D00242C1D0024481D00244D
:1018200000000024FD150408B823002465140408F2
:101830002C1C0024501C0024741C0024981C002420
:1018400081140408A8210024B0220024E71504080C
:101850008C20002434200024882100248C210024A2
:10186000382000247514040854200024702000241B
:1018700067140408014A01804260704778260024FA
:10188000034B044A1A6001221A715A71704700BF53
:101890005826002440420F007047D0F8043101332D
:1018A000C0F80431704738B50446043007F0B8FA80
:1018B000054604F1540007F0B3FA237840EA4500E6
:1018C000C4F8FC00E3B9D4F8F830032B06D140B9D2
:1018D000D4F800310133C4F8003102E023B9032801
:1018E000F6D0C4F8F80038BD022B05D10128F8D194
:1018F000D4F80031013BEEE7012BF2D10228F6E7E4
:10190000012BEED1D4F8F83080EA0302032AE8D0A4
:101910009842E6D083EA6003D4F8002113F0010373
:1019200008BF4FF0FF33D31AD5E70B6803604B684D
:1019300043608B6883607047C3680BB19B6818472E
:10194000704710B50446FFF7F7FF204610BD10B4EE
:10195000D0E9003409686210E4075DF8044B01EB3C
:10196000020044BF8A58D35818470146043008B5CE
:10197000FFF7EDFF08BD0000034A0346C26007C938
:1019800083E80700704700BFD871060810B586B01D
:1019900004460391684606A980E80C0001E90C00A2
:1019A000204603A9FFF7E8FF204606B010BD37B573
:1019B0006C46054684E80C0094E80C00FFF7E6FF4F
:1019C000284603B030BD08B5FFF7CFFF08BD08B506
:1019D000FFF7F9FF08BD00002DE9F0470446061D9A
:1019E0008EB0154604F15407304699469DF85CA028
:1019F00007F01EFA2946384607F01AFA04F1A4083F
:101A00004946404607F014FA002384F800A0304607
:101A1000C4F80031C4F80431169BC4F8F43007F060
:101A2000FFF90546384607F0FBF9002340EA450078
:101A3000384D214601936B460095C4E93E000CCB1E
:101A40000AA8FFF7B4FF0AA9304607F035FA0AA83A
:101A5000FFF777FF002302952146039302AB0AA804
:101A60000CCBFFF7A4FF0AA9304607F042FA0AA8F8
:101A7000FFF767FFBAF1010F1FD10023049521463C
:101A80000AA8059304AB0CCBFFF791FF0AA93846CF
:101A900007F012FA0AA8FFF754FF00230695214623
:101AA000079306AB0AA80CCBFFF781FF0AA93846BB
:101AB00007F01FFA0AA8FFF744FFB9F1FF3F10D063
:101AC000154B21460AA808930023099308AB0CCBB9
:101AD000FFF76DFF0AA9404607F0EEF90AA8FFF7E5
:101AE00030FF20460EB0BDE8F0870AA8FFF729FFB7
:101AF000404607F0C3F9384607F0C0F9304607F012
:101B0000BDF91CF0A5FDF0E7EFE7EEE7EDE7EFE745
:101B1000F1E7F3E7A71804089B18040870470000D2
:101B2000C0E90112044AC260002210B50274012209
:101B3000024C4274046010BD00093D006666064018
:101B400010B504460021007903F02AF8207900211D
:101B500003F0AAF8A0680368BDE810401B6B1847A3
:101B600070B5002104460079042603F09DF8012099
:101B700002F0D4FFA0680368DD6904F10C0393E868
:101B80000600A8470025A06800212D0203689B6875
:101B90009847013E45EA0005F5D1A06803681B6A35
:101BA00098472079012103F07FF8284670BD10B5D1
:101BB00004460121007902F0F3FF0121207903F0AE
:101BC00073F8A0680368DB6A98472046FFF7C8FFF0
:101BD0006FF07F43984204D12046FFF7B1FF002009
:101BE00010BD0120FCE7000043EC152BDDE90003EC
:101BF000002282421EDA1946183313ED047BB4EE3C
:101C0000C57BF1EE10FA13DD086898B1B7EE006BF2
:101C100000239FED0B7B98420EDD0A6902EBC302A5
:101C2000013392ED004BA4EE067B26EE056BF2E746
:101C30000132DEE79FED047B51EC170B704700BFCC
:101C40000000000000000000000000000000F87F1D
:101C500010B543EC132B2DED028B0C4682B061B313
:101C60001D4B012918BF002301930323009353EC5C
:101C7000132BFFF7B9FF41EC180BC4B9B5EEC03B0D
:101C8000F1EE10FA13DD9FED0E7B33EE473B9FED37
:101C90000E7B23EE033B23EE077B51EC170B1EF06C
:101CA0007FF99FED0B7B41EC160BA6EE078B51ECF9
:101CB000180B02B0BDEC028B10BD084BD4E700BF7F
:101CC000F5B9DA8AFDBD5F404175DFB1E0051FBFA0
:101CD000B253628D695CBE3F507206089872060866
:101CE00037B514461D4669B1074B01290CBF19468B
:101CF000002104232246019100932B46FFF774FF35
:101D000003B030BD0149F4E718740608787406087A
:101D100038B52DED048B0D460446FFF721FF410732
:101D200041D1830C00284FEA101094ED007AB8BF1F
:101D30006FEA83332946B7EEC77AB8BF6FEA9333A9
:101D4000020508EE103AC0F30B03204648BF6FEAC5
:101D50000353BAEECF8A48BF6FEA1353B7EEC88A6F
:101D600009EE103ABAEECE9AB7EEC99A39EE477B31
:101D700053EC172BFFF76CFF38EE498B9FED0C7B74
:101D800041EC160B29462046A8EE076B53EC162BA8
:101D9000FFF7A6FF41EC170BF7EEC77B17EE900A93
:101DA000BDEC048B38BDDFED047AF7E7AFF30080BC
:101DB000000000C02022A53F0000C07F01607047E6
:101DC000064B074A1A6007225A60064A9A60064A7A
:101DD000DA6000221A7401225A74704760260024C7
:101DE000666606407826002400093D00014800F0A0
:101DF00003B800BF7426002422230370704710B577
:101E0000C36886B001228DF80F100DF10F0118681C
:101E100003680092DC680DF11703A0479DF81700D6
:101E200006B010BDF8B5427A044603680E46CFB23C
:101E30009B680D0A62B939469847236860F3070624
:101E400029469B682046984760F30F26B0B2F8BD3C
:101E500029469847236860F30F2639469B68204639
:101E6000984760F30706F1E7C36813B5186803687D
:101E70000092DC680B46A04702B010BD7047704767
:101E80007047C36810B5044653B1186840B1036881
:101E90005B6898470421E0680CF038F80023E360A1
:101EA00010BD10B5044618210CF030F8204610BDC6
:101EB000436873B599426D4604460E4685E80600B0
:101EC00004D1BDF8042003899A420FD0E3680821A9
:101ED0009DF80420186807F0D4FAE36831461868C2
:101EE00007F0EDFA0098AB886060238102B070BD06
:101EF00073B5C568044625B904200BF0D3FFE06034
:101F00000560E3681B6883B94FF0FF3674200BF05F
:101F1000C9FFB4F91430B4F910200546B4F9121011
:101F2000009607F0AFFBE3681D6002B070BD74213E
:101F300028460BF0EBFF1CF08BFB000038B50A20A5
:101F400002F0B2FD0546082002F0AEFD044609206D
:101F500002F0AAFD094B0A4A0121988218461A602C
:101F6000002259725A601A72DA601D825C82054A38
:101F70000549BDE838400BF045BD00BF7826002478
:101F8000E875060800000024811E04080268322358
:101F900013B50093946A40F21342A04702B010BDFB
:101FA00013B5046800931346A46A40F21342A04795
:101FB00002B010BD13B5322304680093A46AA04791
:101FC00002B010BD006903681B6918470069036807
:101FD0009B691847006903685B69184700690368D3
:101FE000DB6818470120704770B504460D46164659
:101FF0000499C5622286026A002A08BF1A46436A0B
:10200000002B18BF1946026241628069002807DB75
:102010000121C0B202F0C4FD0021207E02F044FE86
:10202000E069002807DB0121C0B202F0B9FD0121FF
:10203000207F02F039FE002320693246294684F8C9
:1020400028300368BDE870401B6A184710B5044685
:10205000006903685B6A9847A069002807DB0021D4
:10206000C0B202F021FE0021207E02F099FDE0695D
:10207000002809DB0021C0B202F016FE207F0021FB
:10208000BDE8104002F08CBD10BD034690F828005A
:1020900018B1186903681B68184701225A60704715
:1020A00070B500254FF47A768361049B456280F811
:1020B0002850C0E90156034EC0E904120660C0E989
:1020C000073570BD247606080A4B00224FF47A715A
:1020D00001205A6283F82820C3E9012106491960CA
:1020E000064919611521C3E905011421C3E9071245
:1020F000704700BF9026002424760608DC2F0024B9
:102100000368C9B21B68184749000023C161C0F8C1
:102110002C327047036801211B6B184710B4036809
:102120009C6B0123A4465DF8044B6047D0F82C3229
:10213000B3F5807F1FBF5A1CC0F82C22C01880F84E
:102140002C1114BF012000207047D0F828017047DF
:102150007047C0F830127047C0F834127047D0F89A
:102160002831A3B1D0F828318BB1D0F82431D0F880
:1021700024210344013293F82030D2B2C0F8242144
:10218000D0F82821013AC0F82821184670474FF0AE
:10219000FF307047D0F828312BB1D0F824311844E3
:1021A00090F8200070474FF0FF30704738B5036853
:1021B00004465B6A9847FC200BF074FEB4F91A20C1
:1021C000B4F91810054606F0A1FD656138BDFC2183
:1021D00028460BF09BFE1CF03BFA38B5D0F82C32A9
:1021E0001446054600F596701A441844B2F5807FEF
:1021F00088BFC3F5807422461FF024FCD5F82C322A
:1022000020462344C5F82C3238BD38B50446406911
:102210000D4608B106F08FFC206920B12946BDE8C3
:10222000384006F0CBBD38BD07B581F0010100F59F
:1022300096720091D0F82C32C169406906F08EFC8C
:10224000002814BF0220002003B05DF804FB10B585
:102250000446406920B10368DB6898470023636146
:1022600023699BB1D4F838020CF086F9D4F838020F
:102270000CF0E7F9D4F8380210B103685B689847AE
:102280009C2120690BF042FE0023236110BD70B534
:10229000C2B083F001030446154602AE0093490024
:1022A00013464069324606F07AFCC8B9A84218D0F5
:1022B000D4F82831B3F5807F10D0D4F82031325CC7
:1022C000234483F82020D4F820310133DBB2C4F852
:1022D0002031D4F828310133C4F828310130E5E742
:1022E0000025284642B070BD30B50446BDB000257B
:1022F000206906F06CFD0328FAD8DFE800F04A02F6
:102300001212D4F8343203B19847D4F82C22002AA0
:10231000EED004F59671206906F05DFDC4F82C52EC
:10232000E6E7C4F82051F022C4F824516946C4F805
:102330002851206906F04DFD002282421DDAD4F8B2
:102340002831B3F5807F18D0D4F82831B3F5807FD9
:1023500011D0D4F820311DF80210234483F8201046
:10236000D4F820310133DBB2C4F82031D4F828315D
:102370000133C4F828310132DFE7D4F82831002BCB
:10238000B6DDD4F83032002BB2D0D4F8280198470B
:10239000AEE702F0D3FBABE70022C260704700005B
:1023A00038B500254FF47A730446018342832946E9
:1023B0004FF48072C0E901530A4BC0E90455036031
:1023C00020301FF03DFCC4F82051C4F82C522046A8
:1023D000C4F82451C4F83052C4F82851C4F8345217
:1023E00038BD00BF7876060810B504460021FFF717
:1023F000D3FF204610BD10B4D0E900340968621044
:10240000E4075DF8044B01EB020044BF8A58D3583F
:1024100018470146043008B5FFF7EDFF08BD00007E
:10242000034A0346C26007C983E80700704700BF3C
:102430005876060810B586B004460391684606A98A
:1024400080E80C0001E90C00204603A9FFF7E8FF33
:10245000204606B010BD37B56C46054684E80C0032
:1024600094E80C00FFF7E6FF284603B030BD0000FB
:102470002DE9F0410368054688B00E465B6A98472F
:102480009C200BF00FFDB5F91A20B5F91810044681
:1024900006F07AFC710020462C6106F091FCBC200D
:1024A0000BF000FD04460646234B04F1400746F8B6
:1024B000043B3046FFF798FF002138460BF062FFDF
:1024C00004F1540840460BF0FDFE1C4B4FF4006233
:1024D00018212046009300230BF0DCFF184B2946FF
:1024E00004A8C5F8384202930023039302AB0CCB37
:1024F000FFF7B1FF04A920460BF0D8FF10E04046DB
:102500000BF01EFF38460BF066FF3046FFF719FA56
:10251000BC2120460BF0FAFC1CF09AF8F2E7F4E735
:1025200004A8FFF70EFA08B0BDE8F0819C21F0E79F
:1025300004A8FFF706FAEFE7849506086476060814
:10254000E922040808B5FFF764FF08BD08B5FFF7E6
:10255000F9FF08BD10B50B2002F0A6FA04460C20C6
:1025600002F0A2FA214602460748FFF719FF162299
:1025700017210648FFF714FF7B227C210448BDE8A1
:102580001040FFF70DBF00BFC4260024002900241F
:102590003C2B002473B505461446002940D025295C
:1025A00005D1806802B0BDE8704002F038B97329E7
:1025B00009D1136880681A1D1968226002B0BDE84D
:1025C000704002F028B9532909D1136880681A1D98
:1025D0001968226002B0BDE8704002F018B96429A1
:1025E00001D069290AD12368A8681A1D22600A222D
:1025F000196802B0BDE8704002F073B901F0FD0245
:10260000442A0FD123688068073323F0070303F1BE
:102610000802226002220092D3E9002302F004FAA9
:1026200002B070BD782905D1236880681A1D226028
:102630001022DDE7582920D14849806802F0EBF8E4
:1026400023681A1D1E6840F6FE732260B4B29C42D5
:102650000FD83021A86802F0E2F8FE2C09D830210A
:10266000A86802F0DCF80E2C03D83021A86802F02C
:10267000D6F81022B1B2A868BBE7702909D1236847
:1026800080681A1D1968226002B0BDE8704002F02F
:10269000C9B8622905D12368A8681A1D22600222E0
:1026A000A6E7422904D12E49806802F0B4F8F2E787
:1026B0006C290AD1236880681A1D196822600A22D1
:1026C00002B0BDE8704002F0EAB875290AD123686B
:1026D00080681A1D196822600A2202B0BDE87040A5
:1026E00002F001B9632905D1236880681A1D1978A1
:1026F000226057E7432916D1236880681A1D22609B
:102700001C78A4F120035E2B01D821464AE7134927
:1027100002F081F80E2C03D83021A86802F07FF86F
:1027200010222146A7E774290AD1236880681A1D60
:102730001B68012B226001D10A493FE70A493DE7A6
:1027400054297FF46DAF236880681A1D1B68012B24
:1027500022600CBF054906493CE700BFC876060861
:10276000CB7606086970060890950608EF80060883
:102770000E810608F7B5064602AD0C4645F8042D55
:10278000217871B1252908D1671C61782A46304625
:102790003C46FFF7FFFE0134F2E7B06802F03FF875
:1027A000F9E703B0F0BD0000044B002201211A60DC
:1027B00019711A61C3E90222704700BF782D002405
:1027C000002070470020704730B5A1F110040025AB
:1027D00000F00F02CD7302390009D3B2092ACCBF31
:1027E000373330330B748C42F2D130BD2DE9FF47C3
:1027F0000024061D05468A469046994600942346C5
:102800004FF0FF32B1213046CDE9014406F05DFDC5
:1028100029682846DDE90C23CDE9002342464F69AB
:102820004B465146B847009423464FF0FF32C12132
:102830003046CDE9014406F048FD204604B0BDE82D
:10284000F0872DE9D04F9B460368924604469B6A69
:10285000DDE90889984702460B46504659461CF068
:1028600099FA134302D00020BDE8D08F2368204698
:102870009B6A984702460B46404649461CF08AFA36
:102880001343F0D11AEB0806236820464BEB0907E7
:102890009B6B9847B94208BFB0422CBF0120002073
:1028A000E2E701682DE9F04114461D46096B064632
:1028B000884702460B46204629461CF06BFA134314
:1028C00002D00020BDE8F081DDE906233046A718DC
:1028D00045EB030817F1FF323368196B48F1FF33FA
:1028E000884702460B46384641461CF053FA1343CC
:1028F000E7D1336830469B6B9847414508BFB842E3
:102900002CBF01200020DDE72DE9D04F9B46036856
:10291000924604465B6ADDE90889984702460B4601
:10292000504659461CF036FA134302D00020BDE849
:10293000D08F236820465B6A984702460B46404684
:1029400049461CF027FA1343F0D11AEB0806236816
:1029500020464BEB09079B6B9847B94208BFB04232
:102960002CBF01200020E2E7C2207047244830B588
:10297000037887B0BFF35B8F13F001041CD10BF019
:1029800051F8C8B11F4B66223B211F48CDE90343D4
:102990005A23CDE901323D233C22009357230CF00A
:1029A000D5FF194C194B164823600BF05DF8184AF7
:1029B000204618490BF026F813480DF005FA164D7D
:1029C0001A22002329461048CDE9002300230022C3
:1029D000FFF70CFF2B780446B52B04D10F4B0122D7
:1029E0001D600F4B1A7008480DF046F8B4FA84F0D9
:1029F000400907B030BD02480BF03CFA1BF028FE3E
:102A0000B02D0024005A6202B82D0024D8760608A2
:102A100000000024DD2B0408C02F002458000024EF
:102A2000B42D0024014B1868704700BF58000024E3
:102A300010B504460DF078FE2146FFF7C5FE0DF0F7
:102A400079FE04F11001FFF7BFFE0DF079FE04F1ED
:102A50002001FFF7B9FE302010BD000008B54DF68B
:102A600059720021074813F0C9FFBFF34F8F064981
:102A7000064BCA6802F4E0621343CB60BFF34F8F8A
:102A800000BFFDE78C2D002400ED00E00400FA05F6
:102A900010B50446FEF750FF204610BD064B10B59A
:102AA00004460360806A08B109F0CEFD201DFFF7DF
:102AB000EFFF204610BD00BF6083060800B5C3B01D
:102AC0001622172103A806F021F94FF4A17302AAD8
:102AD0001021ADF80830002303A80093022306F06C
:102AE0003DF803A8FFF7DAFF43B05DF804FB03A845
:102AF000FFF7D4FF1BF0ACFD1D4B01211D4AA620A2
:102B000070B51A6002F096F80121A62002F012F9C1
:102B1000FFF7D4FF184B43F2D2021A60FFF726FFEB
:102B2000164B1B7833B1164B1B689A8840F2094349
:102B30009A421BD8134B9B6D03F46043B3F5004FCF
:102B400014D001F0CBFF104D044601F0D9FF06462A
:102B500001F0D6FF801BA842FAD901F0BFFF001B8D
:102B6000642803D0BDE8704018F0B4BD70BD00BF4C
:102B70008C2D00240040005800400052B42D002449
:102B800058000024004402589F86010010B50446F6
:102B9000FFF784FFFC2120460BF0B8F9204610BD5A
:102BA00038B5074B0546044645F8BC3B0CF064FFBE
:102BB00028460BF0C5FB201D06F0C6FB204638BD9D
:102BC000A4A1060810B50446FFF7EAFF4FF402710E
:102BD00020460BF09BF9204610BD0000034B10B5BA
:102BE00004460360FFF7DCFF204610BDD8760608D8
:102BF00010B50446FFF7F2FF4FF4027120460BF0C8
:102C000085F9204610BD70B590F838310546144658
:102C1000F3B90368DB69984704F4706304F00F02AA
:102C2000B3F5407F04F0F0030CBF07210821302BDF
:102C30000CBF02230123012A08D0901E42424241C8
:102C4000A869BDE87040006806F052BE0222F7E7AE
:102C500070BD10B590F8383104462BB9A3691868D7
:102C600006F088FE0028F9D010BD38B590F838512C
:102C70000446A5B983695BB1186848B10368DB688D
:102C80009847A36904211D60A0690BF03FF9A56175
:102C90000023C4F82831C4F82C31C4F8303138BDD1
:102CA00013B590F8383104466BBBA369186806F079
:102CB00037FE40B30AF0BEFAA36901220DF1070105
:102CC000186803685B699847D4F83031B3F5807FA2
:102CD00016D0D4F83031B3F5807F11D0D4F8283134
:102CE0009DF80720234483F82820D4F828310133A5
:102CF000DBB2C4F82831D4F830310133C4F83031B4
:102D00000AF0AEFAD1E702B010BD000008B590F8A5
:102D100038313BB1012001F0FFFE0648BDE8084014
:102D200001F059BA82691AB11368003318BF012340
:102D3000184608BD603A002470B504460D4601F0FF
:102D40004AFA30B12368294620461B6CBDE8704022
:102D5000184770BDA0F59860EEE7000013B590F835
:102D6000383104468DF807102BB1C9B20B48FFF774
:102D7000E3FF02B010BDA369186806F0FBFD002850
:102D8000F9D0A36901220DF10701186803681B69D6
:102D90009847013018BF0120EBE700BF603A0024DC
:102DA0002DE9F04107468846164601F014FA80B135
:102DB0000024A6420ED9351B08EB04013846B5F5B0
:102DC000007F28BF4FF400752A462C4400F044FFD2
:102DD000EFE704462046BDE8F081A0F59860DFE704
:102DE00070B590F8383105460E4614462BB10F48A1
:102DF000FFF7D6FF0446204670BDAB69186806F0A1
:102E0000B9FD0028F9D0AB6901211868D0F88830E5
:102E100088301B6B9847AB692246314618680368B7
:102E20001B699847013008BF0024E4E7603A00249A
:102E300030B50446C3B001F0B9F90546D4F8D83529
:102E4000C3F58073984203DDD4F8D855C5F5807575
:102E50002A4601AB02A9204600F0F5FF019902AB1A
:102E600000226D1A1D44D4F8D835B3F5807F19D0EF
:102E70008A4217D0D4F8D835B3F5807F10D0D4F873
:102E8000D035A85C234483F8D004D4F8D03501337E
:102E9000DBB2C4F8D035D4F8D8350133C4F8D8350E
:102EA0000132E0E743B030BD38B5044600F0BCFB6A
:102EB0002046FFF7BDFFD4F8D855204600F0BCFBF4
:102EC000284638BDA0F59860EEE7000010B590F8F0
:102ED000383104462BB10648FFF7E6FF044620468A
:102EE00010BD0AF0A7F9D4F830410AF0B9F9F6E7B5
:102EF000603A002438B5044600F096FB2046FFF700
:102F000097FFD4F8D8354BB1D4F8D435234493F88F
:102F1000D054204600F090FB284638BD4FF0FF35D6
:102F2000F7E7A0F59860E5E710B590F8383104466A
:102F30002BB10B48FFF7DEFF0446204610BD0AF018
:102F400079F9D4F830313BB1D4F82C01044494F829
:102F500028400AF085F9F0E74FF0FF34F9E700BFA9
:102F6000603A002438B5044600F05EFB2046FFF7C7
:102F70005FFFD4F8D835A3B1D4F8D435234493F8FF
:102F8000D054D4F8D4350133DBB2C4F8D435D4F8F6
:102F9000D835013BC4F8D835204600F04DFB284613
:102FA00038BD4FF0FF35F7E7A0F59860DAE700008D
:102FB00010B590F8383104462BB11148FFF7D2FF15
:102FC0000446204610BD0AF035F9D4F830319BB1E3
:102FD000D4F82C31234493F82800D4F82C31013351
:102FE000DBB2C4F82C31D4F83031013BC4F83031B5
:102FF00004460AF035F9E4E74FF0FF34F9E700BF83
:10300000603A002408B54FF4807200211EF018FECB
:103010000022C0F80021C0F80421C0F8082108BD32
:1030200010B4D0E9003409686210E4075DF8044B7D
:1030300001EB020044BF8A58D358184701460430B8
:1030400008B5FFF7EDFF08BD034A0346C26007C994
:1030500083E80700704700BF2877060810B586B0E0
:1030600004460391684606A980E80C0001E90C00BB
:10307000204603A9FFF7E8FF204606B010BD37B58C
:103080006C46054684E80C0094E80C00FFF7E6FF68
:10309000284603B030BD000070B590F8383186B0D6
:1030A00004460E46002B3BD1856925B904200AF061
:1030B000F9FEA0610560A369186850BB8C200AF076
:1030C000F1FE3346B4F922200546B4F9201006F08B
:1030D0002FFFA3691D60B4F92420531C06D0A069FA
:1030E0000321B4F92630006806F030FFA3691D689B
:1030F000B5B1114B0026214602A800936B460196FC
:103100000CCBFFF7BCFF324602A9284606F098FC1C
:1031100003E0314606F0D9FBDDE702A8FEF711FC1B
:1031200006B070BD8C2128460AF0F0FE1BF090FA24
:1031300002A8FEF706FCF9E7A12C040808B5FFF782
:103140007DFF08BD08B5FFF7F9FF08BD2DE9F8437D
:1031500000242D4D4FF47A782C4F202605F12800BD
:103160002F60EC61C5E90148C5E90564FFF74AFF36
:1031700001230E2085F8383101F096FC244D81465C
:103180000D2001F091FCA5F820904FF6FF7968849E
:1031900005F128002F60EC61A5F82490A5F8269091
:1031A000C5E90148C5E90564FFF72CFF85F83841FA
:1031B0000F23184D2B84562305F128002F606B84B4
:1031C0005823EC61AB845923C5E90148EB84C5E978
:1031D0000564FFF717FF85F8384198230E4D2B84BF
:1031E000992305F128002F60EC616B84A5F82490E9
:1031F000A5F82690C5E90148C5E90564FFF702FF77
:1032000085F83841BDE8F883903300243C77060800
:10321000DC2F002418310024543200240020704791
:103220007047704710B5D0F88C452CB12368204604
:103230005B689847A468F8E710BD38B50D46D0F82C
:103240008C4534B12368204629469B689847A4687A
:10325000F7E738BD00487047FC770608054B10B506
:103260000446036008F036F9204608F0D9F92046F4
:1032700010BD00BF7C77060810B50446FFF7EEFFCF
:103280004FF4B26120460AF041FE204610BDF7B56A
:10329000002305460E46D0F88C45A4B1236831467C
:1032A0000DF103022046DF6801ABB8479DF803101B
:1032B0000346042905D0019A284607F0B7FB03B05E
:1032C000F0BDA468E9E7019A9DF80310F4E770B532
:1032D00005460E4622B10021BDE8704007F0A8B9AE
:1032E000D0F88C455CB123680022314620461B692A
:1032F000984710B101212846EEE7A468F2E721467D
:10330000F9E770B50E460546D0F88C4500213CB172
:103310002368314620465B699847A4680146F6E772
:103320002846BDE8704007F07DBAF8B505460E4660
:103330001746D0F88C453CB1236820463A463146C2
:103340009B699847A468F6E728460121BDE8F84044
:1033500007F0C6BA70B5002186B0044607F017FD25
:1033600000234FF48975A188EF26ADF80630238934
:10337000ADF8045002258DF810301B0AE2888DF854
:10338000113040F201238DF80750ADF8123040F2B1
:1033900003138DF809500125ADF8143004F10A0328
:1033A0008DF8086005AE8DF80A501C468DF80C109B
:1033B00001AD090A8DF80E20120A8DF80B008DF868
:1033C0000D108DF80F202A46083303CAB24243F885
:1033D000080C43F8041C1546F5D1128820461A80C3
:1033E00006B070BDF8B5002406460D4627463046A7
:1033F0001FF026F9A04207D9335D05F8143005EB1C
:10340000440301345F70F2E7400000F0FE00F8BDB5
:1034100038B50446D0F88C5535B12B6828461B6A60
:10342000984710B9AD68F7E7284640F2023304F236
:103430004A51A4F84835FFF7D5FF94F848351844A9
:1034400084F8480504F5A96038BD000040F2023355
:1034500000F20A5110B50446A0F808350548FFF7F8
:10346000C1FF94F80835184484F8080504F5A160F4
:1034700010BD00BF6877060840F2023310B504465D
:10348000A0F8C83400F2CA40FFF7D2FA94F8C83462
:10349000184484F8C80404F5996010BD2DE9FF4173
:1034A00000231D4A044600F54E788DF80A300925A0
:1034B00090F888350192FA228DF8083001238DF8B2
:1034C0000C208DF80930C0238DF80B3001AB03CBF5
:1034D000C4F83803C8F8041088F80820D4F88C65BC
:1034E0008EB13368002130461B689847478805F540
:1034F0004E7300F10901093FE0183A463D441EF0C1
:10350000A1FAB668ECE784F83A5340462D1284F8E5
:103510003B5304B0BDE8F0810902FFFF73B50446D8
:103520000D46164616F04AFB4FF4807301462A46B4
:1035300020460093334608F031F8024B20462360C2
:1035400002B070BD7C77060810B5D0F88C35044603
:10355000A3B9C0F88C1594F8883508464A790B71E0
:1035600094F88835134484F888350B685B6A98476B
:10357000238918442081012010BD13469A68002A2F
:10358000FBD19960E7E71FB5044607F0FBFB014656
:10359000684606F0A3FD4021684606F00DFED4F80B
:1035A0008C4534B1236869462046DB699847A46896
:1035B000F7E7684606F099FD04B010BD684606F0CE
:1035C00094FD1BF045F810B50446FFF7DCFF2046DC
:1035D000BDE8104007F056BB0F4808B50378BFF3AD
:1035E0005B8FDB0711D40AF01DFA70B140F25B2249
:1035F00042F241310948FFF791FF07480AF034FAD7
:10360000074A084905480AF0FDF9044808BD024880
:103610000AF030FC1BF01CF8CC340024D034002419
:10362000000000245D32040810B5FFF7D5FF0368E1
:10363000BDE810405B6F184710B5FFF7CDFF03687A
:10364000BDE810409B6F184710B5FFF7C5FF036832
:10365000BDE81040DB6F184706F00ABF06F0CCBE8D
:1036600006F0F6BE704770477047436A93F87800DB
:103670007047D0F8A4047047012070470048704795
:10368000687906082DE9F04794B004460F464B22AE
:10369000002101A81EF0D4FA2679D4F8A434751CB0
:1036A00094F80E90002B94F80C80EDB294F80DE095
:1036B00014BF05200020002F40F0938040F2092322
:1036C00009218DF81D0042F20540ADF804304FF499
:1036D00081738DF815100121ADF808308023ADF805
:1036E0001E0010208DF80B3032234FF0040A2427DF
:1036F0008DF80C3008234FF0030C4B228DF80D3061
:103700000B238DF819101D348DF80E3040F2022372
:103710008DF81C10ADF8103002238DF82100052023
:103720008DF822108DF825108DF8271006218DF8C0
:1037300006208DF80F608DF812308DF817608DF827
:103740001A308DF81B308DF823008DF826C08DF8C7
:103750002A308DF82B108DF82C008DF816A08DF8DE
:1037600024708DF828A08DF829708DF82D708DF8B3
:103770002E1007218DF82F6041F202068DF83110CE
:103780008DF8411040F207518DF83050ADF8366099
:1037900040F209468DF83A5040F602258DF8320085
:1037A0008DF842002046ADF848100DEB0A018DF867
:1037B00033908DF834C0ADF83860ADF83C508DF8DA
:1037C00043808DF844308DF846308DF84AE08DF80E
:1037D0004B308DF84D301EF035F9204614B0BDE861
:1037E000F0870020FAE700000A4B10B5044603609A
:1037F000FFF7F2FE07F06EFE04F5247006F076FD8A
:1038000004F17C0006F072FD04F1700006F06EFD1C
:10381000204610BD2879060810B50446FFF7E4FFDE
:103820004FF4956120460AF071FB204610BDFFF76A
:103830000BBF0000034B10B50446036006F016FCF6
:10384000204610BD4478060810B50446FFF7F2FF85
:10385000282120460AF05AFB204610BD034B10B524
:103860000446036006F002FC204610BD14780608EA
:1038700010B50446FFF7F2FF342120460AF046FB5C
:10388000204610BD034B10B50446036006F0EEFB66
:10389000204610BD2C78060810B50446FFF7F2FF4D
:1038A000382120460AF032FB204610BD38B51E4BA9
:1038B0000D4604464FF400721968C0F80F1099883D
:1038C0009B79A0F8131002214375284606F06AFC84
:1038D0004FF4007220730221284606F068FC4FF472
:1038E000007260730321284606F05CFCA073284632
:1038F00006F0FCFB20B9AF220C490D4809F0AEFBE5
:1039000004F185020023C4F8882204F2992284F885
:10391000783084F88430C4F88C3284F89832C4F853
:103920009C24C4F8A03438BD6078060804790608E1
:103930000F7906082DE9F34104460E461546FFF7B8
:1039400083FEF28823799A4237D1002D35D17778DA
:10395000012F2ED1F378202B27D13289072A24D1A9
:1039600004F10F0804F11605404629461EF038F808
:10397000D0B1D4F81630C4F80F30638B207CE17BD3
:10398000A4F8133001EB0021E57C607C237F01EB80
:1039900000410095A07C2568637501EB0061237DE3
:1039A0002046627D6D6BA8473D46F378212B08BF0A
:1039B0000125284602B0BDE8F0810025F9E710B5E1
:1039C0000446FFF741FEFFF707FE217B07F026FCC8
:1039D00004F1850304F17C00C4F888320023C4F8A4
:1039E0008C3284F8843006F036FC94F884302BB99D
:1039F00023682046DB6BBDE81040184710BD00006F
:103A000070B50446FFF720FED4F8A0542DB140F263
:103A1000DD120F490F4809F021FB04F29923C4F885
:103A20009C34FFF7D9FD617B07F054FB84F8985272
:103A3000C4F8A00404F5247006F00DFC94F8983244
:103A40002BB9236820469B6BBDE87040184770BDBA
:103A5000047906086C78060802232DE9F0414371C9
:103A600000230446054683609046144B04F17C060F
:103A700045F8703B284606F0E1FB304606F0DEFBD9
:103A800004F52477384606F0D9FBC4F8A484FFF780
:103A9000A3FD2146FFF758FD0CE0384606F026FC52
:103AA000304606F023FC284606F020FC1AF0D0FD34
:103AB000F6E7F8E72046BDE8F08100BF2879060860
:103AC00070B504460D46FFF7BFFD84F87850002D11
:103AD0003ED194F8843033B1FFF77EFD217B07F0AF
:103AE00071F984F8845004F1850304F17C06002503
:103AF0003046C4F88832C4F88C5206F0ACFB30462D
:103B000006F0A2FB28B94FF4A2721449144809F038
:103B1000A5FA94F8983233B1FFF75EFD217B07F0E8
:103B200051F984F8985204F2992304F52475C4F8E5
:103B30009C3400232846C4F8A03406F08CFB2846A9
:103B400006F082FB20B94FF4A77204490548DEE76E
:103B500004F17000BDE8704006F07DBB04790608F2
:103B60007A7806088B78060810B50446FFF76CFDD6
:103B700000212046BDE81040FFF7A2BF38B50D4632
:103B80000446FFF761FD042D05D020460021BDE865
:103B90003840FFF795BF38BDF8B5164604460D46C8
:103BA0001F46FFF751FD0423EA88337023799A42B8
:103BB00025D16978012922D1EA78212A08D0222A40
:103BC0000BD0202A4FF000001BD13070163401E0DA
:103BD0000F34317007203C60F8BDAB88204613F0ED
:103BE000010308BF1946FFF76BFFAB8803F0010321
:103BF000E366AB8803F00203A36602233370002060
:103C0000EAE703233370E7E710B58AB00446FFF70D
:103C10000BFD684606F01AFA0D4B694604F1700078
:103C20000093099406F02FFB2046FFF705FD094B92
:103C3000002168461A6806F0CFF96846FFF7FAFDDA
:103C40000AB010BD6846FFF7F5FD1AF001FD00BF90
:103C5000447806086878060870B58EB004460E46AB
:103C60001546FFF7E1FC01A806F0F0F9114B01A998
:103C700004F17C00019300230C958DF83430CDE9DC
:103C80000A4606F000FB2046FFF7D6FC0A4B00214F
:103C900001A81A6806F0A0F904E001A8FFF7DEFD0C
:103CA0001AF0D6FC9DF8344001A8FFF7D7FD204656
:103CB0000EB070BD147806086878060810B5044682
:103CC000FFF7C2FC94F884307BB9D4F88C3263B12E
:103CD000FFF782FCD4F88C3204F18502217B07F0D7
:103CE00039FA10B1012384F8843010BD2DE9F8436E
:103CF0001E460446894690469DF82070FFF794FCC6
:103D00000023336094F87830E3B194F88430CBB971
:103D1000D4F88C52C5F50075454528BF4546B8F125
:103D2000000F05D02A464946D4F888021DF08AFEC5
:103D3000D4F88C322B44C4F88C32356017B120464D
:103D4000FFF7BCFF2046BDE8F843FFF775BCF0B5B0
:103D50000446406A85B0012690F878502DB984F861
:103D600030503546284605B0F0BD04AB0027D4E9F5
:103D70000A1243F8047D0096FFF7B8FF0399E36A3F
:103D8000A26A5B1A0A44E362A26213B984F8306043
:103D9000E8E7606A3D46FFF791FFE3E72DE9F0436E
:103DA0001C4691B0054689469046FFF73DFC002C25
:103DB0004FF0000602A806BF01AC012700272660CD
:103DC00006F044F9134B02A905F5247002938DF80F
:103DD0003C708DF83D60CDE90B59CDE90D8406F0BE
:103DE00052FA2846FFF728FC0B4B314602A81A6806
:103DF00006F0F2F804E002A8FFF744FD1AF028FCF0
:103E00009DF83D4002A8FFF73DFD204611B0BDE8FA
:103E1000F08300BF2C7806086878060810B5D0F843
:103E2000A034044673B990F898325BB9FFF7D4FB1D
:103E30004FF4007304F29922617B07F0EBF8012341
:103E400084F8983210BD70B504461E46002308461B
:103E5000336094F87830EBB194F89832D3B9D4F851
:103E6000A054D4F89C14954228BF15462A461DF04C
:103E7000E9FD3560D4F89C34D4F8A0242B44551BBC
:103E8000C4F89C34C4F8A05425B92046BDE870405D
:103E9000FFF7C4BF70BD37B50446406A90F878504C
:103EA0002DB984F835500125284603B030BD02AB4A
:103EB000002243F8042DD4E90A12FFF7C4FF019948
:103EC000A26A0A44A262226B13680B441360019930
:103ED000E36A5B1A94F83410E36209B9126802B914
:103EE0001BB9012384F83530DEE7606A0025FFF74F
:103EF00095FFD9E710B50446FEF776FA204610BDC7
:103F000010B4D0E9003409686210E4075DF8044B8E
:103F100001EB020044BF8A58D358184701460430C9
:103F200008B5FFF7EDFF08BD034A0346C26007C9A5
:103F300083E80700704700BF5478060810B586B0C4
:103F400004460391684606A980E80C0001E90C00CC
:103F5000204603A9FFF7E8FF204606B010BD37B59D
:103F60006C46054684E80C0094E80C00FFF7E6FF79
:103F7000284603B030BD0000F0B58BB00546FFF712
:103F800063FB06ACFFF728FBAF7B0646002120460B
:103F9000FFF7B0FF009403234FF400723946304618
:103FA00006F08AFE2046FDF7CCFCFFF715FB234BFD
:103FB00006462F7B0293002329462046039302AB3B
:103FC0000CCBFFF7CCFF009402234FF4007239466C
:103FD000304606F071FE2046FDF7B3FCFFF7FCFA11
:103FE000174B06466F7B0493002329462046059312
:103FF00004AB0CCBFFF7B3FF009402234FF4007225
:104000003946304606F058FE06E02046FDF799FC9A
:104010001AF01EFBF9E7F8E72046FDF792FCFFF7E0
:10402000DBFA4FF40073D5F89C24697B06F0F2FFAD
:10403000012085F898020BB0F0BD00BFBF3904081D
:10404000013A040808B5FFF769FF08BD08B5FFF796
:10405000F9FF08BD6FF01500704700290CBF6FF025
:10406000180000207047012070476FF0150070475E
:104070006FF0150070471120704770477047704708
:1040800003689B6C1847A0F59860F9E77047704784
:104090007047704710B50446012000F03DFD94F8CC
:1040A000780010BDA0F59860F4E7000038B54FF037
:1040B000FF320123FF210B480AF0C4F80A4D00F03B
:1040C0000DFD044695F878301BB1012000F024FD69
:1040D000F8E700F003FD001BC728F6D9BDE838401B
:1040E000FEF7BCBC98400024603A002407B502AB40
:1040F000012243F8041D1946FFF7AEFD18B10198DF
:1041000003B05DF804FB4FF0FF30F9E7A0F59560D0
:10411000FFF7ECBF07B5002302A9012201F8013D1A
:10412000FFF73CFE20B19DF8070003B05DF804FBEB
:104130004FF0FF30F9E7A0F59560FFF7EBBF2DE9F1
:10414000F8430446884617461E46089DFFF77CFA4A
:10415000D4F8F095B9F1000F04D02B463246394619
:104160004046C847C4F8E085C4F8E475C4F8E8657B
:10417000C4F8EC55BDE8F883B0F5966F03D1012182
:1041800001480AF041B87047984000240068704721
:104190000C30704708B5FFF7FBFF0023036008BD34
:1041A000CB68C3600BB15B681847704738B50546EC
:1041B000FFF73AFA95F898325BB9D5F8A044B4F510
:1041C000007F28BF4FF400742846FFF735FA2046D9
:1041D00038BD0024F8E790F878007047114B03F1E0
:1041E000780270B503600446C0F8A82400F2F456C3
:1041F00003F1D80200F23465E833C0F8AC24C0F80B
:10420000C034AE4204D0103D2846FDF79AFBF8E7D3
:1042100004F5956008F096FB2046FFF7E5FA204686
:1042200070BD00BF447A0608A0F59560FFF7D6BFC1
:10423000A0F2AC40FFF7D2BF10B50446FFF7CEFFA7
:104240004FF4C761204609F061FE204610BDA0F280
:10425000AC40FFF7F1BFA0F59560FFF7EDBF0000A0
:104260002DE9F74304461E468846154615F0A6FC80
:10427000BDF82C3004F59567014601932A46BDF838
:104280002830204600933346FFF7E6FB00213846EE
:1042900008F02EFB4FF47A73002504F2F45904F56C
:1042A0009A60C4F8C8342946204B4E46C4F8C4541A
:1042B00003F178022360C4F8A82403F1D802E8339C
:1042C000C4F8AC244FF48072C4F8C0341DF0B8FCBC
:1042D000C4F8D055C4F8D455C4F8D85504F23465A0
:1042E00030461036FEF780F8B542F9D10023C4F805
:1042F0003436C4F8F035B8F1000F13D02046FFF77C
:1043000083FC0FE04D4504D0103D2846FDF719FB16
:10431000F8E7384608F016FB2046FFF765FA1AF072
:1043200097F9F9E7204603B0BDE8F083447A060820
:10433000884238B5044606D00D46FDF7FDFA204602
:104340002946FFF72DFF204638BD08B5FFF720FFAF
:104350000068003018BF012008BD000010B50446F9
:10436000FFF7F3FF28B940F202220649064808F099
:1043700075FEE068FFF70AFF03462046BDE81040DF
:10438000184700BF227A06082D7A0608F8B50646B7
:104390000025FFF759F906F2F454D6F83436AB424B
:1043A0000AD920462746FFF7D0FF103420B13846FF
:1043B0000135FFF7D3FFF0E7F8BD0000044BC36001
:1043C00003460A6843F8042B002242605A60704793
:1043D0008C79060813B50446019121B9FFF7DAFE7E
:1043E000204602B010BD01A9FFF7E8FFF8E710B4BE
:1043F000D0E9003409686210E4075DF8044B01EB72
:10440000020044BF8A58D35818470146043008B503
:10441000FFF7EDFF08BD0000034A0346C26007C96D
:1044200083E80700704700BF8079060810B586B0A2
:1044300004460391684606A980E80C0001E90C00D7
:10444000204603A9FFF7E8FF204606B010BD37B5A8
:104450006C46054684E80C0094E80C00FFF7E6FF84
:10446000284603B030BD00002DE9F04188B0044675
:10447000FFF7DAF8384B2046C4F8F035FFF7DCF8E0
:10448000364B04A8214602930023039302AB0CCBC6
:10449000FFF7DDFF2046FFF7C7F8D4F834060328FE
:1044A00003D92046FFF7C8F80AE0431C04EB0010CC
:1044B00004A9C4F8343600F2F450FFF739FFF0E7EE
:1044C00004A8FDF73EFABC2009F0ECFC05460646C0
:1044D000234B05F1400746F8043B3046FDF784FFC7
:1044E0000021384609F04EFF05F15408404609F016
:1044F000E9FE1C4B4FF480721821284600930023DC
:1045000009F0C8FF184904A8C4F8DC55FFF762FF9A
:1045100004A9284609F0CAFF10E0404609F010FF40
:10452000384609F058FF3046FDF70BFABC21284603
:1045300009F0ECFC1AF08CF8F2E7F4E704A8FDF7B8
:1045400000FA2046FEF774FC08B0BDE8F08104A82C
:10455000FDF7F7F9EEE7FAE779410408312E040890
:104560008495060898790608AD400408A0F598607F
:10457000FFF77ABF0368184708B5FFF7FBFF08BDD0
:1045800008B5FFF742FF08BD08B5FFF7F9FF08BD02
:1045900037B50F4C0F4D204609F026FE2A460E492E
:1045A000204609F02FFA42F2120301220B4CCDE90A
:1045B000003200224FF4F85320461146FFF750FE18
:1045C0002A460749204603B0BDE8304009F01ABA30
:1045D00098400024000000240FE20408603A002400
:1045E000DD41040808B51BF08BFE2DE9F04F027D7C
:1045F00085B005460E46012A40F08E8000214FF01E
:10460000FF3B04460B465F4694F804C048B2BCF139
:10461000000F73D194F805C0BCF1000F6ED1B7F153
:10462000FF3F17BF0133012338465BB2934201DDE0
:104630001A4683460131023408295DD1002402EB79
:104640000B03A1460293CB4502DC029B4B4558DC91
:1046500095F8058095F804A04FEA281708F00F0890
:104660000AF00F035FEA2A1AFAB201926FD05FFADA
:104670008AF1BAF1090F30460393D4BF3031573174
:1046800000F0CDF8039B0444092B3046039394BFFC
:1046900003F1300103F1570100F0C1F80444BAF10D
:1046A000000F02D1039B03B94FB1092F019F304680
:1046B000D4BF30375737F9B200F0B1F80444B8F13D
:1046C000090F304694BF08F1300108F1570100F09E
:1046D000A6F8B9F1070F044404D03A21304600F09F
:1046E0009EF8044409F101090235B9F1080FAAD175
:1046F000204605B0BDE8F08F074685E74FF0FF3054
:1047000098E7CB45EED1BBF1000FE6D13A21304618
:1047100000F085F80444E0E700F1100700F1130908
:10472000002417F8011B0A22304600F0E9F8804601
:104730002E21304600F073F8B94540440444F0D1CE
:104740000A22E97C304600F0DBF80444D0E7002B75
:104750009AD1A9E7054B102210B5044603600175F4
:10476000002104301DF06CFA204610BD607B060865
:1047700070B5074D8374056000259DF810300575F0
:1047800045608560C56001744274C37470BD00BF2C
:10479000607B060807B501210648FFF7DBFF002311
:1047A00005481A4619460093FFF7E2FF03B05DF88B
:1047B00004FB00BFAC400024C44000242DE9F041BC
:1047C00006460D4601EB02080C464445A4EB0507DE
:1047D00007D03368304614F8011B1B68984700283F
:1047E000F3D13846BDE8F08170B5044608460D4661
:1047F0001DF026FF23680246294620465B68BDE877
:104800007040184709B1FFF7EFBF0846704708B579
:10481000FFF7F8FF08BD08B5FFF7F4FF08BD036810
:104820001B6818470B460A6801461268184610476D
:104830000149FFF7D9BF00BFCDC6060838B5054608
:10484000FFF7E0FF04462846FFF7F2FF204438BD9B
:1048500038B50546FFF7D6FF04462846FFF7E8FFC0
:10486000204438BD70B58AB00D460023012A98BF98
:104870000A220AA901F8043DB5FBF2F402FB145622
:104880002546F3B2092E94BF30333733DBB201F83B
:10489000013D002CF0D1FFF7B5FF0AB070BD2DE946
:1048A000F04107460E4615462AB90368C9B21B688F
:1048B000BDE8F04118470A2A05D1002905DBBDE80B
:1048C000F041FFF7CFBFD2B2F9E72D21FFF7A7FFE5
:1048D00004462A4671423846FFF7C4FF2044BDE82B
:1048E000F081FFF7DCBF10B42AB90368C9B25DF8E4
:1048F000044B1B681847D2B25DF8044BFFF7B2BFF8
:10490000FFF7F1BF0000000070B52DED068B0A9D8A
:10491000064643EC182BB4EE488B002DB8BF022599
:10492000F1EE10FA06D73C49BDEC068BBDE87040AD
:10493000FFF75ABFB0EEC87B9FED316BB4EE467BFC
:10494000F1EE10FA01DD3549EEE79FED2F7BB4EE75
:10495000C78BF1EE10FA02DD31493046E4E79FEDF6
:104960002C7BB4EEC78BF1EE10FAF5D4B5EEC08B0C
:10497000F1EE10FA11D52D21B1EE488BFFF74FFF64
:104980000446B6EE007B0023B2EE046BDAB20133CC
:10499000AA4204DA87EE067BF8E70024F1E738EE56
:1049A000078B0A223046BCEEC89B19EE101AFFF79F
:1049B00059FF0444EDB1B8EE499B1A493046B2EEB6
:1049C00004ABFFF711FF044438EE498B15F1FF35B6
:1049D0000FD328EE0A8B0A223046BCEEC89B19EE94
:1049E000101AFFF73FFFB8EE499B044438EE498B9D
:1049F000ECE7BDEC068B204670BD00BFAFF3008036
:104A0000FFFFFFFFFFFFEF7F000000E0FFFFEF4130
:104A1000000000E0FFFFEFC1647B0608687B06082A
:104A20006C7B0608C4870608FFF76EBF37B506998A
:104A300005460091FFF768FF04462846FFF7F8FE99
:104A4000204403B030BD000010B500F069F80A4CF6
:104A5000FEF752F8FEF7C0FDFEF7B5FD4FF4E13169
:104A60000648FFF701FDFCF771FBFCF779FB002C12
:104A7000FBD0AFF30080F8E700000000603A0024AC
:104A800070B505460024074EFDF76EFFE3B298426D
:104A900006D918461B010134F35EAB42F4D170BD58
:104AA000FF20FCE75C00002410B50446FDF75CFF26
:104AB00084423BBF2401024B4FF0FF30185F10BD12
:104AC0005C00002410B5044605F0E0F8204610BD57
:104AD00010B5044605F0DAF8204610BD07B50749C1
:104AE000684605F010F94FF47A720023DDE9000101
:104AF0001AF000F903B05DF804FB00BFE0400024A9
:104B000007B50449684605F0FEF8009803B05DF863
:104B100004FB00BFF840002409F064BC09F040BB6E
:104B200008B5044805F0BCF80348BDE8084005F0A6
:104B3000B7B800BFF8400024E040002409F062BC90
:104B400038B50A4C0A4D204605F01AF92046094CA2
:104B50002A46094908F056FF204605F01CF92A4666
:104B600020460649BDE8384008F04CBFF840002414
:104B700000000024E0400024D14A0408C54A04088B
:104B800070B504460D46164600211C221DF058F84B
:104B900020463246294607F002F9204670BD000043
:104BA0002DE9F04104460E46FDF7DEFE84423CD27C
:104BB0001F4D2701EA19D06810B11C2109F0A6F990
:104BC0002046FFF771FF80461C2009F06BF9044670
:104BD00000211C221DF034F84146204607F0DCF885
:104BE000EB19012EDC6010D006D3022E12D0204625
:104BF00003F05CFF022103E0204603F057FF002191
:104C00002046BDE8F04103F05DBF2046BDE8F0411D
:104C100003F040BF204603F049FF0121F0E71C21CB
:104C2000204609F073F919F013FDBDE8F08100BFCB
:104C30005C00002430B589B004460D46FFF720FF24
:104C4000C0B2FF2804D02946FFF7AAFF09B030BD43
:104C5000012D14D00AD3022D1CD00222214601A816
:104C6000FFF78EFF01A807F021F8EFE700222146A9
:104C700001A8FFF785FF01A807F018F8E6E71C2256
:104C8000002101A81CF0DCFF0022214601A807F04A
:104C900088F8DBE70122214601A8FFF771FF01A890
:104CA00007F004F8D2E700002DE9F34106460F466D
:104CB000FDF75AFE86422AD21B4D4FEA061805EB35
:104CC0000802D468ACB93046FFF7EEFE06461C2059
:104CD00009F0E8F804461C2200211CF0B1FF0097FF
:104CE000002301223146204607F062F805EB080355
:104CF000DC600E4B0E491A46D3F894008842FBD173
:104D000023683FB1A1680B604FF44073536102B058
:104D1000BDE8F081E1681B04F5E71C21204609F09D
:104D2000F5F819F095FC00BF5C00002400640258FF
:104D30000003008030B589B005460C46FFF7A0FEA1
:104D4000C0B2FF2804D02146FFF7AEFF09B030BD46
:104D50001C22002101A81CF073FF294601A807F0BE
:104D600024F8094B09491A46D3F894008842FBD12C
:104D7000019B2CB103990B604FF440735361E5E73D
:104D80001B040499F7E700BF006402580003008089
:104D90001EF0040F0CBFEFF30880EFF30980816968
:104DA00011F8021C002932D101B590E80F10E0473C
:104DB000BDE800508CE80300244B93E806009142C4
:104DC00008BF70471A6041B91EF0100F10D1204B78
:104DD000186820F0010018600AE02CE9F00F1EF0BE
:104DE000100F08BF2CED108A81F822E0C1F838C0FE
:104DF000906B92F8221061F0FF0E1EF0100F08BFAA
:104E0000B0EC108AB0E8F00F80F309887047114ABF
:104E100013689942FAD801B552F821C00FC8E0478B
:104E2000BDE80050CCF80000704701B501F0C6FBAA
:104E3000BDE80140EFF3098CBEE701B501F082FB4C
:104E4000BDE80140EFF3098CB6E70000900C0024A8
:104E500034EF00E0247C0608014608B530B96FF055
:104E6000030000F01FFA6FF0030008BD132001F0EB
:104E700079FF30B94FF0FF3000F014FA4FF0FF30F7
:104E8000F3E70020F1E7000008B5EFF305834BB925
:104E9000EFF3108333B9EFF311831BB9DFF814C0BC
:104EA00000DF08BD6FF0050000F0FCF96FF00500B1
:104EB000F7E700BF594E0408EFF310832BB9EFF367
:104EC0001180003818BF012070470120704710B5CD
:104ED00020B10378F32B01D1002906DA6FF003012A
:104EE00002F038FA6FF0030010BD00F10C0353E834
:104EF000000F20EA010243E8002404B1F7E7F3E7DA
:104F0000034610B528B30468806860B110F003024E
:104F100002D1DB680F2B25D86FF00801002002F0CA
:104F200019FA002014E0DB68002BF5D1104BD3F800
:104F3000900080B100F084FCB0B10123F3228370B3
:104F40000023446002700B4AC0E90233084B5A66E2
:104F500010BD0446EAE701221021D3F8800000F0DA
:104F6000FAFBE9E71346E9E76FF00401D7E700BF72
:104F70007C0C00244950040810B5044610B1037895
:104F8000F32B07D020466FF0030102F0E3F96FF036
:104F9000030010BD836863B1204601F06BFC002262
:104FA0006FF0020101F0FAFDA0680028F4D101F0D1
:104FB000E9FC00232370A378DB0701D40020E8E795
:104FC000064B2146D3F8900010B100F054FCF5E7F1
:104FD000D3F8800000F0F3FBF0E700BF7C0C002466
:104FE000930710B502F0010422D400F10C0384B140
:104FF00053E8000F00EA01028A4203D0BFF32F8F6B
:10500000002005E020EA010243E8002404B1EFE7B4
:1050100010BD53E8000F084203D1BFF32F8F0020CB
:1050200005E020EA010243E8002404B1F1E7EFE7DC
:10503000C06800EA01031CB1994218BF0020E7E7ED
:10504000002B08BF0020E3E7F8B50546846804B9E3
:10505000F8BD94F823202846616AA768FFF7C0FFCF
:10506000064638B1204601F00EFC002231462046AB
:1050700001F094FD3C46EAE7F8B50D4617461E469A
:10508000044620B10378F32B01D1002907DA20462A
:105090006FF0030102F05EF96FF00300F8BDFFF757
:1050A0009FFF0028FAD186B13146432001F05AFE15
:1050B00040B1074B20465E69314601F0C9FB75627D
:1050C00086F823706FF00100E8E76FF00200E5E773
:1050D0007C0C00242DE9F041064620B10378F32B27
:1050E00001D1002909DA6FF003056FF003013046A2
:1050F00002F030F92846BDE8F08100F10C0353E8D6
:10510000002F42EA010543E8005000B1F7E7B46818
:105110001CB9204601F036FCECE794F82320304619
:10512000616AD4F80880FFF75BFF074678B194F80E
:1051300023309B0756BF656A054620EA05052046D1
:1051400001F0A1FB00223946204601F027FD44462C
:10515000DEE70000024608B5EFF3058333B1002017
:105160006FF0050102F0F6F8002008BDFFF7A4FE7D
:105170000028F4D11046DFF808C000DFF5E700BFD3
:10518000014F040838B502460D46EFF305834BB1D5
:1051900092B96FF003046FF00301104602F0DAF8E1
:1051A000204638BDFFF788FE0028F1D11046DFF811
:1051B00030C000DF0446F3E71378F32BE9D1002D6C
:1051C000E7DB02F10C0353E8001F41EA050443E862
:1051D000004000B1F7E7104601F038FAE0E700BF01
:1051E000D550040810B502460C46EFF305832BB1E9
:1051F00021461046BDE81040FFF769BEFFF75CFE90
:105200000028F5D11046DFF808C000DF10BD00BF50
:10521000CF4E0408F8B504460E4617461D46EFF378
:10522000058343B18CB920466FF0030102F092F878
:105230006FF00300F8BDFFF73FFE0028F2D12046D3
:105240002B46DFF828C000DFF4E72378F32BEAD100
:10525000002DE8D1002EE6DB3A4631462046FFF726
:10526000BFFE002808BF6FF00200E3E77950040892
:10527000024608B5EFF305833BB110466FF0050118
:1052800002F068F86FF0050008BDFFF715FE002872
:10529000F3D11046DFF804C000DFF5E7794F0408CA
:1052A000704770477047EFF310832BB9EFF311800D
:1052B000003818BF0120704701207047064BDA6A9A
:1052C0003AB1D0695B6C1BB11B69984228BF184684
:1052D00070474FF0FF30F5E77C0C0024014BD86895
:1052E000704700BF7C0C002408B5094B1A7A022ACB
:1052F00008D0032A0AD04FF0FF3002F01FF84FF019
:10530000FF3002E0032200201A7208BD0120FCE7F2
:105310007C0C002408B50A4B1A7A023A012A02D8FA
:1053200040B1012809D04FF0FF3002F007F84FF0EC
:10533000FF3001E002221A7208BD0322FBE700BF22
:105340007C0C002470B5464C237A012B00F085803C
:1053500033B14FF0FF3001F0F1FF4FF0FF3070BD7F
:10536000404DEB68E3652B8AD5E90B61A4F8543016
:10537000AB683046236400F0D7F908B1C4F8806008
:10538000D5E90561304600F0CFF908B9D4F880605E
:105390006667D5E90761304600F0C6F908B9D4F868
:1053A0008060A667D5E90961304600F0BDF908B90B
:1053B000D4F88060E6676E6B3EB131683046D6E95E
:1053C000022300F01CFAC4F88460AE6B3EB1316871
:1053D0003046D6E9022300F012FAC4F88860EE6B7A
:1053E0003EB131683046D6E9022300F008FAC4F82D
:1053F0008C602E6C3EB131683046D6E9022300F055
:10540000FEF9C4F890606E6C3EB131683046D6E962
:10541000022300F0F4F9C4F89460AE6C3EB1316838
:105420003046D6E9022300F0EAF9C4F89860EE6C41
:105430003EB131683046D6E9022300F0E0F9C4F805
:105440009C602D6D3DB129682846D5E9022300F006
:10545000D6F9C4F8A0500123237200207FE700BFD3
:105460007C0C0024B47B060870B5254D2B7A012BEB
:1054700007D06FF006004FF0FF3401F05FFF2046C9
:1054800070BD01F0E1FC10B94FF0FF30F3E71D4AA9
:10549000FF231D4E82F8223092F82230D26863F04A
:1054A000FF031A49C2F302227068DB4314BFB3FA48
:1054B00083F32023C3F12003934298BF531CFE22A1
:1054C00002FA03F30F4ADBB2D37701F093FF0446ED
:1054D0000028D9D101F0E6FF286101F0CFFF0C4888
:1054E00001F0C8F901F046FA3368DB074CBF02232C
:1054F000032383F31488BFF36F8F02232B72BEE75D
:105500007C0C002400ED00E0B47B06083B4E040850
:10551000980C002410B50F4C237A022B13D101F004
:10552000B5FF01236372BFF34F8F0B4A5168C90067
:1055300003D54FF000615160A37204232372BDE8CC
:105540001040FFF7BBBE6FF0070001F0F7FE002030
:1055500010BD00BF7C0C002400ED00E038B51D4CF0
:105560000546237A042B34D1FFF7A8FEE26A854270
:105570002CBF00F1FF332B4612B1D069C01AD061A5
:10558000626C12B11069C01A1061E26813441544CC
:10559000E360E3689D4213D102230020237201F0EF
:1055A000F1F900236372BFF34F8FA27A22B1A37285
:1055B0004FF08052084B5A60BDE8384001F05EBFA2
:1055C0000133E36001F09CF9236D002BE1D0984793
:1055D000DFE738BD7C0C002400ED00E0704738B5F3
:1055E00004460D46FFF75CFE29462046BDE83840DC
:1055F00001F066BE08B5FFF7F1FFEFF3058333B1A5
:105600006FF0050001F09AFE6FF0050008BDFFF78E
:105610004AFE0028F4D1DFF808C000DFF6E700BF3B
:105620004553040808B5EFF3058333B16FF0050067
:1056300001F084FE6FF0050008BDFFF734FE00287E
:10564000F4D1DFF808C000DFF6E700BF69540408B2
:1056500008B5EFF3058333B16FF0050001F06EFE7E
:105660006FF0050008BDFFF71EFE0028F4D1DFF83B
:1056700008C000DFF6E700BFE9520408024608B59B
:10568000EFF3058333B16FF0050001F057FE6FF0C3
:10569000050008BDFFF707FE0028F4D11046DFF82B
:1056A00008C000DFF5E700BF1553040808B5EFF3A5
:1056B00005832BB16FF0050001F040FE002008BD0E
:1056C000FFF7F1FD0028F5D1DFF804C000DFF6E7B1
:1056D00015550408024608B5EFF305832BB16FF0AA
:1056E0000500BDE8084001F029BEFFF7DCFD0028F9
:1056F000F5D11046DFF804C000DF08BD5D55040891
:1057000008B5EFF3058313B1054BD86808BDFFF763
:10571000CAFD0028F8D1DFF80CC000DFF6E700BFB3
:105720007C0C0024DD520408034610B588B1084300
:1057300010F007000DD117290AD919600839102275
:10574000CC185A609C60585099684A60D860012013
:1057500010BD0020FCE7034670B570B369B3032A9F
:105760002BD80F3100F1080421F0070621462468E8
:105770004D68601A25F00305401B864203D9206856
:105780000028F3D170BD5D683243186835445D6010
:10579000034453F8040C083B854288BF5D604B68A6
:1057A0001BB901F108004A60ECE723F00303C818B5
:1057B000CC50426008600830E4E70020E2E703468E
:1057C00010B580B1C9B1A1F1080400F108020021AF
:1057D000A24209D1506820F003045868001B5860A9
:1057E00041B95160012010BD106811460028FAD05F
:1057F0000246EDE713680B60F4E70846F3E730B5BF
:10580000C0B189B1C2B1CBB100240160C3604361B2
:10581000C0E9014202FB01F41D1905611846013976
:1058200004D1A41A19510121084630BD851805601C
:105830002846F4E70146F7E71146F5E71946F3E78E
:1058400010B570B100F1140353E8002F12B9BFF383
:105850002F8F04E0116843E8001404B1F4E70AB99B
:10586000104610BD043050E8003F591C40E80014B9
:1058700004B1F8E7F4E730B5F0B1C3688B421BD848
:1058800003698B4218D900F114031A680A60BFF348
:105890005F8F53E8002F0C689442F6D143E800155F
:1058A00005B1F2E7043050E8003F5A1E40E80021FD
:1058B00001B1F8E7002030BD6FF00300FBE7EFF324
:1058C00010832BB9EFF31180003818BF0120704707
:1058D00001207047D1E9013223B19A608A681AB178
:1058E00053607047C262F9E7036370472DE9F84FD0
:1058F0008846074638B131B1B0FA80F1B8FA88F37A
:105900000B441F2B08DC6FF003010024002001F082
:1059100037FD2046BDE8F88F08F1030626F00306A0
:105920000C3606FB00FAF2B19468D2F80090D2E986
:1059300004533CB1A10702D1D268332A05D86FF0D5
:105940000801E2E7D268002AF9D13DB115F0030B56
:1059500001D19A4552D96FF00901D6E7002BFAD14F
:105960001CB19B460CE091461546264BD3F8A0008F
:10597000D8B1FFF765FF0446A0B14FF0010B35BB6E
:10598000204B00225146D86FFFF7E5FE0546C0B90F
:10599000BBF1000F06D01B4B2146D3F8A00058B135
:1059A000FFF769FF6FF00401AFE701223421D3F85C
:1059B0008000FFF7D0FEDEE7D3F88000FFF7FFFEA0
:1059C000F0E74BF0020B524600211CF039F9FA23A4
:1059D0003246394604F10C002370002384F802B0EB
:1059E000A360C4F80490C4E90983C4E90B332B46CF
:1059F000FFF705FF034B044A1A678AE7002CE6D13C
:105A0000B3E700BF7C0C0024995A040800F1280376
:105A100010B553E8002F12B9BFF32F8F04E0511EC9
:105A200043E8001404B1F4E70AB9002010BDC06ACD
:105A300001220028F9D0811CD1E84F3FC1E8442F52
:105A400004B1F9E7DBB2002BF0D08068F1E7036B1B
:105A500030B5E3B1CD780024DA78AA420FD31A46E4
:105A6000C1E901248AB19160A4B16160283050E895
:105A7000003F5A1C40E8002101B1F8E730BD5A68E8
:105A80001C46002AECD01346E6E7C162ECE7C1E908
:105A90000133C1620163E9E7F8B5877804468FB343
:105AA000C568002701462846FFF714FF277005F157
:105AB0000C042046FFF7DFFEAB68002B48D02046E1
:105AC000FFF7BEFE0446002842D0284600F0D2FE72
:105AD00006463A46394601F061F8304600F040FF8C
:105AE0006A6A0646816804F10C001BF0ABFFF923DB
:105AF000A7702370F368E37021462846BDE8F8409C
:105B0000FFF7A5BF8568AB68002BF5D05B78832BCA
:105B1000F2D1284600F0AEFE06463A46394601F07C
:105B20003DF8304600F01CFF06466A6A04F10C019D
:105B300080681BF087FFF3680BB1E2781A700023CE
:105B4000214605F10C002370BDE8F840FFF793BE35
:105B5000F8BD00002DE9F0410E4617469846044670
:105B600018B10378FA2B00D141B920466FF0030138
:105B700001F006FC6FF00300BDE8F0818368BBB163
:105B80005B78832B14D100F075FE054601220021BD
:105B900001F004F8284600F0E3FE0546626A31464B
:105BA00080681BF04FFFEB6803B11F700020E3E734
:105BB00004F10C00FFF744FE054670B13146626AFD
:105BC0000C301BF03FFFF923294620462B700023A1
:105BD000EF70AB70FFF73BFFE8E7B8F1000F11D0B3
:105BE0004146932001F0BEF810B96FF00100C3E701
:105BF000064B2046596900F02BFEEFF30983C3E9F9
:105C00000267F2E76FF00200B6E700BF7C0C0024E9
:105C10002DE9F0410F4616469846044618B1037820
:105C2000FA2B00D141B920466FF0030101F0A8FB27
:105C30006FF00300BDE8F081FFF7E8FE054600289D
:105C40003AD001462046FFF745FE626A05F10C0195
:105C500038461BF0F7FE0EB1EB783370002704F1E5
:105C60000C06294630462F70FFF705FEA3680BB9D6
:105C70000020DFE73046FFF7E3FD05460028F7D0B8
:105C8000204600F0F7FD06463946012200F086FF67
:105C9000304600F065FE626A0646816805F10C0038
:105CA0001BF0D0FEF923AF7029462B702046F36815
:105CB000EB70FFF7CCFEDBE7B8F1000F11D04146E7
:105CC000832001F04FF810B96FF00100B2E7064BE6
:105CD0002046596900F0BCFDEFF30983C3E9027661
:105CE000F2E76FF00200A5E77C0C002408B5064B34
:105CF00008219A6ED86EFFF7F9FD044BD864B0FA0C
:105D000080F04009404208BDB47B06087C0C0024AA
:105D10002DE9F04106460F4690461C46EFF30583F9
:105D20004BB196B930466FF0030101F029FB6FF0DB
:105D30000300BDE8F081FFF7C2FD0028F1D1304635
:105D40002346DFF848C000DFF3E73378FA2BE9D1C8
:105D5000002FE7D0002CE5D106F10C00FFF770FD15
:105D6000054680B1726A39460C301BF06BFEF92390
:105D70002846AC702B7085F80380C5E9017600F0E9
:105D800065FC2046D5E76FF00200D2E7555B0408BA
:105D9000F8B504460F4616461D46EFF3058343B19A
:105DA0008CB920466FF0030101F0EAFA6FF00300AE
:105DB000F8BDFFF784FD0028F2D120462B46DFF81E
:105DC00044C000DFF4E72378FA2BEAD1002FE8D0B3
:105DD000002DE6D12046FFF719FE054670B100F10F
:105DE0000C01626A38461BF02DFE0EB1EB78337061
:105DF0002846EC6000F02AFC0020D9E76FF0020092
:105E0000D6E700BF115C0408EFF310832BB9EFF362
:105E10001180003818BF0120704701207047000032
:105E200038B5034698B3D0E90045806860B110F0FA
:105E3000030202D1DB681B2B24D86FF0080100207D
:105E400001F08EFA00201CE0DB68002BF5D1114B2D
:105E5000D3F8940030B901221C21D3F88000FFF759
:105E60007AFC01E0FFF7ECFC70B10123F5228370AE
:105E70000023C570027044600376C0E90233C0E9B4
:105E8000043338BD1346F1E76FF00401D8E7044648
:105E90000546DCE77C0C0024294B70B55D6904469F
:105EA0000E4635B96FF0070101F05AFA4FF0FF3096
:105EB00070BD10B10378F52B07D020466FF00301B9
:105EC00001F04EFA6FF00300F2E7037E53B9C0E928
:105ED0000353EB6A436103B118610123EC620020B4
:105EE0002376E5E7C278D1070DD5C168A9420AD16A
:105EF000FF2B06D16FF00F0101F032FA6FF00200B4
:105F0000D6E70133EBE7002EF8D093070AD5E06817
:105F100095F9203090F920209A4203DA80F8203059
:105F200000F0BAFC3146532000F01CFF10B96FF0AE
:105F30000100BDE72946204600F08AFCF7E700BFD4
:105F40007C0C00242F4B5A6970B5044632B96FF0AF
:105F5000070101F005FA4FF0FF3070BD10B1037872
:105F6000F52B07D020466FF0030101F0F9F96FF02F
:105F70000300F2E7037E33B96FF00E0101F0F0F990
:105F80006FF00200E9E7C168914202D06FF00D01A5
:105F9000F4E7013BDBB203760BB10020DDE7436998
:105FA0000BB1016919612169E9B14B6192F92130A5
:105FB000D56AD5B982F82030A36883B1204600F0B5
:105FC00059FC06462A46294600F0E8FDF36AC4E972
:105FD0000365636103B11C610123F4622376002031
:105FE00000F0D0FCD9E7D362E0E7E978890706D56D
:105FF000A96821B191F920108B42B8BF0B466D6999
:10600000D7E700BF7C0C002410B5044610B103781C
:10601000F52B07D020466FF0030101F0A1F96FF0D6
:10602000030010BD037EBBB16369C0680BB1226978
:106030001A612269BAB1536190F92120C36AA3B9E8
:1060400090F92030934203D080F8202000F024FC07
:10605000A068B0B900F096FC00232370A378DB079A
:1060600018D40020DDE7C362E6E7D978890706D5B2
:10607000996821B191F920108A42B8BF0A465B693C
:10608000DDE7204600F0F6FB00226FF0020100F091
:1060900085FDDDE7064B2146D3F8940010B1FFF7EC
:1060A000EAFBDEE7D3F88000FFF789FBD9E700BF02
:1060B0007C0C00242DE9F0410446002601270CB990
:1060C000BDE8F081E378D4F814801B0712D5A368EB
:1060D00026767BB1204600F0CDFB00220546114616
:1060E00000F05CFDEB6AC4E90356636103B11C6117
:1060F000EC6227764446E2E710B4C3789B071DD5CF
:10610000C06890F92120C36ADC78A40709D59C688F
:106110008C4208BF8C6824B194F92040A242B8BFD9
:1061200022465B69002BEFD190F92030934205D0D5
:1061300080F820205DF8044B00F0AEBB5DF8044B06
:1061400070470000024608B5EFF3058333B1002025
:106150006FF0050101F004F9002008BDFFF754FEBF
:106160000028F4D11046DFF808C000DFF5E700BFD3
:10617000215E0408024608B5EFF305833BB11046E3
:106180006FF0050101F0ECF86FF0050008BDFFF7B6
:106190003BFE0028F3D11046DFF804C000DFF5E72E
:1061A000995E0408024608B5EFF305833BB110463B
:1061B0006FF0050101F0D4F86FF0050008BDFFF79E
:1061C00023FE0028F3D11046DFF804C000DFF5E716
:1061D000455F0408024608B5EFF305833BB110465E
:1061E0006FF0050101F0BCF86FF0050008BDFFF786
:1061F0000BFE0028F3D11046DFF804C000DFF5E7FE
:1062000009600408EFF310832BB9EFF31180003815
:1062100018BF01207047012070470C30D0E85F3F65
:1062200013B9BFF32F8F04E05A1EC0E8512F01B1FC
:10623000F4E798B2003818BF0120704730B500F17C
:106240000C02C189D2E85F3F994202D8BFF32F8F79
:1062500004E05C1CC2E8554F05B1F3E7C0899BB26E
:10626000984294BF0020012030BD000070B54FF669
:10627000FE730D46411E0446994201D8A84206D23B
:106280006FF00301002001F071F8002070BD12B31F
:106290009068166840B110F0030302D1D2680F2A4B
:1062A0000DD86FF00801EDE7D368002BF9D1104B42
:1062B000D3F8980088B1FFF7C3FAA8B10123F622FA
:1062C000837000234660027083600A4A084B858110
:1062D000C4819A66DAE71646E9E701221021D3F86D
:1062E0008000FFF738FAE8E76FF00401CBE700BF62
:1062F0007C0C0024A963040810B5044610B103788F
:10630000F62B07D020466FF0030101F02FF86FF055
:10631000030010BD83683BB100F0ACFA01220021FC
:1063200000F03CFC0020F4E7FFF788FF0028F9D1DB
:1063300020466FF0100101F019F86FF00200E8E755
:1063400010B5044610B10378F62B07D020466FF045
:10635000030101F00BF86FF0030010BD836863B117
:10636000204600F087FA00226FF0020100F016FCD0
:10637000A0680028F4D100F005FB00232370A37867
:10638000DB0701D40020E8E7064B2146D3F898004C
:1063900010B1FFF770FAF5E7D3F88000FFF70FFAB6
:1063A000F0E700BF7C0C0024836810B504465BB1A5
:1063B000FFF733FF40B1204600F05CFA0022BDE851
:1063C0001040114600F0EABB10BD000038B50D4684
:1063D000044610B10378F62B07D020466FF0030176
:1063E00000F0C4FF6FF0030038BDFFF716FF68B977
:1063F00075B12946632000F0B5FC20B1064B20465C
:10640000596900F025FA6FF00100EDE70020EBE795
:106410006FF00200E8E700BF7C0C002410B50446D2
:10642000EFF3058333B100206FF0050100F09EFF0C
:10643000002010BDFFF7E6FE0028F4D12046DFF86B
:1064400008C000DFF5E700BF6D62040810B5024622
:106450000C46EFF3058343B182B910466FF0030198
:1064600000F084FF6FF0030010BDFFF7CBFE0028A3
:10647000F2D11046DFF820C000DFF5E71378F62BE5
:10648000EBD1002CE9D11046FFF7C7FE00280CBF66
:106490006FF002000020E7E7CD63040810B5044662
:1064A000EFF3058343B184B920466FF0030100F098
:1064B0005DFF6FF0030010BDFFF7A4FE0028F2D1CE
:1064C0002046DFF830C000DFF5E72378F62BEBD16C
:1064D0002046FFF7B3FE20B1204600F0B7F80020B9
:1064E000E9E720466FF0100100F040FF6FF0020076
:1064F000E1E700BFF9620408024608B5EFF305833F
:106500003BB110466FF0050100F030FF6FF0050061
:1065100008BDFFF777FE0028F3D11046DFF804C06E
:1065200000DFF5E74163040810B5D0E85F3F5A1C6F
:10653000914200D80022C0E8542F04B1F5E798B288
:1065400010BD000038B51C4C00F0A6FFE368013315
:10655000E36000F0D5F9002000F014FA236D03B1D8
:106560009847226C32B3A369E06BD969984202D094
:10657000E36301B9DA61DA69C2B9237A022B19D16E
:10658000656ABDB1E36B95F9202093F920309A42FA
:1065900010D1284600F077F9E06B00F08FF928461B
:1065A00000F0E8F9236CE563EB6103E0013ADA619E
:1065B000002AE2D038BD00BF7C0C002470B5224C0C
:1065C00004F1560504F15A06B4F85410D5E85F3FBB
:1065D00013B9BFF32F8F04E05A1EC5E8502F00B146
:1065E000F4E79BB25BB33046FFF79EFFE36D53F8D1
:1065F000200020B30378F13B082BE5D801A252F824
:1066000023F000BF29660408C96504082F66040842
:10661000C9650408C96504083366040837660408B8
:10662000C96504083B660408236E9847CCE7636E8F
:10663000FBE7A36EF9E7E36EF7E7236FF5E70020CA
:10664000BDE8704000F09EB97C0C002470B5164C7B
:106650000546B4F8541004F15602D2E85F3F99425F
:1066600002D8BFF32F8F04E0581CC2E8560F06B1C2
:10667000F3E79BB2994205D829460220BDE8704055
:10668000FEF7ADBF04F15800FFF74EFFE36D43F88E
:106690002050637A23B9054B4FF080525A6070BD89
:1066A0000123A372FBE700BF7C0C002400ED00E097
:1066B000EFF310832BB9EFF31180003818BF0120DE
:1066C0007047012070470378F12B00D07047C068F5
:1066D000F9E7000010B5C469621CD0E904310CD19F
:1066E00003B1596142691AB113610023436101E0AA
:1066F000074A13630023C36110BD1BB1DA695961F6
:106700002244DA614269002AEED1014AD362F1E7FC
:106710007C0C002401230A4A90F9201043701C329B
:10672000936810B51BB193F920408C4205DCC0E999
:106730000232906003B1D86010BD1A469B68F1E741
:106740007C0C0024014B5869704700BF7C0C00246E
:10675000002310B50380044683789A0708D513F008
:10676000100F016B0E4B0FD0D3F88400FFF783F8A6
:10677000A378DB0712D50A4B2146D3F8880038B13D
:10678000BDE81040FFF777B8586FFFF718F8EFE74C
:10679000D3F88000BDE81040FFF711B810BD00BF6E
:1067A0007C0C002408B500F0F1FDDFF810C000DF1C
:1067B0004FF0FF31002000F0C7FDFEE7056C040834
:1067C000930710B502F0010422D400F1280384B12C
:1067D00053E8000F00EA01028A4203D0BFF32F8F73
:1067E000002005E020EA010243E8002404B1EFE7BD
:1067F00010BD53E8000F084203D1BFF32F8F0020D4
:1068000005E020EA010243E8002404B1F1E7EFE7E4
:10681000806A00EA01031CB1994218BF0020E7E733
:10682000002B08BF0020E3E7C2780346D20701D45B
:10683000FFF78EBF0422054942700022C2604A6BF6
:10684000826002B1D0604B63704700BF7C0C0024B3
:1068500091F92020836810B51BB193F92040944230
:1068600005DAC1E90230816003B1D96010BD184674
:106870009B68F1E70346806882689A6002B1D36042
:106880000023C3607047C2682AB18368936003B174
:10689000DA600023C360704710B5044664B1237802
:1068A000F12B07D0FFF7EFFF01462046BDE810406F
:1068B000FFF7CEBFE468F1E710BD000001230146F9
:1068C00043700148FFF7C4BF980C002470B50B4D0E
:1068D0002E7A022E10D16C6A74B1696994F9202065
:1068E00091F920309A4207D12046FFF7CCFF0846A5
:1068F000FFF7E4FF6670AC61002070BD7C0C0024E3
:1069000038B5164DEC6A44B3E369013BE36123BB40
:106910006378732B06D009D8532B0BD003F0DF0319
:10692000432B0DD12046FFF7CEFE09E003F0EF0325
:10693000832BF6E720462146FFF7C5FEFFF7DCFB79
:106940002046FFF7A0FFFFF7B9FF246924B1E369F0
:10695000002BDDD000236361EC6238BD7C0C002489
:1069600090F82230826B13F0100F14BF20206020AB
:106970001044704702234370014B9861704700BF79
:106980007C0C002470B5124D04462E7A696990B9CA
:10699000022E0FD16C6A6CB194F9202091F920304D
:1069A0009A4207DD2046FFF76EFF0846FFF7B2FE6A
:1069B0006670AC6170BD022E05D190F9202091F96E
:1069C00020309A42F1DC2046BDE87040FFF776BFE8
:1069D0007C0C00242DE9F74F8246019140B96FF0FD
:1069E0000301002400F0B0FC204603B0BDE8F08FA6
:1069F000002A00F0868094689769D2E90093D2E972
:106A00000456009344B1A00702D1D368432B06D8A3
:106A10006FF008010020E4E7D368002BF8D13DB106
:106A2000690702D1002E40F09E806FF00A01F1E765
:106A30002FB17B1E372B03D96FF00B01EAE7182724
:106A4000002E40F09480002C68D14E4BD3F8880083
:106A500000285CD0FEF7F4FE0446002873D04FF007
:106A6000010BDFF8208185B9002E5AD1464AD8F8AB
:106A70008400566D002854D0FEF7E2FE054600283B
:106A800058D04BF0100B4BF0020B009B40F2F11270
:106A90007FB284F802B0E37000232280FD22C4F8A4
:106AA000049084F8207084F8217062846663C4E9DD
:106AB0000233C4E90433C4E90633C4E90933C4E941
:106AC0000B35A6F140032B44C4E90E3A2F4B2B6043
:106AD0002D4B1B685B073ED4A36B34220021184664
:106AE0001BF0AEF82A4A2B4BC0E90D2A4FF08072FA
:106AF000C263019A02622046C8F86030FFF742FF85
:106B000072E7914615461827164600929DE7012226
:106B10004421D3F88000FEF71EFE9DE74FF0000BE6
:106B20009FE72A463146D8F87400FEF714FE054662
:106B30000028A8D1BBF1000F05D0D8F88800214665
:106B400020B1FEF798FE6FF0040163E7D8F88000EB
:106B5000FEF735FEF7E726F00302CC21281D443A64
:106B60001BF06EF8B8E7002F7FF463AF18277207A9
:106B70007FF45BAFA6F14802074B9A427FF663AF02
:106B800053E700BF7C0C0024B47B0608A52E5AE214
:106B9000A5670408C16B0408B7FFFF7F38B5054639
:106BA0001446FFF7DDFE01602846FFF793FD1CB198
:106BB000BDE83840FFF7E6BEBDE83840FFF77EBECF
:106BC00010B543780446332B0CD1416A90F823204A
:106BD000FFF7F6FD014628B120460022BDE810402F
:106BE000FFF7DCBF10BD10B50446806918B1002264
:106BF0001146FFF7D3FF6378232B02BFA36800225F
:106C00009A6110BD70B50F4C267A022E18D1636AB6
:106C1000B3B16569E86AFFF74DFA2846FFF7E3FF6D
:106C200004F11C00FFF726FE4670A061EFF3098314
:106C3000AB63002328466361BDE87040FFF7F4BDF5
:106C400070BD00BF7C0C002410B5044610B1037861
:106C5000F12B07D020466FF0030100F075FB6FF0B9
:106C6000030010BD437803F00F03022B06D0032B63
:106C70002DD0012B10D06FF0020108E0184B1A7ACA
:106C8000022A01D15B6A4BB96FF00201204600F085
:106C90005BFB6FF00200E4E7FFF7F5FDE06AFFF74A
:106CA00009FA2046FFF79FFF6178022914D10D48A9
:106CB000FFF7E0FD0A4B41709861EFF30982A26390
:106CC00000225A612046FFF7AFFD0020C9E7FFF719
:106CD000DAFDFFF7FFFCE1E70020FFF753FEF1E7E5
:106CE0007C0C0024980C002470B5044620B1037875
:106CF000F12B01D1002908DA6FF003056FF00301D1
:106D00002046FEF7CEFA284670BD4378042B06D104
:106D10006FF002016FF00205FEF7C3FAF3E700F12E
:106D2000280353E8002F42EA010543E8005606B164
:106D3000F7E74378332BE6D1416A90F82320FFF739
:106D40003FFD01460028DED094F8233001229B0746
:106D500056BF656A054620EA05052046FFF71EFF77
:106D6000D1E7000038B51E4C0246237A022B34D1FD
:106D7000606AA0B163695A704A1C16D1226B002167
:106D800072B94FF0FF30C3E90421D86159B10B61EA
:106D90001448FFF76FFD02234370A061012038BD46
:106DA00011461269ECE72363F2E7E26A002012B1B0
:106DB000D569A9420BD2D961C3E9042058B1036156
:106DC000002AE5D0D0695361401AD061E0E710464F
:106DD000491B1269EBE7E362F2E70020DFE700BF3F
:106DE0007C0C0024980C0024F8B5164B05460F4681
:106DF00016465C693CB920466FF00701FEF751FA70
:106E00004FF0FF30F8BD002807DA20466FF003018D
:106E1000FEF747FA6FF00300F4E70A460146204602
:106E2000FFF7CEFC0028EDD14EB13146332065622C
:106E300084F82370FFF796FF6FF00100E2E76FF030
:106E40000200DFE77C0C002438B50D4C00210D4812
:106E5000A26DFFF7BFFD0C4D636EA8625BB1984752
:106E600058B9E26DE96C206EFFF7B4FDA8640038F4
:106E700018BF012038BD0120FCE70020FAE700BF61
:106E8000B47B0608B97204087C0C002410B50446D3
:106E9000EFF3058333B100206FF0050100F054FAE1
:106EA000002010BDFFF704FC0028F4D12046DFF8D5
:106EB00008C000DFF5E700BFD569040808B5EFF3A7
:106EC000058313B1054B586908BDFFF7F1FB002896
:106ED000F8D1DFF80CC000DFF6E700BF7C0C00241F
:106EE0004567040808B5EFF305833BB100206FF058
:106EF000050100F029FA6FF0050008BDFFF7D8FB87
:106F00000028F3D1DFF804C000DFF6E7CD680408FD
:106F100010B5044600F046FAEFF305833BB1204676
:106F20006FF0050100F010FA6FF0050010BDFFF7DB
:106F3000BFFB0028F3D12046DFF804C000DFF5E7EF
:106F4000496C040838B502460D46EFF305834BB192
:106F500092B96FF003046FF003011046FEF7A1F938
:106F6000204638BDFFF7A4FB0028F1D11046DFF81A
:106F700044C000DF0446F3E71378F12BE9D1002D7C
:106F8000E7DB5378042B07D16FF0020110466FF056
:106F90000204FEF786F9E3E702F1280353E8001F35
:106FA00041EA050443E8004000B1F7E71046FFF767
:106FB0004DFBD5E7E96C040810B50446EFF30583F3
:106FC0003BB100206FF00501FEF76BF96FF0050093
:106FD00010BDFFF76DFB0028F3D12046DFF804C099
:106FE00000DFF5E7E96D040830B50C4D00226B6C4D
:106FF00013B11C698C420AD90161C0E902231BB19B
:107000001C699860641A1C612AB1D06030BD1A46B0
:10701000091BDB68ECE76864F8E700BF7C0C002420
:107020002DE9F041184D6C6C54B3236901276E694A
:10703000013B2361236913BBE3680BB1A2689A602B
:107040006B64002304F11801E86C1A46FEF760FE39
:1070500058B121460320D5E905836B61FEF7BFFADD
:107060006B6913B9B04508BF0026E378012B09D13D
:1070700061692046FFF7B8FF6C6C002CDAD16E61B5
:10708000BDE8F0816770F7E77C0C002408B5FEF7D7
:107090002DFE18B9034B044A1A6508BD4FF0FF30A6
:1070A000FBE700BF7C0C002421700408044607B5F0
:1070B0004FF0FF33002269462046FEF769FE0028A4
:1070C000F6D1DDE900309847F2E7000008B5094A3B
:1070D000094B1A60094B9B1A094A1360094A0A4B6B
:1070E0001A600A4B9B1A0A4A136000F051F800F02C
:1070F00083F800BF00FC0724444900240000082452
:107100004049002498170124D0FD002400FC0724E6
:10711000CCFD002438B50E480B250E4B1C244560D1
:1071200003600D4BC4608360FFF70CF80B4B1860D5
:107130000B480C4BC460C0E900350B4B8360FFF774
:1071400001F80A4B1860BDE838401AF077B800BF64
:10715000104900249C7C0608204900243C49002456
:10716000E0480024A97C0608F04800240C490024CB
:10717000FDF76ABC024B4FF0FF311868FEF7FABF0B
:107180003C490024014B1868FFF70CB83C49002427
:1071900008B505F0D5F80C4B0C4998684FF0005332
:1071A0001A1802F16042126843F8042B8B42F7D19F
:1071B000054B4FF000529A6014F084FB16F03AFD34
:1071C000BDE8084000F015B800ED00E0980200208E
:1071D0007047704708B500F043F8FFF7F9FFFFF775
:1071E00099FFFFF7F6FF06F0BDF9BDE80840FFF78D
:1071F000BFBFFEF7FFB90000114C124B23614FF4E3
:10720000004363614423E3600F4BA3601823A36131
:107210000E4B07B5224600210D482360FFF736FECE
:10722000034628B922460B4900900B4806F0AAF9FC
:10723000FEF7F8F9002309491A460093F5E700BF65
:10724000B0C90024B049002468490024B37C060872
:10725000D5710408B87C06081D010180D47C06089D
:107260001FB5064B6C460FCB84E80F002046FEF797
:1072700069FF034B186004B010BD00BFFC7C06081A
:107280006449002473B506460C46154606F06CF9B1
:1072900058B90634324628462ABF054B054953F8EB
:1072A00024100023009306F06DF902B070BD00BFFA
:1072B000C07E0608147E060808B500F0F7F8000046
:1072C00007B50023411E024600930023042919D864
:1072D000DFE801F003080C10140001220B490C48F0
:1072E00006F050F902220B490B48F9E703220B493B
:1072F0000B48F5E704220B490B48F1E705220B493F
:107300000B48EDE70B490C48EAE700BF0C7D060887
:10731000250102802D7D060826010280527D060887
:1073200027010280877D060828010280C27D0608A9
:107330002A010280027E0608000102800146014AFD
:10734000FFF7A0BF31010180014AFFF79BBF00BFDB
:1073500032010180014AFFF795BF00BF370101806C
:10736000014AFFF78FBF00BF3301018011F1110FF8
:1073700002D0024AFFF786BF704700BF3401018088
:10738000014AFFF77FBF00BF3801018010B5FFF74A
:1073900095FD034B1B6813B1BDE81040184710BDA5
:1073A000D4C90024024B1B6803B11847704700BFC3
:1073B000D4C90024024B987A003818BF01207047C6
:1073C0007C0C002408B5FEF771F90022064906F08E
:1073D000E7F9C31C04D98B220449054805F03EFE99
:1073E000BDE80840FEF776B9B5730408FB7E0608D1
:1073F0000D7F0608B0F57A7F10B50C4604D0322216
:1074000019491A4805F02AFE05F0E4FA0028184A3E
:1074100016DB00F16043F02103F5614383F80013AC
:10742000916800F1100341F82340BFF34F8F926839
:1074300052F823309C420AD03F220B490D48E1E725
:1074400000F00F03F021043B13441976E8E700280D
:1074500007DB0123410900F01F00074A834042F87F
:107460002130002010BD00BFFB7E06083A7F0608D1
:1074700000ED00E0477F060800E100E008B506F0F7
:1074800017F9BDE8084005F003BB0000014B186880
:1074900005F0C6BA00FD0024014B186805F0B2BA29
:1074A00000FD002408B505F095FA08BD024C08B5AA
:1074B00023689847FCE700BF200D00240C3070477C
:1074C00003680BB108461847704738B504460D46A7
:1074D000102200211AF0B4FB20462946FCF760FE7A
:1074E000204638BD08B5FCF739FF08BD044B002223
:1074F000C3E900229A601A61024ADA60704700BF4D
:10750000D8C90024C174040838B50D4600210446CA
:10751000102200F8011B1AF093FB2046658238BD4B
:1075200042F60211024808B5FFF7EEFF08BD00BFA2
:10753000ECC9002408B5FAF704FA08BD38B50446CA
:107540000D46102200211AF07BFB20462946FCF74D
:1075500027FE204638BD08B5FFF7C4FF08BDD0E9B7
:107560000032096812F0010F01EB620005D010B47F
:1075700054100A595DF8044BD3581847014604309B
:1075800008B5FFF7ECFF08BD034A0346C26007C910
:1075900083E80700704700BF747F060870B586B0A7
:1075A0000E46002104466D4685E80C0010221AF0B4
:1075B00047FB06AB039695E8030003E9030020466A
:1075C00003A9FFF7E1FF204606B070BD37B56C4652
:1075D000054684E80C0094E80C00FFF7DFFF28461E
:1075E00003B030BD08B5FFF7C9FF08BD08B5FFF708
:1075F000F9FF08BD0068704710B50446FAF79CF91A
:10760000204610BD10B50446FAF796F9204610BD85
:1076100010B504460021FAF7BFFE204610BD08B59C
:10762000FFF74CFF0068003818BF012008BD08B5FF
:10763000FFF744FF0068003818BF012008BD10B5EF
:1076400004460021FAF7A8FE204610BD70B5044696
:107650000D46FFF7E4FF28B940F202220649074829
:1076600005F0FCFCE0682946FFF7C4FF034620460E
:10767000BDE87040184700BFA47F06082D7A0608B1
:1076800008B5FFF7E3FF08BD70B504460D46FFF7E8
:10769000CEFF28B940F202220649074805F0DEFC79
:1076A000E0682946FFF7A6FF03462046BDE8704084
:1076B000184700BFA47F06082D7A060808B5FFF713
:1076C000E3FF08BD10B5044606F03AFE204610BDA3
:1076D00010B5084C204606F0F5FD00232046064A6A
:1076E00084F8243023630549C4E90A33BDE8104017
:1076F00006F088B900CA002400000024C5760408FA
:107700000268814B9A422DE9F04393B040F0F98032
:1077100011F03EFA05F08EFD7C4A0023C2F8843059
:10772000BFF34F8F536923F480335361BFF34F8FFF
:10773000D2F8803043F6E074C3F3C900C3F34E338C
:107740005B0103EA0406014646EA81750139C2F885
:107750007452F9D2203B13F1200FF2D1BFF34F8FB7
:10776000BFF36F8F05F07CFD694B01260025D3F830
:10777000E0204FF400470DA9664842F001024FF0A7
:10778000300902244FF00308C3F8E020D3F8E020CA
:1077900002F001020192019AD3F8E02042F00402C3
:1077A000C3F8E020D3F8E02002F004020292029A2B
:1077B000D3F8E02042F04002C3F8E020D3F8E02004
:1077C00002F040020392039AD3F8D82042F4004218
:1077D000C3F8D820D3F8D82002F400420492049AC7
:1077E000D3F8D82042F48032C3F8D820D3F8D82078
:1077F00002F480320592059AD3F8D82042F4003280
:10780000C3F8D820D3F8D82002F400320692069AA2
:10781000D3F8E02042F40072C3F8E020D3F8E0305F
:1078200003F400730793079BCDE90D76CDE90F555F
:107830000AF078FE0DA93848CDF834900AF072FEAF
:107840003246102134480AF04FFF32462021324898
:107850000AF04AFF0DA931480E960D940F950AF0D3
:1078600061FE324621462D480AF03EFF192008F0FD
:1078700043FF39462A4627480AF036FF642008F0BD
:107880003BFF3246394623480AF02EFF0B274FF4C0
:10789000605308A922480A95CDE90834CDE90B8741
:1078A0000AF040FE08A91C480C97CDE90844CDE930
:1078B0000A580AF037FE08A917480C97CDE9089432
:1078C000CDE90A480AF02EFE802308A913480C9738
:1078D000CDE90834CDE90A680AF024FE042308A99A
:1078E0000E480C97CDE90834CDE90A480AF01AFE93
:1078F00008A90A480C97CDE90844CDE90A580AF0CE
:1079000011FE13B0BDE8F0830080024000ED00E0FE
:10791000004402580024025800080258000002588F
:107920000018025830B570B1CC6864B18A6852B1A1
:107930000B6943B10D6849688560C1608361C0E926
:107940000424002030BD4FF0FF30FBE773B5002367
:1079500046680446019366B1A36998470546A36942
:107960009847431BB3F5FA6FF9D9012300256360EB
:1079700027E0836803B198472023002523606369CB
:1079800001AA12213046984700281DDB019B03F015
:107990001F03B3421AD10025266020681F2833D860
:1079A0007DB923694FF400422946984700282EDB11
:1079B000636901AA29462068984700280ADA6FF00F
:1079C0000405284602B070BD6FF004050136202E74
:1079D000D5D1E2E7A36998470646019B1B0402D470
:1079E000002DB9D0EDE7A3699847801BB0F5FA7F69
:1079F00007D8636901AA0021206898470028ECDABB
:107A0000DDE76FF00105E8E76FF00205D9E76FF0F9
:107A10000305D6E737B500254369044601AA0121CD
:107A2000006801959847A84203DA6FF0040003B09C
:107A300030BD636901AA0121206898470028F4DB62
:107A4000019B5B072CD5636901AA294620689847EA
:107A50000028EADB019BDD040ED403F40452B2F5E6
:107A6000045F01D10220E2E7980401D50320DEE79C
:107A7000D90513D40520DAE7636901AA1F2120681C
:107A800098470028D1DB019BDA040BD503F01C03D7
:107A9000182BE7D0082BE9D0142BEBD10420C6E734
:107AA0000120C4E70620C2E740F2DC507047002006
:107AB00070470620704770477047C0F86C117047D8
:107AC0000020704712F040BEF0B500F582769FB0FE
:107AD00005460C46304606F0FDFB7822002168463C
:107AE0001AF0AEF800206A46234601467BB91A49CF
:107AF00032224860281DC1F808D009F08AFD0346EB
:107B000038B3164A0220164904F090FD06E00A290F
:107B100011D1144A0220124904F088FD0025A37BEC
:107B2000012B02D9204600F095FD304606F0EEFB11
:107B300028461FB0F0BD5F6817605F893844576002
:107B400009B142F8042C1B6803B9936001310C326F
:107B5000CCE70125E3E700BFB8CB0024DB7F0608B4
:107B6000D67F0608AF7F0608032A0846024928BFC9
:107B7000032219F067BF00BFCC86060808B5044A87
:107B80000820044904F052FDBDE8084005F050BE4D
:107B900003800608D67F0608884209D038B5044617
:107BA0000D46F9F7C9FE29462046FCF7F9FA38BD1B
:107BB000704700F5AE70FFF7EFBF884209D038B5C7
:107BC00004460D46F9F7B8FE29462046FCF7E8FAC8
:107BD00038BD704700F5A670FFF7EFBF10B5064C33
:107BE00006492046FFF79EFE2046FFF7AFFEB0FA9B
:107BF00080F0400910BD00BFECCB0024240D002410
:107C00000148FFF707BF00BFECCB00240238032870
:107C100015D8DFE800F0020A0C114FF400530B6096
:107C20004FF480430120136070470023F7E74FF4BF
:107C300000530B600023F5E700230B60F2E7002000
:107C4000704708B500F0F0FA08BD000030B5041D1B
:107C500085B000230D46204601A9009309F0B6FD2A
:107C600018B14FF0FF3005B030BD6946204609F02D
:107C7000FCFD28B1164A0220164904F0D7FCF0E7B3
:107C8000204609F00FFE0099002911DD019B03F049
:107C90001F020A44BFF34F8F0F481A44C0F85C32EA
:107CA0002033D11A0029F9DCBFF34F8FBFF36F8F58
:107CB0004FF4C172BDF80010002000F0FDFC2860F8
:107CC00020B1BDF80020019900F07CFD0020CAE73A
:107CD0000E800608D67F060800ED00E03D20002259
:107CE000072108B509F042F83D20BDE8084009F039
:107CF0006FB80020704700000022074BD3F800380F
:107D00000270802243714270E12282701A0CC270AC
:107D10001A0A0271704700BF00E0F11F10B5044657
:107D2000FFF7E7FF20B92046BDE81040FFF7E4BFAA
:107D300010BD000070B586B0044609F069F82F4800
:107D40002F4B02AD01260434CDE903034FF08073BD
:107D50002846ADF80860059309F078F840F2011361
:107D6000DFF8C4C02846ADF80830264BCDE903C380
:107D70004FF48033059309F069F8042009F056F8B0
:107D8000214B28462360FFF7C9FF204B6560082080
:107D900023611F4B2672E36040F2F4531D4A636176
:107DA0000A231D490093042304F040FC204609F0F7
:107DB000DDFF054600BB194B30220146184E184620
:107DC00019F03EFF212240F8042C4FF440320261AA
:107DD0002946013532460023204606F5BF6609F0E4
:107DE00081FB042DF4D10F4A08200B4904F01EFC3E
:107DF000FFF7F4FE06B070BD0020FBE70000043082
:107E0000090000030D000003008002400000043060
:107E10000001043039800608D67F0608BCCB002458
:107E2000000404305380060800400430084608B5BA
:107E3000FFF774FF012008BD002307B51A46024969
:107E40000248009305F09EFB6D8006080500118036
:107E5000002307B51A4602490248009305F092FB39
:107E6000A18006080500118038B50D4B0025044699
:107E7000036000F5827040F8485C06F023FA04F5D0
:107E8000947006F01FFA04F5A670FFF7D8FB04F50E
:107E9000AE70FFF7BDFB2046C4F8705138BD00BF7F
:107EA0003081060810B50B4C2368BFF35B8FDB07EE
:107EB0000ED4204605F0B6FD50B10748FFF7D4FFB9
:107EC000064A0749044805F09DFD204605F0CCFD13
:107ED000014810BD34CA002438CA00240000002420
:107EE000397F040870B50D4616460446FFF7DAFFE1
:107EF00033462A462146043009F0CCFD003818BF2D
:107F00000120404270BD70B50D4616460446FFF78D
:107F1000C9FF33462A462146043009F0E9FD0038FE
:107F200018BF0120404270BD08B5FFF7BBFF043009
:107F300009F0E0FE002008BD0A4B10B504460360BE
:107F400000F5AE70FFF75EFB04F5A670FFF754FB7B
:107F500004F5947006F0F4F904F5827006F0F0F977
:107F6000204610BD30810608F0B59DB00446FFF7ED
:107F700047FE01280546D4F8707131DD012F18DC69
:107F800001AA02A9FFF742FE18B94FF40053CDE948
:107F90000130261D03A9304609F0DAFD019B03A933
:107FA00030460993029B089309F098FE304609F089
:107FB000B8FA04F5AE763046FFF731FB60B1012D1B
:107FC00020DD012F08DC01213046FFF759FB114A63
:107FD0001149082004F02AFBC4F870511DB0F0BD0F
:107FE000012FE6DD0D4B4FF00052C3F88420BFF3A4
:107FF0004F8FBFF36F8F201D09F0DFFA2046FFF788
:108000006DFED6E7012FE7DD00213046FFF738FB94
:10801000034ADDE7D5800608D67F060800E100E0C8
:10802000F480060873B50446002600F594752846CA
:10803000019606F04FF901A92046FFF707FE002838
:1080400005DA284602B0BDE8704006F05FB9019934
:1080500019B104F5A670FFF731FB284606F056F972
:10806000E5E7000038B50E4C05462368BFF35B8F8B
:10807000DA0708D4204605F0D5FC20B1094B20468C
:108080001D6005F0F1FC074C4FF0FF32002101208C
:10809000FEF792FFC307F7D52068FFF7C3FFF3E7AA
:1080A000B0CB0024B4CB0024D0E90032096812F030
:1080B000010F01EB620005D010B454100A595DF8AD
:1080C000044BD35818470146043008B5FFF7ECFFBE
:1080D00008BD0000034A0346C26007C983E80700E1
:1080E000704700BF6C81060870B586B00E4600214F
:1080F00004466D4685E80C00102219F0A1FD06AB80
:10810000039695E8030003E90300204603A9FFF75F
:10811000E1FF204606B070BD37B56C46054684E8E1
:108120000C0094E80C00FFF7DFFF284603B030BDD9
:10813000F0B505468DB005F065FB2846FFF7FAFD62
:10814000064600284ED02022002104A819F078FD10
:10815000264B4FF40060039319F022F905F1C00398
:1081600003AA2946079005934FF40063204808931B
:108170004423069328230993FEF788FEC5F8BC0024
:1081800003F08CFD1B4B07461A4A01930023294636
:1081900003A80293FFF7C0FF1021384603F02CFB21
:1081A0000446A0B103A9FFF7C9F92046C82103F08E
:1081B000C4FC2046C82103F0C3FC20460E4903F04E
:1081C000C2FC22460D49384603F0D5FB044603A8FD
:1081D000C5F87441F9F7B5FB0A20FCF755FE2846AF
:1081E000FFF77CFD30460DB0F0BD00BF14810608DE
:1081F00065800408697F040835750408577504080C
:1082000008B5FFF760FF08BD08B5FFF7F9FF08BD27
:1082100008B5FFF747FED0F8BC0020B10121BDE84A
:108220000840FEF78FBE08BD08B5FFF73BFE0430DF
:10823000BDE8084009F07CBB130911D051F804CB0C
:1082400040F804CB51F804CB40F804CB51F804CBF0
:1082500040F804CB51F804CB40F804CB013BEDD1FE
:1082600012F00F0305D011F801CB00F801CB013B50
:10827000F9D170470222002373B504460E46006808
:108280001146FCF7C7FF021E01DB930709D4002348
:1082900016491748009305F06DF94FF0FF3002B012
:1082A00070BDFDF7D5F994F824300546012103F19E
:1082B0000A020133206803F0070344F8226084F8BF
:1082C0002430FCF75FFF94F8243094F82520013324
:1082D00003F00703934203D102212068FCF782FFD9
:1082E0002846FDF7CBF90020D9E700BF78810608C2
:1082F0000F01038013B504464FF0FF310068FDF70E
:1083000039FF30B10023224603490448009305F0A9
:1083100039F902B010BD00BF908106081501038035
:1083200013B504460068FDF73DFF30B10023224637
:1083300003490448009305F025F902B010BD00BFC1
:10834000A681060817010380094B07B54FF0FF31DE
:108350001868FDF70FFF30B10023064906481A469A
:10836000009305F00FF9012003B05DF804FB00BF96
:108370000CCC0024BE81060815010380074B07B50D
:108380001868FDF70FFF30B10023054905481A466C
:10839000009305F0F7F803B05DF804FB0CCC002463
:1083A000D68106081701038070B5064608200D46E1
:1083B00000F004F9044660B1012301460370C0E9EE
:1083C00001650548FFF756FF28B12146082000F057
:1083D00001F94FF0FF3070BD10CC00242DE9F041C1
:1083E000044600286CD0830705D0FFF7ADFFBDE839
:1083F000F041FFF7C3BFDFF8D880A0F10805D8F837
:108400000030AB42F1D82F4F00F10C033A689A428A
:10841000EBD32D48FFF76EFF14F8043C1BB92A4834
:10842000FFF77EFFE1E734F8086CB6F57A5FF6D81F
:1084300034F8062CB2F57A5FF1D8D8F80030E91A92
:1084400089B2914202D09A5A8A42E8D19819D7F853
:1084500000C0604502D042888A42E0D1002204F880
:10846000042C1A4A1768AF4288BF156085420FD0A6
:1084700007796FB960450BD01768B842985B08BFA1
:108480001560B0F57A5F24F8080C1CBFC018418055
:1084900034F8061C581885420DD006795EB9166866
:1084A000B54208BF106034F8082CB2F57A5F5A5212
:1084B0001CBF9B1859800448BDE8F041FFF730BF4E
:1084C000BDE8F0818CCC00245CCC002458CC002486
:1084D00090CC00242DE9F04140B1C41C24F00304E9
:1084E000A4B20B2C04D9B4F57A5F02D9002045E080
:1084F0000C24A042FAD826486FF00708FFF7FAFECE
:10850000244E254BC4F57A5E32681968531A9BB223
:10851000734503D31E48FFF703FFE7E7CD18CF5A93
:1085200095F804C0BCF1000F30D1A8EB030038442B
:10853000A0422BD304F1140E704521D308341C44FF
:10854000A0B211FA84F484F804C00F5263800123AE
:1085500028802B710B5AB3F57A5F01D00B445880F9
:10856000AA4206D10D4B1B68107908B193420AD17B
:1085700032600748FFF7D4FE05F10800BDE8F0813E
:1085800001232B71ECE712880A44EDE73B46BFE775
:108590005CCC002458CC002490CC00248CCC00244B
:1085A00010B50446FFF7D0FEA3681C680CB1226822
:1085B0001A60FFF7E3FE204610BD00000D2804D826
:1085C000034B53F82000FFF7EBBF0020704700BFBC
:1085D000F08106080D2838B50C460DD861B1074B5F
:1085E00053F82050FFF7B0FEAB681A6822601C6099
:1085F000BDE83840FFF7C2BE38BD00BFF0810608B5
:1086000008B5FFF7A1FE084B00221A70FFF7B6FE6F
:10861000064B186800B908BD436F1BB1BDE80840A0
:1086200000F00AB9C068F5E73BE600243CE6002408
:1086300070B506460C200C461546FFF7BFFF40B14B
:1086400000230481448143730573C0E9003601238C
:10865000C38170BD70B5044660B30025FFF774FE9A
:10866000A67B013EF6B2A673FFF788FE56B9627B81
:1086700026689207237B09D5236920469847013550
:10868000EDB20EB9284670BD3446E7E703F00F039C
:10869000022B04D121460D20FFF79CFFEFE7012BB1
:1086A00002D121460C20F7E7002BE8D12046FFF746
:1086B00095FEE4E70546E5E7B2F5C17F2DE9F04711
:1086C00004460E46074610D008D822F04003012B7E
:1086D00007D10020BDE8F047FFF7AABFB2F5207F21
:1086E00047D000252846BDE8F0870024DFF8D09069
:1086F0002546A0460D20A246FFF760FF0446C8B9F4
:108700002C4EFFF721FE012337783370FFB2FFF7BD
:1087100035FE4FB921462848FFF746FE20B1FFF746
:1087200013FE3470FFF72AFE002DDAD02846FFF73B
:1087300091FFD6E7FB1C0744C0F8008023F0030339
:1087400013370681C3F5147327F00307C0F80C90A4
:108750009BB24760B34228BF334643813DB1CAF85C
:108760000000F31A00279EB2002EC3D1BAE70546D7
:10877000F7E7C31CCA1C23F0030322F003021344CF
:108780009BB203F11000934280B2AAD38242A8D8D0
:10879000FFF7A0FE05460028A4D00444002306816C
:1087A00013340360054B24F003044681C360446026
:1087B00098E700BF3BE60024018604088000010022
:1087C000820001002DE9F0410F4614460546B8B17C
:1087D000B1B10389934216D34FF0000814B9204673
:1087E000BDE8F0816E8907EB08016868A64228BFE2
:1087F00026463246A41BFFF71FFDB0442D68EDE767
:108800006FF00F00ECE74FF0FF30E9E710B50446DA
:1088100048B1406808B1FFF71DFF21460320BDE8BD
:108820001040FFF7D7BE10BD10B500B910BD0468E9
:10883000FFF7ECFF2046F8E710B50446406F18B18B
:10884000FFF7F2FF0023636710BD0000F8B505468F
:10885000064655F8044B8CB90D4F386818B14FF0E7
:10886000FF31FDF787FC346824B928462C4605F013
:1088700029FD3560386808B1FDF794FCAC4204D09E
:108880008B220449044804F0E9FB2046F8BD00BFF0
:1088900064490024F482060803830608704710B573
:1088A0000446702105F032FB204610BD08B5034890
:1088B000FFF7CCFFBDE8084005F00CBD40E6002402
:1088C00008B50348FFF7C2FFBDE8084005F01EBD2C
:1088D00040E6002438B5084B04460D46C2660360E6
:1088E000FFF7E4FF2946201D10F0CCFA2046FFF7E1
:1088F000E7FF204638BD00BF308306080368012229
:1089000000211B691847036800221B69114618479C
:1089100000F59E7005F0DEBC00F59E7005F0F6BC1B
:1089200010B50446F9F708F82046FBF733FC10BDF4
:10893000884209D038B504460D46F8F7FDFF2946B0
:108940002046FBF72DFC38BD704700002DE9F843A9
:1089500004460546114B0F4604F1AC0604F59E791A
:1089600045F8043B90460021A822284619F068F9F2
:1089700030461036F9F738FD4E45F9D1304605F04E
:10898000A1FC42463946284611F04EFB28462246B5
:10899000034911F0B1F92046BDE8F8834883060881
:1089A0007B8A04082DE9F0410368044616460F4609
:1089B0009B6804F1040804EB061598473846AC356B
:1089C000FBF7C3FCA0B12846FBF7BFFC08B904F0D5
:1089D00019FF39462846FFF7ABFF012240463146D2
:1089E00011F028FB23682046DB68BDE8F0411847FA
:1089F0002846FBF7AAFC08B104F01AFF2846FFF747
:108A00008FFF0022EAE700007FB5154B04460025E2
:108A1000036000216846FBF76DFA6946EAB220461A
:108A20000135FFF7BFFF6846F8F78BFF092DF0D13E
:108A3000251D04F1AC06284611F06AF9284604F514
:108A40009E7511F089F9284605F07AFCB54204D0EC
:108A5000103D2846F8F775FFF8E7204604B070BDD2
:108A60004883060810B50446FFF7CEFF4FF4B071F7
:108A7000204605F04BFA204610BD00EB011010B562
:108A800000F1AC042046FBF760FC10B12046FBF778
:108A900065FC10BD10B5044604F0CCFB0121204656
:108AA00011F018FCBDE8104004F0DABB10B5044624
:108AB00004F0C0FB0021204611F00CFCBDE8104082
:108AC00004F0CEBB38B504460D4604F0B3FB29468E
:108AD000204611F0FBFBBDE8384004F0C1BB0000AC
:108AE000084A094B10B5D2F894409C42FBD1036868
:108AF00029B181680B604FF44073536110BDC168A8
:108B00001B04F7E700640258000300804168034635
:108B100030B471B1D0E9032000F0010402B944B1CE
:108B2000451001EB60000CB149598A58996830BC76
:108B3000104730BC7047036870B504460D461B688B
:108B4000984704F130002946C4F8CC5012F004FADA
:108B5000236820465B68BDE8704018472DE9F34163
:108B600006461D4604460F4656F8303B90461B68A5
:108B700098479DF820304246394683F0010330463D
:108B800000932B4612F0DCFB2368064620465B6808
:108B90009847A81B18BF012002B0BDE8F0812DE95D
:108BA000F34106461D4604460F4656F8303B9046B4
:108BB0001B6898479DF820304246394683F00103F0
:108BC000304600932B4612F055FB2368064620469C
:108BD0005B689847A81B18BF012002B0BDE8F08170
:108BE00070B590B00D46144600211C2202A819F061
:108BF00027F801260023294602A800961A4603F00A
:108C0000D7F81C22002109A819F01AF800232146E0
:108C100009A81A46009603F0CBF80A9B1A68099B2C
:108C20001A4203D16FF0010010B070BD039B1968A8
:108C3000029B194046D109A80A24FFF743FF09A85F
:108C4000FFF728FF002109A8FFF73CFF002109A832
:108C5000FFF746FF052005F0A3FA012109A8FFF759
:108C600031FF012109A8FFF73BFF052005F098FA25
:108C7000013CE7D102A8FFF70DFF214602A8FFF74C
:108C80002FFF052005F08CFA012109A8FFF728FF26
:108C9000052005F085FA012102A8FFF721FF052034
:108CA00005F07EFA02A8FFF701FF09A8FFF7FEFE14
:108CB0000A9B1A68099B1A42B4D0039B1A68029B4C
:108CC0001A42AFD00020AFE710B504460021F9F7F3
:108CD00063FB204610BD0021242210B5044640F855
:108CE000041B18F0ADFF204610BD08B5D030FFF7CB
:108CF000ADFDBDE8084005F0EDBA08B5D030FFF78E
:108D0000A5FDBDE8084005F001BB0000F8B51B4B10
:108D100004460D46164640F8043B04F13007FFF7C1
:108D2000D3FF0021164B9C22A18538466361A461C4
:108D3000C4E90711C4E9091118F082FF114B04F1CD
:108D4000D000C4F8CC30FFF7C6FF2046FFF7CDFFB8
:108D5000324629462046A4F8F850A4F8FA60FFF7F6
:108D60003FFFB4F9FA20B4F9F810384612F048FA87
:108D70002046FFF7C2FF2046F8BD00BF608306080B
:108D80000D8B0408A086010070B504460D461646FA
:108D900000219C2218F054FF32462946204612F04A
:108DA0002FFA2046044912F0D7F82046012111F08D
:108DB00086FE204670BD00BFA086010012F0CCB830
:108DC000CAB2002342F00102194611F065BE11F04B
:108DD000BFBE11F0CBBE10B5144611F0FFFE001B54
:108DE00018BF012010BD10B50446F8F7A5FD2046B8
:108DF000FBF7D0F910BD884209D038B504460D46BE
:108E0000F8F79AFD29462046FBF7CAF938BD7047A6
:108E10000346024A203011F055BB00BF2D8F0408D5
:108E200083681A6843681A4214BF01200020704703
:108E300070B5114B054604460E4645F8043B1C220E
:108E40000021284618F0FCFE1022002104F1200029
:108E500018F0F6FE04F13000F9F7C6FA04F140000C
:108E6000F9F7C2FA31462046FFF7D2FF28463146CD
:108E700002F092FF204670BD78830608084B10B5BB
:108E8000044640F8203B11F01DFC04F14000F8F7C7
:108E900058FD04F13000F8F754FD204610BD00BF26
:108EA0007883060810B50446FFF7E8FF50212046F6
:108EB00005F02CF8204610BD70B50E46044604F0AF
:108EC000B9F93046FBF741FA054604F13000203489
:108ED0005DB13146FFF78FFF01222046012111F0DD
:108EE00081FABDE8704004F0BBB9FFF77CFF2A4669
:108EF000F3E770B50E46044604F09CF93046FBF7E4
:108F000024FA054604F1400020345DB13146FFF7F4
:108F100072FF01222046022111F064FABDE8704080
:108F200004F09EB9FFF75FFF2A46F3E7012910B569
:108F300002D002290BD010BD00F130042046FBF70F
:108F400004FA0028F7D02046FEF7CCFAF3E700F148
:108F50004004F3E738B504460D4604F06BF92946A2
:108F6000204612F093FEBDE8384004F079B9837EC4
:108F700010B504461BB904F045FC0123A37610BDCF
:108F8000837E10B504461BB104F052FC0023A37687
:108F900010BD10B5044604F04DF9E37E4BB9B4F9A9
:108FA0001810204613F004F82046FFF7E0FF0123D5
:108FB000E376BDE8104004F053B90023002210B559
:108FC000044601834383C2610362FFF7E2FF204648
:108FD00010BD10B5044604F02DF9E37E3BB12046E8
:108FE00012F04EFE2046FFF7CBFF0023E376BDE8EC
:108FF000104004F035B910B50446FFF7EAFF2046EB
:1090000010BDD0F89030012B10B5044686B01DD8A5
:10901000DBB204300493D0F888300393B0F99C306D
:109020000293B0F99A300193B0F998300093B0F9F7
:109030009630B0F99420B0F9921013F011FBB0FA09
:1090400080F0400984F8940006B010BD0020F9E7D4
:1090500002289ABF014B185C00207047AA830608BB
:1090600038B5044600251C48A4F89A30BDF91030E4
:109070002060201DA4F89C30BDF91430A4F896108F
:109080002946A4F89E30BDF91830A4F898205C2237
:10909000A4F8A030C4F8A45018F0D2FD4FF4003367
:1090A0002046A4F864502366079BC4F88850C4F88F
:1090B00090300A4B84F89450C4F88C30084BC4E9C3
:1090C0002A35FFF79EFF20B942220649064803F0E1
:1090D000C5FF204638BD00BFB883060840420F00D8
:1090E0000390040899830608A28306082DE9F04737
:1090F0009DF8208004460F46164640461D469DF8C2
:1091000024A0FFF7A5FF10B3BAFBF0F300FB13A0F8
:1091100010F0FF091BD1236820469B6898479DF8F3
:109120002830204684F864A084F865300B9B84F8CE
:109130006070C4F88830236884F86160DB6884F864
:10914000625084F8638098474846BDE8F0874FF046
:10915000FF30FAE738B590F8943004460D4693B1E5
:1091600003689B6898472946C4F88C50201D13F06B
:109170005BFA051E2368204618BF0125DB686D4297
:109180009847284638BD4FF0FF35FAE7F8B5044652
:109190000F46164600211F2269301D4618F050FD6B
:1091A00094F86030791C84F868300ABF012384F891
:1091B000697084F86A30721C94F8613018BF2667B1
:1091C00084F86C3094F8623084F86D3004BF012369
:1091D00084F8743094F8633084F8783094F864300C
:1091E00084F879306B1C0ABF0123E56784F880306E
:1091F000D4F8883084F8843094F8653084F8853069
:10920000F8BD2DE9F8431F4690F8943005460E4608
:109210009046DDE908941BB3FCB1B9F1000F1CD0F6
:109220002368EBB103689B68984743463A4631464A
:109230002846FFF7ABFF23464A4605F16801281D83
:1092400013F02BFB041E2B68284618BF0124DB6893
:10925000644298472046BDE8F8836FF00104F9E7BF
:109260004FF0FF34F6E72DE9F8431F4690F89430AD
:1092700005460E469046DDE908941BB3FCB1B9F1F2
:10928000000F1CD02368EBB103689B6898474346E6
:109290003A4631462846FFF779FF23464A4605F10C
:1092A0006801281D13F0D8FA041E2B68284618BF41
:1092B0000124DB68644298472046BDE8F8836FF0DC
:1092C0000104F9E74FF0FF34F6E7F7B51D4690F8D3
:1092D000943004460E461746FBB103689B689847D6
:1092E0004FF0FF333A4631462046FFF74FFF0A9BC7
:1092F0002A4604F168010193201D099B0093089BF5
:1093000013F0EDFA051E2368204618BF0125DB681F
:109310006D429847284603B0F0BD4FF0FF35F9E79E
:1093200008B50348FFF792FABDE8084004F0D2BF41
:1093300068E6002408B50348FFF788FABDE808404E
:1093400004F0E4BF68E6002438B5074B0546044640
:1093500045F8043BFFF7E4FF284613F017F92046D1
:10936000FFF7E8FF204638BDB883060810B504466D
:10937000FFF7EAFFB021204604F0C8FD204610BDEB
:109380004168034630B471B1D0E9032000F0010414
:1093900002B944B1451001EB60000CB149598A583B
:1093A000996830BC104730BC704713B5B0F93830FD
:1093B00044680093B0F93630B0F93420B0F9321077
:1093C000201D14F0AFF802B010BD0000034B186868
:1093D00018B14FF0FF31FCF7CDBE7047644900244F
:1093E00070B5054603F026FF0A4B4FF4AC760A4AE7
:1093F00018680023984204DC002403F031FF204663
:1094000070BD06FB03F18C185158A942F5D0013309
:10941000F0E700BF90E6002494E60024084A08B56F
:109420001368052B04DDAF220649074803F016FE3A
:10943000591C4FF4AC701160044A00FB032008BDB6
:1094400090E60024E1830608E983060894E60024F8
:109450004368D3F8EC30834210B5044610D0036F54
:109460009847606800230430D4E9161214F030FAEB
:109470006068216E043014F079FA6368C3F8EC4038
:1094800010BD036870B504461B690D461646984723
:109490006068D0F8EC30A342C4E916560BD1002323
:1094A00032462946043014F013FA236820465B69DB
:1094B000BDE8704018472046FFF7CAFFF5E703688C
:1094C00070B504461B690D46984760682566D0F85C
:1094D000EC30A34209D12946043014F047FA23683E
:1094E00020465B69BDE8704018472046FFF7B0FF93
:1094F000F5E70000B0F94C30013310B50CD0084A44
:10950000084BD2F894409C42FBD1C36B29B1416C0B
:109510000B604FF44073536110BD816C1B04F7E77F
:10952000006402580003008038B5036804461B69D4
:10953000984794F965506B1C84F8653045B920460E
:10954000FFF786FF29462046BDE83840FFF7D2BF27
:1095500038BD10B590F865300446013B5BB280F829
:10956000653013B90121FFF7C5FF236820465B6909
:10957000BDE81040184738B504460D46FFF7D4FF44
:1095800060682946043014F00FFA05462046FFF7BC
:10959000E0FF284638BDF7B504461F460D4616467F
:1095A000FFF7C2FF94F864306068294601933246A1
:1095B000089B043000933B4614F040FA05462046D1
:1095C000FFF7C7FF284603B0F0BD0021282210B5E1
:1095D000044640F8041B18F033FB04F11800FFF7B1
:1095E00073FB204610BD000070B50646044656F8D1
:1095F000045BB5B9FFF7EAFE25686DB9304635461C
:10960000FFF7E3FF04F13000FFF7DFFF0023C4E9B9
:10961000173384F864302660064B186808B1FCF7ED
:10962000C1FDB54204D08B220349044803F016FD66
:10963000284670BD64490024F482060803830608A6
:109640000023082210B5C0E91623038604460C4BFC
:109650000366FF23A0F8643003F0ECFDE06EFFF733
:10966000BFFE606020B9FFF7D9FEE36E6060036063
:1096700003F0F6FD6068F030FFF7B6FF10BD00BFE5
:1096800040420F002DE9F0411E461A4B00250446CA
:1096900003608846184B174685618360C561C060CA
:1096A000C0E904552030FFF70FFBBDF918301C222C
:1096B0002946238704F13C03A4F832801846A78684
:1096C000E68618F0BDFA4FF0FF3102F06EFB0B4B4F
:1096D000B4F93620B4F934102367B4F93200A56622
:1096E00013F0F2FEE0662046FFF7AAFF2046BDE831
:1096F000F08100BF1C84060881930408AB93040822
:10970000406808B5C430FFF7A1F8BDE8084004F090
:10971000E1BD406808B5C430FFF798F8BDE80840DF
:1097200004F0F4BD0D4B10B504460360FFF7E8FFED
:1097300063682046D3F8EC20A24204BF0022C3F89D
:10974000EC20FFF7E6FF04F12000F9F7A1F9E0694A
:1097500008B102F079FF204610BD00BF1C84060846
:1097600010B50446FFF7DEFF7421204604F0CEFB5F
:10977000204610BD7047000070B500F10C0604468D
:10978000B0F95820B0F95610304613F063FBD4E915
:1097900018530DB9DA070ED55A1094F8681004EB77
:1097A0006300DB0748BFA358B4F96A2048BF5D597E
:1097B000B4F96C30A847216D304613F065FA2246A3
:1097C00030460249BDE870400FF0E6BCC99A040873
:1097D0002DE9F0411F46C36D04460E4615462BB1D8
:1097E00040F235122B492C4803F038FC2B4AC0E9D3
:1097F000182303681B68984784F86860A4F86A50C7
:10980000A4F86C70042E0CD8DFE806F016031116CD
:109810001A004FF0FF332A46012104F10C000FF02B
:10982000B3FD236820465B68BDE8F04118472B462E
:109830004FF0FF320221F0E73B462A463146ECE783
:109840000123013584F884300ED01C2004F02AFB5B
:10985000B4F96A6005461C22002118F0F1F931467E
:10986000284602F099FA2567B4F96C300133D8D054
:109870001C2004F017FBB4F96C6005461C22002183
:1098800018F0DEF900223146284602F08AFA6567B0
:10989000C7E700BF4D8406085C840608D19704081A
:1098A00010B50446F8F748F82046FAF773FC10BDE7
:1098B000884209D038B504460D46F8F73DF82946E8
:1098C0002046FAF76DFC38BD704770B506460D4668
:1098D000044656F80C3B1B6898473046294613F05F
:1098E000D3F92368204625655B68BDE870401847BA
:1098F0002DE9F041054698460E46174655F80C3BB3
:1099000004461B689847434628463A46314613F0BA
:109910002FFA236820465B68BDE8F0411847000035
:1099200038B50546044655F80C3B1B689847284651
:1099300013F042F994F88430054673B1626F62B156
:109940000A490B4BD1F894009842FBD1136855B9E2
:10995000926813604FF440734B61236820465B6844
:109960009847284638BDD2681B04F2E700640258C5
:109970000003008038B50546044655F80C3B1B68CB
:109980009847284613F028F994F88430054643B1E7
:10999000236F00F001055A681B6812681A4218BF4D
:1099A0000025236820465B689847284638BD0C3060
:1099B0000FF0A0BC10B50C460C300FF0D1FC2046C7
:1099C00010BD00002DE9F04198461B4B00250446D0
:1099D00003600F46194B29461646856024224360D2
:1099E0000C3018F02DF904F13000F8F7FDFC04F10B
:1099F0004000F8F7F9FC40F201132046C4F850800B
:109A0000A4F854304FF6FF73A4F85670A4F85860C9
:109A1000656684F86850A4F86A30A4F86C30C4F81D
:109A2000805084F88450C4E91755C4E91E55FFF7E7
:109A3000A3FE2046BDE8F0817C84060879970408DF
:109A400003682DE9F04104461B6815460F46984708
:109A500094F85430EE1C03B17DB194F855300BB13D
:109A6000012D0AD0394604EB0610FFF721FF2368C9
:109A700020465B68BDE8F041184703F0DBFB384641
:109A800004EB061604F10C08FAF75FFC88B13046C7
:109A9000FAF75BFC08B903F0B5FE39463046FFF72C
:109AA00007FF0122294640460FF082FB03F0D8FB56
:109AB000DDE73046FAF749FC08B103F0B9FE30465D
:109AC000FFF7EEFE0022EDE7033110B500EB0114C5
:109AD0002046FAF73AFC10B12046FDF703FD10BD11
:109AE000036870B504461B680D46984794F85430D7
:109AF000AB423BD004F1300675B903F09BFB04F197
:109B00000C002A4629460FF053FB3046FAF71DFC9D
:109B100000B303F08DFE1DE094F855304BB9A268F8
:109B20006368511004EB6200D20744BF6258D358F7
:109B3000984703F07FFB3046FAF707FC50B13046F8
:109B4000FAF70CFC03F05EFE0122002104F10C0088
:109B50000FF02EFB03F084FB84F8545035B994F8D1
:109B600055301BB904F10C0012F00CFF236820469D
:109B70005B68BDE870401847036870B504461B6811
:109B80000D46984794F85530AB423BD004F140065F
:109B900075B903F04FFB04F10C002A4601210FF0C8
:109BA00007FB3046FAF7D1FB00B303F041FE1DE09E
:109BB00094F854304BB9A2686368511004EB62000A
:109BC000D20744BF6258D358984703F033FB30465E
:109BD000FAF7BBFB50B13046FAF7C0FB03F012FEB8
:109BE000012204F10C0011460FF0E2FA03F038FBF9
:109BF00084F8555035B994F854301BB904F10C0071
:109C000012F0C0FE236820465B68BDE8704018472C
:109C10001FB5184B0446002103606846FAF76AF93D
:109C2000002269462046FFF70BFF6846F7F789FEDA
:109C300000216846FAF75EF9012269462046FFF7DF
:109C4000FFFE6846F7F77DFE94F8543013B994F898
:109C500055301BB104F10C0012F094FE04F14000E9
:109C6000F7F76FFE04F13000F7F76BFE204604B003
:109C700010BD00BF7C84060810B50446FFF7C8FF7E
:109C80008821204604F042F9204610BD437D10B5DE
:109C900004461BB1037D0BB103F0CAFD204610BD85
:109CA00013B5044601A802F0D7FC637D53B9237DA8
:109CB0000BB103F0A7FD206902F022FB0123C4E9E8
:109CC0000001637501A802F0CDFC02B010BD37B5EC
:109CD000044601A80D4602F0BFFC00230022C4E99F
:109CE00000236B7D4BB1286902F00AFBD5E90032F5
:109CF000C01A61EB0201C4E9000101A802F0B2FC44
:109D0000204603B030BD30B585B00D46044603A8EB
:109D100002F0A2FC29466846FFF7D9FF009B03A882
:109D2000D5E902219B18019A42EB0102C4E90032F5
:109D300002F098FC204605B030BD13B5044601A8DA
:109D400002F08AFC206902F0DBFA00220023C4E959
:109D50000001C4E9022301A802F084FC02B010BD96
:109D6000D0B5002300260027044601610275437523
:109D7000C0E90067C0E90267FFF7DFFF2046D0BDFA
:109D800010B5044602F0CEFA012201462046FFF744
:109D9000E7FF204610BD10B5044602F023F800226C
:109DA00001462046FFF7DCFF204610BD03681B6814
:109DB0001847000010B5084B0446002208462360EF
:109DC0000023A1610549C4E902230023C4E9043347
:109DD00002F024FA204610BD94840608AD9D0408C4
:109DE00007B500F108010090806902F054FA03B051
:109DF0005DF804FB00F10801806902F066BA0020FA
:109E000070476FF01C0070476FF01C0070476FF0D8
:109E1000150070476FF01500704701207047012052
:109E20007047002070470020704770B511F00104A2
:109E300006460D4604D0FFF773FD041E18BF01242B
:109E4000EB0605D53046FFF795FD08B144F0100448
:109E5000204670BDA0F18800FFF7E7BF08B5FFF707
:109E60003FFE002008BDA0F18800FFF7F7BF08B54E
:109E7000FFF782FE002008BDA0F18800FFF7F7BFC2
:109E8000034B10B504460360FFF7C2FE204610BD29
:109E9000A0840608A0F18800F2E700BF10B50446D0
:109EA000FFF7EEFF8C21204604F030F8204610BD6D
:109EB000A0F18800F2E72DE9F04106460D4617466D
:109EC000C2B103F0B4F980F0010313F0FF0403D032
:109ED000336830461B68984705EB070815F8011BE7
:109EE0003046FFF767FDA845F8D11CB1336830460E
:109EF0005B6898473846BDE8F081A0F18800FFF71D
:109F0000DABF38B504460D4662B103681B6898474E
:109F10002046FFF74CFD2870236820465B68984771
:109F2000012038BD1046FCE7A0F18800FFF7E9BF2B
:109F300010B50446FFF746FD034B204623603C3333
:109F4000C4F8883010BD00BFA08406082DE9F04198
:109F50001F46036804460D4616461B6898473B4655
:109F6000204632462946FFF733FC236820465B68CB
:109F7000BDE8F041184710B50446F7F7DDFC204670
:109F8000FAF708F910BD70B504460D4603F052F912
:109F9000A6691EB9BDE8704003F062B904F108007B
:109FA000FFF7E9FF012384F8215084F820300023D3
:109FB000E361A36103F054F921463046BDE87040E7
:109FC00000F073B908B104F085B903F033B908B1F2
:109FD00004F09CB903F044B92DE9F041044686B081
:109FE0000E46174603F026F9A56903F039F935B393
:109FF00001AD0021284604F0C5F903F01BF9D4E9AE
:10A00000068323B139220F490F4803F027F8E56191
:10A0100003F026F9B8F1000F0ED03946284604F0B7
:10A02000B9F948B93046FFF7CDFF20460121FFF7C7
:10A03000AAFF3046FFF7CBFF284604F0CCF906B064
:10A04000BDE8F081418506084D85060838B5002534
:10A05000054B0446456040F8083BF8F7C5F9204633
:10A060002584C4E9065538BD74850608074B10B52C
:10A0700003600446836923B126220549054802F09E
:10A08000EDFF0830F7F75DFC204610BD748506082B
:10A09000418506085B85060830B5044685B003F0A7
:10A0A000C9F804F1080568462946FDF70EFA284666
:10A0B000FFF761FF0023E069A36108B104F088F9AC
:10A0C00003F0CEF86846FAF740F910B16846FDF79C
:10A0D00009FA6846F7F735FC05B030BD002201608B
:10A0E000C0E9012201220273704770470346007BDA
:10A0F00030B1D3E90020136898428CBF00200120C2
:10A1000070472DE9F041012605460068002306FA54
:10A1100001F182EA060E071D17F813400C4204D025
:10A1200004F030043AB1102C07D10233202BF3D1C4
:10A130004FF0FF3013E0002CF7D042EA0300D5F8CF
:10A1400008C006FA00F818EA0C0FEED1202C06D150
:10A150004EEA030406FA04F414EA0C0FE5D1BDE854
:10A16000F08170B50D46114604461E462A46FFF79B
:10A17000C8FF002802DA0020207370BD420825685D
:10A18000636805EB8205E98819446B7906FB0313C4
:10A19000012163608140A36842EAC0100B43C0B252
:10A1A000A360EAE713460A460121FFF7DABF134628
:10A1B0000A460021FFF7D5BF38B505460C460A46CA
:10A1C0000021FFF7EFFF224628460021BDE8384076
:10A1D000FFF7EDBF0022C0E900227047704700681A
:10A1E000704700230B60436813B9016041607047FA
:10A1F0001960FBE70346006828B1026802B95A609B
:10A200001A6000230360704710B5046800222346DB
:10A210008B420ED10AB10B6813608C4204BF0B68ED
:10A22000036043688B424FF0000308BF42600B603D
:10A2300010BD002BFCD01A461B68E9E710B5044698
:10A24000FFF7C8FF204610BD08B5FFF7C8FFB0FAFA
:10A2500080F0400908BD70B505462846FFF7BFFFEE
:10A26000044678B150F8043C061F9B683046984776
:10A2700040B12846FFF7BEFF54F8043C3046DB6887
:10A280009847EAE770BD70B504460D46FFF7A7FF93
:10A290000646291D2046AC61FFF7A3FF26B92046DC
:10A2A000BDE87040FFF7D7BF70BD70B50C460546DE
:10A2B000FFF795FF064604B1043421462846FFF710
:10A2C000A3FFA64204D12846BDE87040FFF7C3BFF4
:10A2D00070BD10B504462046FFF781FF28B150F845
:10A2E000043C0438DB689847F5E710BD10B5044618
:10A2F000FFF7EFFF2046FFF771FF204610BD7047C4
:10A30000F7B51F460D4B0446164640F8043B0D4674
:10A31000F8F76AF8002104F1400004F033F804F182
:10A32000540003F0CFFF089B204632460093294695
:10A330003B4604F0AFF8204603B0F0BD8495060814
:10A34000704703689B6D184770B5164B86B090F840
:10A35000204301930023416805AEADF808308DF825
:10A360000A3040F201230289ADF8123040F20313A3
:10A370008DF80B4001ACADF8143000F10A030391E5
:10A380001D46ADF810202246083303CAB24243F8F6
:10A39000080C43F8041C1446F5D1128828461A808C
:10A3A00006B070BD1201000200487047A888060878
:10A3B000004870479688060800487047808806085D
:10A3C000004870477A880608004870477288060877
:10A3D000004870475C880608036810B504465B6F48
:10A3E0009847D4F8EC0203681B6F9847236820460F
:10A3F0009B6FBDE81040184738B5D0F83433044699
:10A40000012B10D10025D4E9C93000F0010203B9B5
:10A410004AB1411004EB6000C4E9C9550AB1625861
:10A42000D3589847EFE7D4F834332BB940F2C662DB
:10A430000549064802F012FE013BC4F83433BDE87A
:10A44000384002F00DBF00BFA1850608AF850608A1
:10A4500008B5D0F834332BB940F2CD620249034835
:10A4600002F0FCFD08BD00BFA1850608AF85060807
:10A4700010B5044602F0DEFED4F834330133C4F8DC
:10A4800034332BB94FF4D7620249034802F0E6FD9A
:10A4900010BD00BFA1850608AF850608884209D017
:10A4A00038B504460D46F7F747FA29462046F9F72E
:10A4B00077FE38BD7047036870B50446DB6F984778
:10A4C000B4F8F8522B0A022B24D0032B55D0012BC1
:10A4D00004D1236820461B6B984708B9002070BD43
:10A4E000236820461B6B98470678122EF6D1236806
:10A4F00020461B6B98474578012DEFD123682046F5
:10A50000C4F804631B6B984784F80853C4F800032D
:10A510000120E4E7EDB2236820465B6B29469847AB
:10A520000028DBD02368294620465B6B98470378D8
:10A53000092BD3D12368294620465B6B9847437883
:10A54000022BCBD12368294620465B6B98472368B2
:10A55000867829465B6B20469847C3782946204673
:10A5600046EA03262368C4F804635B6B984701231B
:10A57000C4F8000384F80833CAE7EDB2052DADD85E
:10A58000DFE805F0030F19232D37236820469B6B66
:10A5900098470378C4F8043323689B6B2046984798
:10A5A000E5E723682046DB6B98470378C4F804335B
:10A5B0002368DB6BF2E7236820461B6C984703781F
:10A5C000C4F8043323681B6CE8E7236820465B6CFF
:10A5D00098470378C4F8043323685B6CDEE723688C
:10A5E00020469B6C98470378C4F8043323689B6C1F
:10A5F000D4E723682046DB6C98470378C4F804331B
:10A600002368DB6CCAE70B78DB0913700B78C3F3A4
:10A61000411353700B7803F01F0393704B78D37082
:10A620004B8893808B88D380CB8813817047000040
:10A63000036870B504465B6F0D46984794F80C3379
:10A64000022B05D040F23D120849094802F006FDF0
:10A65000084B204684F81053C4F824330023C4F870
:10A6600028332368BDE870409B6F1847A185060812
:10A67000BB85060849AB0408036810B50446DB6FC8
:10A68000984794F808330BB1002010BDD4F8EC02C1
:10A6900003685B6C9847D4F804238242F4D3D4F85F
:10A6A0000013121A0144C4F80423C4F80013A2B919
:10A6B000022384F80C3394F80A334BB1236804F571
:10A6C0003D71204684F80A239B6E98470120DCE701
:10A6D00001212046FFF7ACFFF8E7D4F8EC02D4F8EC
:10A6E00020430368A2421B6C28BF22469847EDE72F
:10A6F000036813B50446DB6F984794F81C33012BAD
:10A7000006D800230F491A4600930F4802F03AFF7B
:10A7100094F80C3323B100230C491A460093F4E754
:10A7200094F80B33032B0BD02046FFF7A5FF38B965
:10A73000D4F8EC020368DB6C02B0BDE810401847A7
:10A7400002B010BDE68506080E0115800E860608CB
:10A7500038B503680446DB6F984794F80833012B3B
:10A7600037D1D4F8045325B994F8093353B384F896
:10A770000953D4F82033D4F8EC029D42D4F80013E6
:10A7800028BF1D4603682A469B6C9847D4F80033BF
:10A790002B44C4F80033D4F804335B1BC4F80433EF
:10A7A00083B994F809236AB9022384F80C3394F826
:10A7B0000A334BB1236804F53D71204684F80A231F
:10A7C0009B6E9847012038BD01212046FFF730FFDE
:10A7D000F8E70020F7E70000036813B50446DB6FD5
:10A7E000984794F81C33012B06D800230B490C48DA
:10A7F0001A46009302F0C6FE94F80B33032B0BD0DD
:10A800002046FFF7A5FF38B9D4F8EC020368DB6CEB
:10A8100002B0BDE81040184702B010BDE68506083A
:10A820000E011580036870B504465B6F0D469847AE
:10A8300094F80C33032B05D04FF4C3720849094830
:10A8400002F00CFC084B204684F81053C4F8243363
:10A850000023C4F828332368BDE870409B6F184775
:10A86000A18506085886060829B50408036810B5AE
:10A870000446DB6F9847012004F21D33C4F804033B
:10A88000C4F8003384F8080310BD036810B504460B
:10A89000DB6F984794F81C33042B05BFB4F82E33B4
:10A8A00001200020A4F8FA3201BF04F54C73C4F86B
:10A8B0000403C4F8003384F8080310BD036810B51E
:10A8C000DB6F044698470423204694F8F82284F866
:10A8D0000C332368B4F8FA121B6F9847012010BD9F
:10A8E000036870B504465B6F0D46984794F80C33C7
:10A8F000042B05D04FF4EB720849094802F0AEFB77
:10A90000084B204684F81053C4F824330023C4F8BD
:10A9100028332368BDE870409B6F1847A18506085F
:10A9200084860608D9AB0408036810B50446DB6FBB
:10A93000984794F81C33042B02D0B4F8FA3233B998
:10A9400094F8F632012B25D0022B02D023B300203D
:10A950001FE0B4F8FA2222F08F03002BF7D112F097
:10A960000F030CD0530003F01E0343EAD213182246
:10A97000023B02FB034393F83030C3F34003074A22
:10A98000012013800223C4F80023C4F8043384F8A0
:10A99000080310BD0023F2E70123F0E7A4EE002432
:10A9A000036810B5044690B0DB6F9847D4F8EC020A
:10A9B000D4F8202369460368DB6B984704F53D72A1
:10A9C00069462046FFF71FFE00231146C4F80833EE
:10A9D000C4E9C033012384F80C3323685B6E9847C5
:10A9E00010B010BD036813B50446DB6F984794F8A8
:10A9F0001C33012B06D800230A490B481A46009342
:10AA000002F0C0FD012394F80C2384F82C332AB9FA
:10AA1000204602B0BDE81040FFF7C2BF84F82D33D6
:10AA200002B010BDE68506080E0115802DE9F04143
:10AA30001D46036804460F465B6F1646984794F818
:10AA40000C33012B05D040F2BA220A490A4802F021
:10AA500005FB0A4B204684F81073C4F82433002306
:10AA6000C4F828332368C4E9C5659B6FBDE8F0418D
:10AA7000184700BFA1850608AC860608E1B30408A4
:10AA8000036870B50446DB6F9847B4F8FC120029E0
:10AA90003FD094F8F42294F80833012A23D1012BF3
:10AAA00006D0D4F8EC020368DB6CBDE870401847B0
:10AAB000D4F804338B4202D90B46C4F804139942EC
:10AAC00009D9D4F82023B3FBF2F102FB113313B9F7
:10AAD000012384F809330223204684F80B33BDE8B0
:10AAE0007040FFF735BED4F8EC02002BDBD1D4F870
:10AAF00004338B42D7D10122016884F80B23D4F8A8
:10AB000020230D6C9A42D4F8001328BF1A462B4616
:10AB10000BE0D4F8EC02D4F804230368002AC3D174
:10AB200003219B6C84F80B131146BDE87040184755
:10AB3000036810B5DB6F04469847002384F82D3373
:10AB4000032384F80B3310BD036810B5DB6F044694
:10AB50009847002294F8103384F80C2394F82D239E
:10AB600022B12046BDE81040FFF7E2BF33B9D4F868
:10AB7000EC020368BDE81040DB6C184794F80B3317
:10AB8000012B0AD10323D4F8EC0284F80B330368B9
:10AB90009B6C1146BDE810401847022B07D10323D8
:10ABA000D4F8EC0284F80B3303681B6CF1E710BD9A
:10ABB000036810B5DB6F04469847002384F82C33F4
:10ABC00094F80C3323B92046BDE81040FFF7B0BF1E
:10ABD000012384F82D3310BD036810B5DB6F0446E4
:10ABE0009847002294F8103384F80C2394F82D230E
:10ABF00022B12046BDE81040FFF79ABF63B1B4F818
:10AC0000FA322046A4F82E33B4F8F83284F8303300
:10AC1000BDE81040FFF734BFD4F8EC020368BDE88C
:10AC20001040DB6C1847036810B504465B6F98470B
:10AC300094F8F03283B9D4F8EC02214603689B689B
:10AC40009847D4F8EC02402103689B6B9847012396
:10AC5000C4F8200384F8F032236820469B6FBDE8D7
:10AC60001040184738B5036804465B6F984794F85E
:10AC70001C5323682046EDB29B6F98472B1F584208
:10AC8000584138BD036810B504465B6F98472046AD
:10AC9000FFF7C9FF94F8F1323BB9D4F8EC0203682E
:10ACA0005B699847012384F8F132236820469B6F43
:10ACB000BDE81040184700002DE9F74F984603689B
:10ACC0000E4605465B6F1746984716F0700F01D188
:10ACD000330706D10023264926481A46009302F07E
:10ACE00051FC95F8F292B9F1000F07D12B68284674
:10ACF0009B6F9847484603B0BDE8F08F7400182357
:10AD000004F01E0444EAD614023C5C4305EB040A3A
:10AD10009AF830B01BF0010B05D04FF48E62164943
:10AD2000164802F09BF9B7F5806F04D940F27142E2
:10AD300011491348F5E7D5F8EC023A463146036865
:10AD4000D3F850904346C84781460028CED004F13E
:10AD50001C000C992844FFF7A1FB9AF830308AF8C0
:10AD600031B043F00103AAF82C708AF83030BDE707
:10AD7000CF86060804011580A1850608EE86060820
:10AD800010870608D0F8EC0203685B6B184738B5EB
:10AD900003680D4604465B6F98472B0720461BBF90
:10ADA0006B001822D4F8205303F01E031FBF43EAA0
:10ADB000D513023B02FB03439D8D23689B6F98478D
:10ADC000284638BD0368F7B50E465B6F05469847C1
:10ADD00036F08F0701D1320706D1002317491848F2
:10ADE0001A46009302F0CEFB7400182304F01E04F0
:10ADF00044EAD614023C03FB045494F83030DB07D9
:10AE000009D42846FFF72EFF80B140F28C520D493D
:10AE10000D4802F023F994F831303BB1D5F8EC023B
:10AE200031460368DB6E984784F831702B682846FA
:10AE30009B6F03B0BDE8F040184700BFCF860608FF
:10AE400004011580A185060828870608036873B5E4
:10AE50000E465B6F0446984716F0700F01D131071C
:10AE600006D100231A491B481A46009302F08AFBB8
:10AE70007500182305F01E0545EAD615023D03FBB3
:10AE8000054595F83030DA0709D42046FFF7EAFE89
:10AE9000B0B140F2CC421049104802F0DFF843F064
:10AEA0000203314685F83030D4F8EC0203689B6D1C
:10AEB000984795F831301BB131462046FFF782FFA5
:10AEC000236820469B6F02B0BDE87040184700BF62
:10AED000CF86060804011580A18506082887060884
:10AEE000036810B50446DB6F984794F81C33042BB5
:10AEF00002D0B4F8FA32A3B994F8F632022B10D18A
:10AF0000B4F8FA1231F08F000BD111F00F030AD010
:10AF1000B4F8F83223B92046C9B2FFF797FF0120F1
:10AF200010BD0020FCE71846FAE700000368F7B5FB
:10AF30000E465B6F0446984716F0700F01D131073B
:10AF400006D100231C491D481A46009302F01AFB43
:10AF50007500182705F01E0545EAD615023D07FBCA
:10AF6000054393F83020D20709D42046FFF77AFE34
:10AF7000D0B140F2F1421249124802F06FF893F852
:10AF800031301BB131462046FFF71CFF07FB05455A
:10AF9000314695F8303023F0020385F83030D4F88C
:10AFA000EC020368DB6D9847236820469B6F03B073
:10AFB000BDE8F040184700BFCF86060804011580A1
:10AFC000A185060828870608036810B50446DB6FCC
:10AFD000984794F81C33042B02D0B4F8FA32A3B982
:10AFE00094F8F632022B10D1B4F8FA1231F08F0037
:10AFF0000BD111F00F030AD0B4F8F83223B9204670
:10B00000C9B2FFF793FF012010BD0020FCE71846EE
:10B01000FAE700002DE9F341984603680D4617460C
:10B020005B6F0646984735F08F0201D1290706D19C
:10B030000023224922481A46009302F0A3FA6C002A
:10B04000182304F01E0444EAD514023C03FB0464F4
:10B0500094F83030DB0709D43046FFF703FE80B1A7
:10B0600040F2AF521749184801F0F8FFA38D43454D
:10B0700004D91346154916480092DEE794F83120AA
:10B0800042B13368002530469B6F9847284602B08E
:10B09000BDE8F081D6F8EC0229460268D2F860805B
:10B0A0003A46C047054620B194F83130013384F860
:10B0B0003130336830469B6F9847E7E7CF86060804
:10B0C00004011580A185060828870608368706082A
:10B0D00005011580036837B50D465B6F0446984738
:10B0E00015F0700F01D12A0706D100231549164823
:10B0F0001A46009302F046FA6B00182203F01E0372
:10B1000043EAD513023B02FB034393F83030DB07DD
:10B110000AD42046FFF7A6FD054660B140F2E95289
:10B120000A490B4801F09AFFD4F8EC02294603685B
:10B130005B6E98470546236820469B6F98472846D4
:10B1400003B030BDCF86060804011580A18506082E
:10B15000288706082DE9F7431F4603680D46064673
:10B160005B6F9046984735F08F0301D1290706D1D0
:10B170000023244924481A46009302F003FA6C0085
:10B18000182204F01E0444EAD514023C02FB0464B5
:10B1900094F83020D20709D43046FFF763FD80B120
:10B1A00040F20A6219491A4801F058FFA28DBA42CA
:10B1B00004D21A46174918480093DEE794F8313054
:10B1C00043B13368002530469B6F9847284603B04B
:10B1D000BDE8F083D6F8EC02294642460368D3F86E
:10B1E00068903B46C847054650B194F83130E78532
:10B1F000013384F83130336830469B6F9847E5E778
:10B20000E085F8E78787060804011580A185060810
:10B2100028870608A587060805011580036837B545
:10B220000D465B6F0446984715F0700F01D1290752
:10B2300006D10023124913481A46009302F0A2F9DE
:10B240006B00182203F01E0343EAD513023B02FBF6
:10B25000034393F83020D2070AD42046FFF702FDBB
:10B26000054630B140F249620749084801F0F6FE50
:10B27000DD8D236820469B6F9847284603B030BD7C
:10B28000CF86060804011580A185060828870608D0
:10B29000036870B50446DB6F0D46984794F81C238D
:10B2A00084F81C53AA42D3B21FD0032B08D9032D14
:10B2B0000ED92368294620461B6EBDE8704018470A
:10B2C000012BF6D9012DF4D82046FFF771FCF0E7E9
:10B2D0004FF43472002104F11C0016F0B1FC00237D
:10B2E00084F81D3384F8F232ECE770BD036810B5C2
:10B2F0000446DB6F9847D4F8EC0294F8F812036820
:10B30000DB6A9847B4F8F8322BB902212046FFF7E0
:10B31000BFFF012010BD0321F8E7036810B5044604
:10B32000DB6F984794F8F81284F81D1351B9D4F8DC
:10B33000EC0203681B6A984703212046FFF7A8FF29
:10B34000012010BD0123204684F8F232032384F843
:10B350000C332368DB6E9847F2E7036810B50446A8
:10B36000DB6F984794F8F532C3BB94F8F7320B2B98
:10B3700034D8DFE803F0060B331033151A331F24DB
:10B38000292E2046BDE81040FFF7CEBA2046BDE882
:10B390001040FFF719BE2046BDE81040FFF7A0BDE2
:10B3A0002046BDE81040FFF7A1BF2046BDE8104091
:10B3B000FFF781B82046BDE81040FFF757BA204696
:10B3C000BDE81040FFF7A9BF2046BDE81040FFF7D9
:10B3D0005CBA2046BDE81040FFF770BA002010BDEF
:10B3E000036810B5DB6F04469847002094F81033CB
:10B3F00084F80C0394F82D03D4E9C52190B1012BF6
:10B400000BD8022304F53D712046012284F80C3349
:10B410002368BDE810409B6E18472046BDE81040E9
:10B42000FFF786BB042B12D12046FFF796FF30B9F9
:10B43000D4F8EC020368BDE81040DB6C184794F8C0
:10B440000C3373B92046BDE81040FFF719BB032B3E
:10B45000EED0012084F8083384F80A03C4E9C0213F
:10B46000F0E710BD036810B50446DB6F9847022172
:10B470002046FFF70DFF0023204684F81E33FFF718
:10B4800097FB23682046DB6DBDE810401847036832
:10B4900010B504465B6F984794F8F1323BB1D4F88D
:10B4A000EC0203689B699847002384F8F13294F812
:10B4B0001C33012B03D901212046FFF7E9FE0023AD
:10B4C000204684F81D3384F81E332368BDE81040FD
:10B4D0009B6F1847036810B504465B6F984794F854
:10B4E000F03253B12046FFF7D2FFD4F8EC020368E4
:10B4F000DB689847002384F8F032236820469B6F6E
:10B50000BDE81040184738B503680D460446DB6FA8
:10B51000984745B994F81C332BB129462046BDE81D
:10B520003840FFF7B5BE38BD036870B50446DB6F21
:10B53000984794F82D3394F8106303B97EB92046E8
:10B54000FFF790FB054650B901464FF4347204F101
:10B550001C0016F075FB84F81D5384F8F25200238A
:10B5600084F80C3394F82D3323B12046BDE87040A5
:10B57000FFF7DEBAD4F8EC02036856B1DB699847EE
:10B5800020460421FFF784FE2046BDE87040FFF707
:10B5900077BADB6CBDE87040184700002DE9F04732
:10B5A000054698461D4B04460F46914645F81C3B00
:10B5B00000F53B7A2E4630461836F6F715FF56450D
:10B5C000F9D1BDF820304FF4347200212846238190
:10B5D000A4F80490A4F8068016F032FB282200217B
:10B5E00004F53D7016F02CFB002301222046C4F820
:10B5F000EC72A4F8F03284F8F232C4F8343384F8F0
:10B60000303384F81C2384F81D3384F81E33C4E9D6
:10B61000C833C4E9CA33BDE8F08700BFDC87060839
:10B620000D4B70B50360044690F8F0322BB140F238
:10B6300062520A490A4801F011FD04F53B7504F114
:10B640001C06FFF747FFB54204D0183D2846F6F721
:10B6500078F9F8E7204670BDDC870608A185060862
:10B66000C6870608036837B50D46DB6F0446984762
:10B6700015F0700F01D12B0706D100230F49104898
:10B680001A46009301F07EFF6B00182203F01E03A0
:10B6900043EAD513023B5343E11891F831205AB1E4
:10B6A0001C33013A1C4481F831202046F8F74DFE46
:10B6B00010B12046FBF716FF03B030BDCF86060859
:10B6C000040115804FF0FF3100F076B970B50D46DA
:10B6D00004464C301646FDF7F7FA2DB92A4629469E
:10B6E000204600F015F804E02EB92946204600F067
:10B6F00046F8204670BD32462946F1E710B50446AB
:10B7000000F04FF804F14C00F7F7C2F9204610BDE5
:10B71000032938B5044607D9D31C23F003039A1A2A
:10B72000891A1A4621F0030100230D46E260636185
:10B7300015BB236122622560C4E9065100F006FAB8
:10B7400000F006FA2581606004F13000A57284F8EB
:10B750002450C4E90A5500F01BFA00280BDB04F161
:10B76000440000F00DFA002805DB04F1480000F069
:10B7700007FA00EAE07038BD01336D08D8E770B50C
:10B78000054608460E4615F00BFE044630B102464B
:10B7900031462846FFF7BCFF6C6170BD4FF0FF30AB
:10B7A000FBE770B504460568B5B9A36A1BB14FF055
:10B7B000FF31E06A984704F1480000F0E3F904F132
:10B7C000440000F0DFF904F1300000F0E9F96069AD
:10B7D000BDE8704015F0ECBDEE6836B9EB6913B109
:10B7E00005F124009847AD68DEE7F36913B106F16F
:10B7F00024009847F668F0E7F8B500F148070646D8
:10B8000001F12705384600F0BEF925F0030506F1E1
:10B810001803B4695CB9F3699D4223D8346A5B1B91
:10B820006219F361012332622560A37107E0226887
:10B83000954213D8E26872B11A60A36893603846E3
:10B8400000F0A3F900234FF0FF32E361C4E90532B1
:10B8500024342046F8BDA2681A60F0E704F108031A
:10B86000A468D7E7384600F090F9F2E7F8B551F848
:10B87000083C05460C460BB108469847EB6833B1C7
:10B88000A4F12406B34202D82B6AB34203D20023A8
:10B8900004F81E3CF8BD05F14807384600F073F97E
:10B8A00005F11802AB69A3B1186854F8241C88424A
:10B8B0000BD30ED144F8183C9B6844F81C3C384626
:10B8C0001660BDE8F84000F060B903F108029B681B
:10B8D000E9E7002344F8183C1368EEE7F8B54B6934
:10B8E000164600F1440705469B1A0C46002BA8BFDC
:10B8F000D218038938464A618B8000F044F92A4601
:10B9000013687BB358696169A0EB010CBCF1000FAF
:10B9100025DB88422AD19B68A36013B104F108019A
:10B92000196113682146002041F80C3F98601961A5
:10B93000AB6A146022616BB195F8242052B12A6879
:10B94000A24207D1E2682AB96169E86A891B21EA43
:10B95000E17198473846BDE8F84000F016B903F1A8
:10B960000802CDE7A3600023E360E1E7214641F848
:10B97000083F1961F7E7F8B5144605460F46A2F1EE
:10B98000240600F0E5F854F8103C02463146034422
:10B9900044F8047C284644F8103CFFF79FFF2B69CD
:10B9A00014F81E4C05F130009C40EB68F61A00F0CC
:10B9B000F9F834432046F8BD2DE9F34704460F4615
:10B9C0004FF0000800F0C4F804F14406054607EB08
:10B9D000000984F82480304600F0D5F8636801A996
:10B9E0005B1B002B2368D8BF65600193002B3CD004
:10B9F0005A69521B002A34DD23601C61C1F80080A3
:10BA0000019D15B1238901332381304600F0BDF833
:10BA100001A965BB019D002D36D100F099F8002FDA
:10BA200082465DDBA9EB0005002D5BDCA36A9BB1C0
:10BA3000304600F0A8F8A36A43B1226832B15169D8
:10BA4000E06AA1EB0A0121EAE1719847012330463F
:10BA500084F8243000F099F80023A37202B0BDE806
:10BA6000F08703F108019B68C0E72360C6E7A86878
:10BA70002B4600229A601A46DB68002BFAD10A6036
:10BA800005F108010546C4E72B6AD5F808A013B1F3
:10BA900005F124009847AA69002A0BDB6B6913445F
:10BAA0006B6100F055F8294602462046FFF716FF65
:10BAB0005546B0E7E3686BB1AB420BD8236AAB42A3
:10BAC00008D3AB7922690133DBB213FA02F208BF63
:10BAD0000123AB7105F124012046FFF7C7FEE7E71C
:10BAE0004FF0FF35304600F04EF823683BB15869FF
:10BAF000A0EB0A0020EAE070854228BF05463046E8
:10BB000000F043F8294604F1300000F04EF8A37A23
:10BB10007BB1304600F037F8A37A3BB100233046C2
:10BB2000A37202B0BDE8F04700F02FB8304600F035
:10BB30002CF800F00DF805464DE740F8101C704752
:10BB400040F80C1C704740F8081C704701F0B0BD6D
:10BB500007B501F066FB70B1084B6846196800F044
:10BB600077FF4FF47A720023DDE9000113F0C2F889
:10BB700003B05DF804FB02F067FBF9E700FD002469
:10BB800000207047704701F055BB01F069BB000011
:10BB9000024908B502F032FB002008BDAC88060857
:10BBA00002F035BB012102F02FBB08B5012341EAA9
:10BBB000E172194602F046FB431E5842584108BD47
:10BBC00030B52A4C89B005462368BFF35B8FDA078E
:10BBD00011D4204601F026FF68B1254A4FF4407188
:10BBE0002448FFF773FD244A2449224801F00AFF44
:10BBF000204601F039FF224C2368BFF35B8FDB073F
:10BC000013D4204601F00EFF78B11E4B4FF40062B2
:10BC100018211D480095FEF773FB174A1B491A4867
:10BC200001F0F0FE204601F01FFF174802F0C5FCAE
:10BC300010F0EF0016D1164B154A0E49CDE902302F
:10BC4000034604A8FBF7C2FC04A90F4802F02EFC2F
:10BC5000044604A8F5F775FE24B12F220D490E48BD
:10BC600001F0FCF9034809B030BD00BF68F70024BB
:10BC7000C8F700246CF7002400000024FDB6040877
:10BC8000A8EE002468EF0024ACEE002465E604086A
:10BC9000C5B60408CB880608E288060808B502483D
:10BCA000FFF78EFF08BD00BFF1880608704700004F
:10BCB000EFF3108372B6054A117831B9DB430449BA
:10BCC00003F001030B70012313707047C8FA0024BE
:10BCD000C9FA002408B5EFF31083DB4313F0010326
:10BCE00004D036220549064801F0B8F9054A137018
:10BCF000054B1B7803B162B608BD00BF1989060861
:10BD000035890608C8FA0024C9FA0024014B1878BE
:10BD1000704700BFC8FA0024084A094B10B5D2F892
:10BD200094409C42FBD1036829B181680B604FF4B9
:10BD30004073536110BDC1681B04F7E700640258EB
:10BD40000003008070B50E46044615460EF09EFABC
:10BD5000013609D0204600210EF0BCFA29462046C3
:10BD6000BDE870400EF0B2BA70BDF8B50F4604469B
:10BD700015461E460EF08AFA01370CD02046314691
:10BD8000FFF7CAFF01210EF0A5FA29462046BDE8BB
:10BD9000F8400EF09BBAF8BD0022FFF7D3BFFFF7C3
:10BDA000D1BF13460022FFF7E0BF0022FFF7F9BF23
:10BDB0002DE9F041174604460D461A46069E4FB936
:10BDC000FFF7C0FF01350AD031462046BDE8F041FB
:10BDD000FFF7A2BF3346BDE8F041FFF7C6BFBDE89D
:10BDE000F08100000048704750890608024B1B682C
:10BDF0000BB1024818477047380D002450890608D7
:10BE000013B50446601C0FD102B010BDA3420AD185
:10BE1000204689680FF006FE0021204602B0BDE8EA
:10BE200010400FF0B9BE0C31B1F900305A1CEDD101
:10BE30000023224602490348009301F0A3FB00BF00
:10BE40007C8906083001018007B5024608468A420F
:10BE50000AD0531C08D0013005D0002304490548FE
:10BE6000009301F08FFB104603B05DF804FB00BFA8
:10BE70008D89060830010180B1F900305A1C01D1CA
:10BE800018467047834201D1486870470C31F3E788
:10BE9000421C13B504460AD0FFF7EEFF431C06D13F
:10BEA0000023224603490448009301F06BFB02B0D3
:10BEB00010BD00BF9E89060830010180B1F9003035
:10BEC0005A1C01D118467047834201D188687047D7
:10BED0000C31F3E7421C13B504460AD0FFF7EEFF1E
:10BEE000431C06D10023224603490448009301F075
:10BEF00049FB02B010BD00BFBE89060830010180B9
:10BF0000F8B5446894F832608EBB03685B68984764
:10BF1000226A82422BD02369821A20621A40A368C7
:10BF2000A2FB03C194F93420CAB1606A10EB0C057E
:10BF300041F10001002A1BDBC2F12000A2F1200325
:10BF400025FA02FC01FA00F021FA03F3D1404CEA91
:10BF5000000C4CEA030C0CFA02F2AA1A6262D4E951
:10BF60000A3213EB0C0341EB0202C4E90A32F8BDBA
:10BF7000E768334628463A4612F00CFF844607FB32
:10BF800010506062EBE7824206D98A420BD98842A0
:10BF900094BF002001207047884206D98A428CBF96
:10BFA00000200120704701207047002070470000EA
:10BFB0002DE9F04146680546336B23F07F4828F0B1
:10BFC000FF08B8F1000F5CD1FFF79AFF7368002BF0
:10BFD00059D0D3E90003D6E90A1281429A4104D329
:10BFE0002B68BDE8F0415B6918476C68D4E90A1218
:10BFF000401A63EB020CE369D4E90572824273EBE9
:10C000000C031FD3E368A3FB000103FB0C1194F99D
:10C010003330A3B1A26802F1FF3C1CEB000041F1F8
:10C020000001002B1BDBC3F1200CA3F12002D84040
:10C0300001FA0CFC21FA02F240EA0C00104387429C
:10C0400028BF0746236A1F4423691F40336ABB4247
:10C0500009D140F2C9121149114800F0FFFF4346CF
:10C0600012F098FEEBE72B6838461B6998472B685F
:10C070005B6898473A460146306AFFF784FF00281C
:10C08000AED1BDE8F0817369306A326918442B681B
:10C0900010401B69BDE8F041184700BFF189060850
:10C0A000038A06084368F7B593F830200546002A4E
:10C0B00040F0838093F83230002B7ED103681B68F8
:10C0C00098472B68DB69984703682BB91A463C49A7
:10C0D0003C48009301F056FA1F463B4A1446B7FB12
:10C0E000F2F204FB12722746002AF7D136491F22CA
:10C0F0006E680127B1FBF4F1B160013A03D307FA8E
:10C1000002FC6145F9D186F83320B3FBF4F2B2F1B9
:10C11000004F4FF01F03F26006D00124013B03D310
:10C1200004FA03F7BA42F9D186F834304068071FA1
:10C130001C2F05D90023254925481A460093C9E735
:10C1400020284FF0070418BF012304FA07F408BFA2
:10C150004FF0FF334FF0000718BF834074614FEA80
:10C16000E47018BF03F1FF333361A4FB014301FB0B
:10C170000031531E47F1FF3CE0183B4641EB0C01F8
:10C1800012F008FE2B68C6E906015B68C6E9007775
:10C1900098476B6830620021012200205F621A8696
:10C1A00083F83270C3E90A012846FFF7A9FE284642
:10C1B00003B0BDE8F040FFF7FBBE03B0F0BD00BF29
:10C1C000278A06080E01048040420F00408A0608B4
:10C1D00005010480F3B4069C002745688C606C68F8
:10C1E000C1E9002334B9CC607FB9696002B0F0BC0A
:10C1F000FFF7DEBE666801962668B242019E73EBC9
:10C200000606F0D32746E468ECE7F960D5E90A4171
:10C2100094429941EAD202B0F0BC704738B5054665
:10C220000C46FFF73FFF01F005F86B681C60BDE8A6
:10C23000384001F015B870B5054600F0FBFFD5E9B0
:10C240000034DB68984794F832301BB1BDE8704089
:10C2500001F006B8012384F831306368A3B12846A1
:10C26000FFF74EFE6368D4E90A62D3E90001864213
:10C270008A4109D36A68DB68526863602368002BCF
:10C28000EBD090689847E8E70023284684F83130DF
:10C29000FFF78EFEDAE72DE9F34104460D46174617
:10C2A0001E46DDF8208000F0C5FF2046FFF728FE7F
:10C2B0003A46334629462046CDF80080FFF78AFFEC
:10C2C00002B0BDE8F04100F0CBBF38B505460C46E2
:10C2D00000F0B0FF6A685368A34209D1DB682846C2
:10C2E0005360FFF765FEBDE8384000F0B9BF134664
:10C2F000002BF8D0DA68A242F9D1E268DA60F2E7FE
:10C3000038B50446FFF7CEFE00F094FF2046FFF755
:10C31000F7FD6368D3E90A4500F0A2FF20462946ED
:10C3200038BD7047004870477C8A0608024B1B687E
:10C330000BB10248184770473C0D00247C8A060860
:10C3400008B5BFF35F8F1C4BD3F8902012F47C4FDD
:10C35000C2F3072104D13B221849194800F07EFEA0
:10C3600000221046C3F894208A421FD11022C3F83D
:10C370009C20144AC3F8A0201322C3F89C20124A20
:10C38000C3F8A0201122C3F89C20104AC3F8A020B3
:10C390000F4AC3F89C200F4AC3F8A0200722C3F815
:10C3A0009420BFF34F8FBFF36F8F08BDC3F8982061
:10C3B0000132C3F8A000D7E700ED00E0C18A06080B
:10C3C000D08A060839F00206390702133FF50B132D
:10C3D0001200008039000213B1F90C20B1F90410E9
:10C3E00010F038BD15F0DABC2DE9F04F814C85B066
:10C3F0000746894601939246636B1BB19847E36BEE
:10C400000133E3632369D3B1002238061A7023D4C1
:10C41000B9F1000F11D0606803781BB1494616F0DE
:10C420006BFB50B9A0680378002B00F0DD80494613
:10C4300016F062FB002840F0D780A3692362A36B4B
:10C440003BB10023E56BE363013DA36B9847002DEF
:10C45000FADC05B0BDE8F08FBAF1000FEDD0B9F10C
:10C46000000FEAD0E36A002BE7D0237803EA070243
:10C47000D106E4D01A06D4E9045601D4012F10D114
:10C48000019B52463146284619F01CF9012F50D124
:10C49000236B002B4DD020699847236B5648984753
:10C4A000CBE713F040085ED09B0640D5534A314697
:10C4B000284615F03DFE864239DD002837DD05446B
:10C4C000361A082F4DD037D8022F39D0042F46D036
:10C4D0004FF00008C346636ADBB10021019B52465E
:10C4E0000846039319F0EEF8B8F100024044636A7D
:10C4F00018BF012200EB82009847414A03463146AB
:10C50000284615F015FEB04203DA002801DD054487
:10C51000361A082F5DD05FD8022F27D0042F55D0B0
:10C52000384A3146284615F003FE0E2024E0002E3E
:10C53000C7DCE36A2069B2E7102FC9D1324B00E0B3
:10C54000324B2F4A3146284615F0F2FD052E48DDC4
:10C550000535053E4FF005084FF0010BBBE72C4BAE
:10C56000EFE72C4BEDE7002EB4DCE2E74B462A4A1E
:10C570003146284615F0DCFDB042DADA0028D8DD75
:10C58000361A0544019B52463146284619F09AF85E
:10C590008642CEDD0028CCDDA36A0544361A63B19D
:10C5A0009847174A03463146284615F0C1FD864292
:10C5B000BFDD0028BDDD0544361ABBF1000FB8D041
:10C5C000164A3146284615F0B3FDB2E74B46144AE9
:10C5D000CEE74B46134ACBE7102FA1D14B46124A68
:10C5E000C6E74FF00008B7E7BAF1000F7FF43AAFA3
:10C5F00023E700BF400D0024D78E0608DD8A060819
:10C60000E98A06083A8B0608F88A0608E38A0608CB
:10C61000EC8A0608F28A0608FE8A0608498B060894
:10C620000D8B06081C8B06082B8B06080CB407B56F
:10C6300004AB53F8042B0193FFF7D6FE03B05DF86B
:10C6400004EB02B070470000024B1B6803B11847AF
:10C65000704700BF40FB002410B5044600F0EAFD1F
:10C66000204610BD10B5044600F0FAFD204610BD6E
:10C67000007B704738B50D4B0D46027304460360CE
:10C680000023C0E901310A48FCF7E0F801F022FE7E
:10C6900055B1084B1A681C6062600548FCF7D6F873
:10C6A00001F034FE204638BD6560F6E7608B060871
:10C6B00048FB002470FB0024144B10B503600446B3
:10C6C0001348FCF7C3F801F005FEA3682BB111492C
:10C6D00062680B68A34212D10A600F4B0C481A68BB
:10C6E000A24204BF00221A60FCF7B0F801F00EFE6F
:10C6F000237B13B9201F01F01FFC204610BD1946F3
:10C700005B68A342FBD14A60E7E700BF608B060885
:10C7100048FB002470FB002444FB002410B50446B1
:10C72000FFF7CAFF1021204601F0F0FB204610BDA4
:10C73000F8B5064617480D46FCF788F801F0CAFD23
:10C74000154B1C6884B9072D1BD12A463146134866
:10C7500015F046F9A8B90F48FCF778F801F0D6FDB6
:10C760000F4B1C682046F8BDA76887B1384615F006
:10C7700067FFA8420BD12A463146384615F030F9FA
:10C7800028B90448FCF762F801F0C0FDEAE76468E4
:10C79000D8E700BF48FB002470FB00244E8B06083E
:10C7A00044FB0024002070470368012200211B691C
:10C7B00070B504469847051E0DDB23680222002150
:10C7C00020461B69984706462368294635460022BD
:10C7D0001B6920469847284670BD000070B50E467C
:10C7E00000240F490546C0E90044304616F014F80D
:10C7F0003044214603461A782F2A07D101332B6093
:10C8000049B92A220749084800F028FC002AF6D036
:10C8100001310133EFE7FFF78BFF6860284670BDF9
:10C82000B88B0608D48B0608E18B060800687047B1
:10C83000406808B520B1FFF71BFF431E584258411E
:10C8400008BD10B50446FFF7F3FF10B1606800B1F2
:10C85000043810BD406808B520B1FFF709FFB0FAF1
:10C8600080F0400908BD10B50446FFF7F3FF10B192
:10C87000606800B1043810BD4068003818BF01205E
:10C88000704700207047F8B50D46036804468F18BE
:10C890002E461B6D9847BE42236806D09B6C2046EF
:10C8A00016F8011B98470130F5D1236820465B6DCF
:10C8B0009847701BF8BDF8B50E46036804468F18FC
:10C8C00035461B6D9847BD42236805D12368204635
:10C8D0005B6D9847A81BF8BDDB6C20469847431C4E
:10C8E000F4D005F8010BEEE7002070477047000018
:10C8F0000F4B002213B5044640F8043BFFF7BAFE85
:10C900000C4B0D4920462360603363600023636154
:10C9100001F070FB0346606128B9024600900749A8
:10C92000074800F02FFE01F071F8204602B010BD5C
:10C93000708B0608688C0608EA8B0608ED8B0608E3
:10C9400019010180094B10B5036060330446436050
:10C95000406913F04BFD064B20462360503340F8EE
:10C96000043FFFF7A9FE204610BD00BF688C0608F3
:10C97000088C06088E220249024808B500F06EFBBA
:10C98000EA8C0608F78C060810B504460846FFF73F
:10C99000B7FCC4E90001204610BD000010B50446F4
:10C9A000FDF708FA0A4B2046A16940F8203BFFF743
:10C9B000EBFF2046D4E90823C4E90A230022002320
:10C9C000C4E90C230023C4E90E3384F8403010BDC1
:10C9D000288D06084FF0FF30704738B590F83F506B
:10C9E00004460DB1FFF7C6FFFDF704FA94F8403096
:10C9F000A5872BB184F84050BDE8384000F018BF3F
:10CA000038BD000008B50121383000F04DFB18B1E9
:10CA1000024B4FF080625A6008BD00BF00ED00E09D
:10CA200010B50446FDF7E6F900234FF0007284F8D4
:10CA30003F30014B5A6010BD00ED00E010B50446D8
:10CA400001F1300000F042FBC4E90001204610BDB6
:10CA500010B504468969FFF797FF204610BDD0E95D
:10CA60000C32013342F10002C0E90C32D0E90A3243
:10CA700013F57A7342F10002C0E90A327047D0E937
:10CA80000A2312F57A7243F10003FDF7A9B90000F9
:10CA900008B5012380F83F30836B1BB1034B4FF087
:10CAA00080625A60FFF7EBFF08BD00BF00ED00E0B9
:10CAB00090F83C3010B504464BB1002380F83C3070
:10CAC00090F83E3013B9012380F83D3010BD90F846
:10CAD0003F30002BFAD0836B4FF0806201338363C9
:10CAE000034B5A60FFF7BBFF2046FFF7C8FFEDE797
:10CAF00000ED00E037B50D46044689696846FFF74A
:10CB000043FF00980199D5E90A32C01A61EB02018E
:10CB1000B0F57A7F71F1000306D200220023C4E948
:10CB20000023204603B030BDB0F5FA6F71F1000369
:10CB300001D20122F2E700294FF47A724FF000038C
:10CB4000D8BF002112F026F9C4E90001E9E700008E
:10CB500091F83F30F7B505460C4613B991F83C60A3
:10CB600026B1E5221149124800F078FA6846FFF72D
:10CB7000C1FF4FF47A71DDE90030A663A3FB0172B7
:10CB800001FB0022D4E90A16C91942EB0602C4E9E6
:10CB90000A12D4E90C125B1842EB00022846C4E9E1
:10CBA0000C32C5E9003203B0F0BD00BFEA8C0608C4
:10CBB000018D06082DE9F743994690F83F30044669
:10CBC0001746154623B158223249334800F046FA39
:10CBD00090F83C3063B901466846FFF7B9FF009B07
:10CBE000BB42019B73EB090305D3012384F83D305D
:10CBF00003B0BDE8F08321466846FFF71FFF009BA6
:10CC0000B7EB03084FF47A73019FA5FB035669EB5A
:10CC1000070703FB0966D4E90832ED184FF001035A
:10CC200046EB020694F84020A38742B9A269126835
:10CC300092F820203ABB84F8403000F0E3FDB8F1D0
:10CC4000050F94F8403077F100070DD2002384F8E7
:10CC50003E3094F8403023B9012384F8403000F08E
:10CC6000D1FD2A46334608E0002BEFD10123B5F56C
:10CC70007A6284F83E3066F10003204603B0BDE8D6
:10CC8000F043FDF7ADB8B8F1050F77F10007DDD33C
:10CC9000ECE700BFEA8C0608F78C0608102300F0CA
:10CCA00007B8202300F004B8302300F001B8402377
:10CCB0009C46F0B404AE7546E80801D3EFF309864C
:10CCC0000E4F0FCE0FC70FBC0FC740464946524606
:10CCD0005B460FC71DCE3100A60A00D304316E0992
:10CCE00000D248311FC7EFF309806946EFF314867D
:10CCF00063C76046014900F079F800BF74FB002467
:10CD0000F0B52C4E85B000242B4F3546214601341A
:10CD100056F8042B384600F071FA0D2CF6D1AB6CA6
:10CD2000264C02936B6C264801932B6C0093696B25
:10CD3000D5E90E2300F062FA2168224800F05EFA7D
:10CD4000E16AA26AA36AA06AD2B2266BC3F3072380
:10CD5000E76B000CCDE9016700901B4800F04EFA2C
:10CD6000A36A1E0603D5616B184800F047FAA36A50
:10CD7000180403D5A16B164800F040FAEB6C1907B4
:10CD800012D5144800F03AFA2B6DDA070FD5124885
:10CD900000F034FAEB6C5B074CBF1048104805B04C
:10CDA000BDE8F04000F02ABA0E4800F027FA0E481D
:10CDB000EEE700BF74FB00242C8D060800ED00E0B8
:10CDC0003A8D0608898D0608978D0608E68D0608B7
:10CDD000F48D0608028E0608118E0608418E06089C
:10CDE0004D8E0608318E06081E8E060807B50446CD
:10CDF0000D461A48012100F060F968BB184800F0A0
:10CE0000FDF9302C19D0402C1CD0202C1FD1154CF2
:10CE1000154800F0F3F9154800F0F0F9FFF770FF3E
:10CE2000134800F0EBF90D4B00221A7000232A463C
:10CE300010492046009300F0A5FB0F480F4C00F06E
:10CE4000DDF9E8E70E480F4C00F0D8F9E3E70E48AB
:10CE50000E4C00F0D3F9DEE70024E7E781FC002464
:10CE6000598E06083E01FF80828E0608AF8E0608A6
:10CE7000BA8E0608D98E0608918E06083F01FF80FB
:10CE80009A8E06084001FF80A58E06083D01FF80AE
:10CE90002DE9F0410C467746154600F0E9FBE4B178
:10CEA00054F8088CDDB1284614F07AFA064648B1E9
:10CEB000A8454246214628BF2A4614F0C3FD204615
:10CEC00014F076FA3B462A462146304600F088FBAD
:10CED00000F0DEFB3046BDE8F081A046E2E72E46DA
:10CEE000F0E72DE9F0410D461646774600F0C0FB0D
:10CEF00006FB05F8404614F053FA044618B14246C2
:10CF0000002114F09DFE3B4632462946204600F0A3
:10CF10007FFB00F0BDFB2046BDE8F081F8B50D4673
:10CF20001646074600F0A4FB2048FBF78FFC204C78
:10CF300001F0D0F915F1090F33D805F10801384691
:10CF400014F03EFA68B3A26800F10807194B2A44AE
:10CF500005604360A2602269236801322B4422618C
:10CF6000626823609342A0F1040288BF636050F8B6
:10CF7000043C002BB8BFD218A36912685B1B22F0D7
:10CF800001021344A3610948FBF760FC01F0BEF9FC
:10CF900032462946384600F00FFB00F079FB384650
:10CFA000F8BD6369002701336361ECE7E4FB00240B
:10CFB000C8FB0024EFBEADDE00B572465DF804EBA1
:10CFC000FFF7ACBFF8B50C460646174600F050FB1D
:10CFD0001C48FBF73BFC01F07DF91CB354F8042C12
:10CFE000194B9A422BD154F80C2CA4F10C0354F891
:10CFF000085C002AB8BF9B181A68002344F8043C58
:10D0000022F00102114B1968491B19601969013995
:10D01000196199690D44A4F10801AD1A9D6130466A
:10D0200013F0A8FC0748FBF711FC01F06FF9394633
:10D03000204600F005FBBDE8F84000F029BB214682
:10D04000EDE700BFE4FB0024EFBEADDEC8FB00242B
:10D0500000B572465DF804EBFFF7B4BF07B50B46A9
:10D06000009201460022014800F08CFA4401FF8042
:10D0700003460122D3E84F0FC3E8412FC0B2002975
:10D08000F8D17047D0E85F3F5B18C0E8523F002AF4
:10D09000F8D198B27047D0E85F3F5B1AC0E8523FC2
:10D0A000002AF8D198B27047034653E8000F401A9F
:10D0B00043E80002002AF8D170470346D3E84F0F37
:10D0C000C3E8421FC0B2002AF8D1704738B5044601
:10D0D00000F0B0F8D4E9004500F0C2F82046294637
:10D0E00038BD0000084A094B10B5D2F894409C4264
:10D0F000FBD1036829B181680B604FF44073536121
:10D1000010BDC1681B04F7E70064025800030080EB
:10D1100000B589B0154D00F08DF8A52101A8FEF7E6
:10D1200044FE0424012101A8FFF7DCFF284601F09A
:10D1300037F8002101A8FFF7D5FF284601F030F8A5
:10D14000013CEFD104240A4E012101A8FFF7CAFFD8
:10D15000304601F025F8002101A8FFF7C3FF304653
:10D1600001F01EF8013CEFD1DBE700BFF0490200FF
:10D17000801A060073B5002201460446022000F022
:10D18000EDFC0D2600F056F80022254614F8013B70
:10D1900023B902B0BDE8704000F062B80A2B09D193
:10D1A0000D2A07D001220DF1070102208DF807603A
:10D1B00000F0D4FC01222946022000F0CFFC14F834
:10D1C000012CE2E700B5A3B002460B46842101A87A
:10D1D00018F078FA832806D9074B1A681B79CDF81E
:10D1E00083208DF88730002802DD01A8FFF7C2FFF9
:10D1F00023B05DF804FB00BFE98E06080FB407B545
:10D2000004A951F8040B0191FFF7DCFF03B05DF8AE
:10D2100004EB04B07047EFF31080C04300F001004E
:10D220007047EFF30580003818BF01207047FEF704
:10D230006DBD000008B5FEF73BFD064A1368591C9A
:10D2400004D13F2204490548FFF708FF013313606A
:10D2500008BD00BF0CFC0024088F0608188F0608C4
:10D26000044A136823B1013B13600BB9FEF732BDCA
:10D27000704700BF0CFC002408B50B48FFF7F8FE10
:10D2800028B1FFF7D7FFBFF34F8F20BFFDE7FFF7B0
:10D29000C8FF08B1FFF73CFFFFF7BDFF0028F9D03A
:10D2A000012000F0C3FD00BF80FC00242DE9F04107
:10D2B0004D4C0E4698B08046216817464B4801F009
:10D2C000C043B3F1C04FC1F307430CBF4D428DB211
:10D2D0002A46FFF793FF6FF498731D44132D0FD860
:10D2E000DFE805F00A5B5E61646A676D0E0E0E0E84
:10D2F0000E0E0E0E0E0E0E70A1683D48FFF77EFF5B
:10D300004046FFF737FF61683A48FFF777FF4EB1B5
:10D310003948FFF72FFF3046FFF72CFF39463748D3
:10D32000FFF76CFFA1683648FFF768FF2368354AAE
:10D330001A44012A02D9344A934247D1A0680028EE
:10D3400049D1E368002B4CD05968304A002908BF06
:10D350001146E2692E4D0392A2690292626901921E
:10D36000226900922B4A002808BF2A462A48FFF764
:10D3700045FF04A800F0E6FE079B284801939DF8AE
:10D38000183000932168DDE90423FFF737FF2448B4
:10D39000FFF734FF18B0BDE8F081A1682148ADE780
:10D3A000A1682148AAE7A1682048A7E7A16820480A
:10D3B000A4E7A1681F48A1E7A1681F489EE7A168EC
:10D3C0001E489BE71E48FFF719FF99E71D4A934245
:10D3D000B4D00020B5E7C06C80F00800C0F3C000F6
:10D3E000AFE70A49B5E700BF14FC00245E8F0608CA
:10D3F000AF8F0608579006086890060870900608D8
:10D4000074900608C2FE007F4001FF80498F060825
:10D41000D88E0608538F060888900608E190060803
:10D4200058910608C58F0608D58F0608E48F0608B0
:10D43000F78F06080B9006081F9006082E90060826
:10D44000449006083D01FF807047000070B5294BED
:10D450008EB00C46164610EA200538BF1D46302215
:10D46000002102A814F0ECFB234B01952B440394FC
:10D47000012B02D9214B9D4233D1E36B0293636BA5
:10D4800008931F4B5B69DA6B049305925A6B1B6B15
:10D4900006920793FFF7CEFE1A4A13680133012B59
:10D4A000136009D101AD184C0FCD0FC40FCD0FC4BF
:10D4B0000FCD0FC42B68236001AC144D0FCC0FC5EA
:10D4C0000FCC0FC50FCC0FC52368A5F130002B6022
:10D4D0000F4B1B685BB19847FFF7C2FE00200EB0F0
:10D4E00070BD0C4B9D42C8D001AB0296C8E7FFF758
:10D4F000ABFFF1E70101FF80C2FE007F4001FF802A
:10D500007C0C00247CFC002448FC002414FC002437
:10D5100010FC00243D01FF800FB407B501210D4828
:10D520007546FFF7CAFD044688B901462A460A48EF
:10D53000FFF78CFF224621460848FFF7B7FE05A9F2
:10D5400004980191FFF73EFE0548FFF713FEFFF731
:10D5500093FE00BF81FC00240001FF807291060849
:10D56000D78E060800207047014B1878C0B270476C
:10D5700081FC002400B5114672465DF804EBFFF70C
:10D5800065BF000080B506460C460A480121F046FA
:10D5900017461D46FFF791FD48B9424639463046C9
:10D5A000FFF754FF029A29462046FFF77FFEFFF758
:10D5B00063FE00BF81FC002438B50B4606490446D3
:10D5C0000D6835B105490978012902D801460020C6
:10D5D000A847204638BD00BFB0FC0024ACFC0024A6
:10D5E00037B5044610461A46074B1D6845B1074B30
:10D5F0001B78012B04D80B46009021460120A84738
:10D60000204603B030BD00BFB0FC0024ACFC0024B9
:10D6100037B5044610461A46074B1D6845B1074BFF
:10D620001B78012B04D80B46009021460220A84706
:10D63000204603B030BD00BFB0FC0024ACFC002489
:10D640000A460949034610B40C684CB107490978E9
:10D65000012905D8A446002103205DF8044B60474A
:10D660005DF8044B704700BFB0FC0024ACFC002404
:10D6700008B50548FBF7EAF800F02CFE034A1378DA
:10D680000133137008BD00BF84FC0024ACFC0024EF
:10D69000054A064808B51378013B1370FBF7D6F826
:10D6A000BDE8084000F032BEACFC002484FC00243D
:10D6B00038B5064C23683BB9054DFEF793FB014690
:10D6C0002846FFF76BF92560206838BD00FD00246F
:10D6D000B8FC002408B5836823B9054B1B6893F890
:10D6E0003D0008BDC06898470028F6D0F9E700BFA4
:10D6F00000FD0024F7B504464FF0FF356FF00046FB
:10D70000164F2046FFF7E6FF30BBD4E90023B342B3
:10D7100008BFAA4202D03868FFF74CFA01A8FEF70A
:10D720009BFF2046FFF7D6FF98B9D4E90023B34208
:10D7300008BFAA4207D100F09FF801A8FEF792FFA8
:10D74000BFF36F8FDDE73B6893F83C30002BF2D1DD
:10D75000F3E701A8FEF786FF03B0F0BD00FD00244B
:10D7600030B587B00D4D0446CDE902230A9B0493E2
:10D770000B9B0593FFF79CFF02A8FFF7BBFF2868F0
:10D78000FFF72BF968462968FFF7E2F92046DDE943
:10D790000023C4E9002307B030BD00BF00FD002412
:10D7A0002DE9F041DFF83C8086B005460E4604A81E
:10D7B000D8F800101746FFF741F9D8F80020DDE946
:10D7C0000443926BA41A02A863EBE2732A19CDE911
:10D7D000006743F10003FFF7C3FF0298001B06B088
:10D7E000BDE8F08100FD002410B5054C236813B995
:10D7F000FEF7F8FA20602068BDE81040FEF780BD13
:10D8000004FD002413B5074C01212046FFF73AFC24
:10D81000034628B90090044922880448FFF7B2FE65
:10D8200002B010BD18FD0024879106082301048072
:10D8300013B5094C01212046FFF72DFC4FF6FF736D
:10D84000984206D100230549054800932288FFF736
:10D8500099FE02B010BD00BF18FD0024A991060872
:10D8600024010480034B188880B2B0FA80F040098C
:10D87000704700BF18FD0024F8B5FFF7DBFCFFF789
:10D88000B3FF07460E46FFF7EDFF0546A8B10FF0C0
:10D8900093FCFFF7A9FF04460A468DB10E49D1E972
:10D8A0000035DB1B65EB06051B1942EB0505C1E9DD
:10D8B0000035BDE8F840FFF7D3BC0FF06BFCE8E79C
:10D8C0000649D1E90030DB1B60EB06001B1942EB77
:10D8D0000002C1E90032ECE708FD002410FD00243D
:10D8E0006FF01C0070476FF0150070470120704703
:10D8F0000020704770470000034B186818B14FF0C4
:10D90000FF31F8F737BC704764490024024B1868B0
:10D9100008B1F8F747BC704764490024F8B51546CC
:10D920000C468E18054FB44201D12846F8BD14F8B4
:10D93000011B38460BF014FDF5E700BF9C160124CF
:10D9400038B511F001040D4605D008480FF034F940
:10D95000041E18BF0124EB0605D504480FF03CF95E
:10D9600008B144F01004204638BD00BF9C160124C5
:10D9700010B510460C4622B102480BF0BBFC2070DB
:10D98000012010BD9C16012438B5084B04461546ED
:10D990000360074B1B6833B90648FEF71DFD294697
:10D9A00004480FF071F9204638BD00BFF092060818
:10D9B000C01601249C1601240020704700207047E7
:10D9C000002307B51A46024902480093FFF7DAFD23
:10D9D000C791060829010180074A084913681844BD
:10D9E000884283BF064B0C224FF0FF3010608CBF83
:10D9F0001A601846704700BF800D002400FC072401
:10DA00006C1701240120704701207047002114F099
:10DA10007DBA08B5F9F7AEFB08BD08B5F9F7B2FB5A
:10DA200008BD000010B50446037803F00303012B82
:10DA300008D0FFF761FF237803F00302012A03D126
:10DA4000FFF764FF002010BD2AB14FF4D4620449EF
:10DA50000448FFF703FB43F0020323700120F2E7C1
:10DA6000EB910608FD91060808B5037803F0030260
:10DA7000022A05D040F2A96206490748FFF7EEFAEC
:10DA800023F0030343F001030370BDE80840FFF7F0
:10DA90003DBF00BFEB9106081B9206083F2870B5FA
:10DAA00004462CDC174E56F820305A1C25D102288B
:10DAB00023DCFFF783FF0346E8B92046FFF77CFF2E
:10DAC0000346C0B9104D2B68BFF35B8FDB0711D441
:10DAD0002846FFF7A7FF68B14FF4E1320B490C4825
:10DAE000FFF752FF0B4A0C490948FFF78BFF284606
:10DAF000FFF7BAFF064B46F82430184670BD0023E6
:10DB0000FBE700BF840D00241CFD002438930608A9
:10DB100020FD002400000024F5D8040838B5044690
:10DB20000025FFF7BBFF0B4B43F8245030B912F030
:10DB3000EFFB092303604FF0FF3038BD03685B69DA
:10DB40009847041E04DA644212F0E2FB0460F2E734
:10DB50002846F2E7840D0024FFF7E0BF38B50C46F5
:10DB60001546FFF79BFF38B912F0D2FB092303607B
:10DB70004FF0FF34204638BD036821462A46DB6853
:10DB80009847041EF6DA644212F0C2FB0460EFE725
:10DB900038B50C461546FFF781FF38B912F0B8FBCF
:10DBA000092303604FF0FF34204638BD0368214647
:10DBB0002A469B689847041EF6DA644212F0A8FBD6
:10DBC0000460EFE710B5FFF769FF30B912F0A0FB72
:10DBD000092303600024204610BD0368DB699847D1
:10DBE000041EF8DA644212F093FB0460F2E740236B
:10DBF00037B50546CDF8010068468DF8003012F0C3
:10DC000017FE044630B12846FFF7DCFF10B120466E
:10DC1000FFF7FCFE204603B030BD00002DE9F74FB2
:10DC200006460F469046FFF7FCFA054630B1002342
:10DC300032462C492C480093FFF7A4FCFFF7EBFA7F
:10DC40000028F4D0B8F1000F09DA12F061FB1623B6
:10DC500003604FF0FF34204603B0BDE8F08F30463C
:10DC6000FFF7B0FF044640B1DFF880A02C464FF02C
:10DC70000D0B1AF80690A84512DCA045EBDDA8EBC9
:10DC8000040239193046FFF769FF0028E1DB04443C
:10DC9000002CC1BF3F19154B17F8012C9A55DAE734
:10DCA0007A5D0A2A1AD1B9F10D0F17D0AC420BDAFE
:10DCB0002A1B39193046FFF751FF0028C9DB0444FD
:10DCC000A542C8DC0AF80690012209493046FFF750
:10DCD00045FF0028BDDBBED00AF806B017F8059056
:10DCE0000135C8E7529206082F01018024FD002467
:10DCF0008C920608FFF766BF7FB504460D461646B0
:10DD0000FFF78FFA30B1002322461F491F480093C6
:10DD1000FFF738FCFFF77FFA0028F4D0002E07DA6F
:10DD200012F0F6FA162303604FF0FF3004B070BD16
:10DD30002046FFF747FFF8B1154E01220DF10F0104
:10DD40002046FFF725FF0028EEDBEFD09DF80F30CF
:10DD50000D2B08D1325D0A2A0AD01A460A23012067
:10DD600032552B70E2E70A2B04D1325D0D2AF3E71E
:10DD70003355E2E71A46F2E732462946204604B018
:10DD8000BDE87040FFF704BF8E9206082F010180A6
:10DD900064FD002438B50C461546FFF77FFE38B900
:10DDA00012F0B6FA092303604FF0FF34204638BD65
:10DDB000036821462A461B699847041EF6DA644226
:10DDC00012F0A6FA0460EFE7FFF7E4BF10B5FFF723
:10DDD00065FE30B912F09CFA092303604FF0FF3062
:10DDE00010BD03689B699847041E04DA644212F070
:10DDF0008FFA0460F2E70020F2E700000A4D0446C3
:10DE000008B52B68986812F0D1FB2B68D86812F01F
:10DE1000CDFB0120FFF7DAFF0220FFF7D7FF0CB19F
:10DE2000FFF776F9FEE700BFA40E002408B5FFF760
:10DE3000E5FF38B50D46FFF731FE044630B912F064
:10DE400067FA092303604FF0FF3038BD0368DB69D0
:10DE50009847002820460CBF4FF400434FF400536E
:10DE60006B6023689B6A984728610020EDE7FFF705
:10DE7000E0BF000008B5037803F00302022A05D0D2
:10DE800040F2B26205490648FFF7E8F823F00203C2
:10DE90000370BDE80840FFF739BD00BFEB910608ED
:10DEA0001B920608084B724613B5014604461868D3
:10DEB000FFF734F8034628B9009022460349044886
:10DEC000FFF760FB02B010BDA40E0024CA92060842
:10DED0001F010180FFF7E6BF044B72460146186838
:10DEE00000B55DF804EBFFF719B800BFA40E0024DD
:10DEF000FFF7F2BF044B72460146186800B55DF8A3
:10DF000004EBFFF75FB800BFA40E0024044B724679
:10DF10000146186800B55DF804EBFFF753B800BF81
:10DF2000A40E002410B504460421FFF7EFFF20469D
:10DF300010BDFFF7DFBF000010B504460B48FAF72D
:10DF400085FC00F0C7F90A4A4023002152F8040B6F
:10DF5000A04208BF42F8041C013BF7D10348FAF77E
:10DF600075FCBDE8104000F0D1B900BFA4FD00244D
:10DF7000840D002410B512480324FAF767FC00F062
:10DF8000A9F9104B53F8242072B10134402CF9D177
:10DF900012F0BEF918234FF0FF3403600848FAF777
:10DFA00055FC00F0B3F908E04FF0FF32044843F8A5
:10DFB0002420FAF74BFC00F0A9F9204610BD00BF61
:10DFC000A4FD0024840D002410B50446FFF7D2FF01
:10DFD000002807DB044B054A43F820400023135474
:10DFE000034A135410BD00BF840D002464FD0024B7
:10DFF00024FD002470B505460E46FFF7E5FF041E1C
:10E0000001DA002070BD3146FFF7F1FD0028F9D19B
:10E01000064B53F82420954202D143F82400F0E740
:10E0200012F076F909230360EBE700BF840D0024AA
:10E030000EB42DE9F04185B00546FFF79BFF041EA5
:10E0400013DB0023294602A8214E0193FEF7C6FBED
:10E0500002A8FEF711FC054668B912F059F913231E
:10E06000036046F824504FF0FF34204605B0BDE869
:10E07000F04103B0704702A8FEF7ECFB074602A888
:10E080005FB1FEF7F0FB0190019B124A46F8243085
:10E0900000231355104A1355E7E7FEF7D2FB054658
:10E0A0000028DAD0036802A8D3F80880FEF7BEFB88
:10E0B0000B9B024601A92846C04705460028E3D02D
:10E0C0006D4212F025F9056046F82470CBE700BFD9
:10E0D000840D002464FD002424FD002470B50E4648
:10E0E0001549054614F030F9044618B9FFF7D6FC77
:10E0F000204670BD1149284614F026F920B90120A8
:10E100000124FFF7CBFCF3E70D49284614F01CF976
:10E1100020B902200224FFF7C1FCE9E72B78402B4D
:10E1200002D1D5F80140E3E726F480312846BDE866
:10E130007040FFF77DBF00BF609306085893060844
:10E140005093060810B5044620B990221049114892
:10E15000FEF784FF4C220021043013F071FD4FF2D2
:10E1600004134FF000614FF0105223604FF400236E
:10E1700021634FF4001123626362074B2261216423
:10E1800062611B68636002232372044BE36010BD6D
:10E19000819306088E93060800ED00E098FC0100CC
:10E1A000034A516A536A5B1A8342FBD3704700BF2C
:10E1B000000C00401FB500230446CDE90013031DE9
:10E1C0006846029310230393F6F7C4FF206020B93A
:10E1D000352203490348FEF741FF04B010BD00BFDC
:10E1E000B2930608C193060810B504460249FFF72A
:10E1F000E1FF204610BD00BFC593060810B50446D8
:10E20000FFF7D8FF204610BD0068F6F7BBBF10B57A
:10E2100004460068F7F72CF8204610BD10B49DF8AE
:10E2200004400CB942F0020200685DF8044BF6F7B6
:10E23000F1BF07B5009313460022FFF7EFFF03B0CD
:10E240005DF804FBFFF7F5BF38B5FEF7F3FFF7F70E
:10E2500057FA084904460B6808608342064B82BFA0
:10E260001A6801321A601D68FEF7FAFF2046294637
:10E2700038BD00BFD4FD0024D8FD00241FB5002305
:10E28000044603620C4B002918BF0B460093031D84
:10E29000684602931C2303930B230193F7F752FF65
:10E2A000206038B9FFF760F920B93D2203490448DE
:10E2B000FEF7D4FE04B010BDE593060815940608D9
:10E2C0001F94060810B504460021FFF7D7FF20462B
:10E2D00010BD000037B504464FF0FF310068F7F776
:10E2E00049FF054648B1FFF73FF9034640B90090A2
:10E2F0002A4604490448FFF745F9236A013323629B
:10E3000003B030BD4394060815010280036A013B47
:10E3100013B503620068F7F745FF044648B1FFF7FD
:10E3200023F9034628B90090224603490348FFF722
:10E3300029F902B010BD00BF5594060817010280EC
:10E3400010B504460068F7F745FF204610BD0000F1
:10E350001FB50446002310466A46CDE90033231D4D
:10E36000029310230393F8F759F8206020B937225D
:10E3700002490348FEF772FE04B010BD7F94060800
:10E380008D94060810B504464FF6FF72FFF7E0FFC4
:10E39000204610BD13B500680C46F8F757F8024642
:10E3A00070B1C11C4FF0000006D15CB10090002399
:10E3B00005490648FFF7E6F8931CF7D102B010BDF7
:10E3C0000120FBE72046F9E79C940608140102802F
:10E3D0000068F8F763B810B504460068F8F78CF8E1
:10E3E000204610BD08B538B1F6F74EFD20B1E32246
:10E3F00002490348FEF732FE08BD00BFCB94060871
:10E40000E2880608F8F76EBD884209D038B50446A0
:10E410000D46F3F791FA29462046F5F7C1FE38BDBF
:10E42000704700002DE9F047DDE90857994604469A
:10E430006B07884692464FF0000118BF25F007068B
:10E440004FF0440200F178000CBF2E46083613F05E
:10E45000F7FBB5FA85F300214D4420225B0904F156
:10E460001C006161AD1B84F83C3084F83D1025F040
:10E47000070513F0E5FB064BC4F830A0002F08BFDA
:10E480001F46E562A662A761C4F83480BDE8F08744
:10E490005F95060813B5049CCDE9003413460A467F
:10E4A0000021FFF7BFFF02B010BD000070B500F102
:10E4B000540504460E462846FFF70CFF636913B95E
:10E4C00094F83D302BB12846FFF720FF6FF0030092
:10E4D00070BDD4E90A304BB300232349E26AB3EBA1
:10E4E000920F36D344233146201D636204F1780332
:10E4F0002362FFF789FF04F1180221461B48F8F751
:10E50000C5FC606150BB94F83C302BB1A06A08B1E7
:10E51000FFF70FFD0023A3622846FFF7F7FE04F183
:10E520004000FFF755FF6FF00200D1E7104B114993
:10E53000984294BF20F003004FF0FF30FFF7D8FC63
:10E54000A0620028C8D12846FFF7E0FE6FF0040063
:10E55000BEE7A26A42F823100133BFE72846FFF75F
:10E56000D5FE0020B4E700BFA52E5AE2B5E60408A8
:10E57000FBFFFF7FDCC7060870B500F154050446B9
:10E580002846FFF7A7FE04F140006669FFF720FF69
:10E590000023636194F83D302BB100242846FFF737
:10E5A000B5FE204670BD012384F83D30002EF4D026
:10E5B0003046F8F7ADFC0446F0E738B500F15405F5
:10E5C00004462846FFF786FE6369A3B194F87940B4
:10E5D0002846FFF79BFE432C27D015D8132C26D0B6
:10E5E0000BD8012C05D0022C03D0003C18BF01240D
:10E5F0002401204638BD0424EAE7232C19D0332C0B
:10E6000014BF10240524F4E7732C14D006D8532C1F
:10E6100013D0632C14BF10240824EAE7832C0ED0F7
:10E62000932C14BF10240B24E3E70624E1E7032412
:10E63000DFE70424DDE70924DBE70724D9E70A2420
:10E64000D7E738B500F1540504462846FFF742FEE7
:10E65000646914B1A26B246B141B2846FFF756FEA5
:10E66000204638BD0D4B10B504460360FFF784FF0C
:10E6700094F83C302BB1A06A08B1FFF75AFC002394
:10E68000A36204F15400FFF75BFE04F14000FFF7C2
:10E69000A2FE201DF3F755F9204610BD849506080B
:10E6A00010B50446FFF7DEFFBC212046FFF72EFC25
:10E6B000204610BD10B504460430F8F713FF04F1EE
:10E6C0005400FFF707FE002304F1400063610123BB
:10E6D00084F83D30BDE81040FFF77ABE01200021EC
:10E6E0007047D0F860010021704700000048704773
:10E6F0008C950608D0E944017047FF207047000060
:10E700002DE9F04F89B01546984606469DF84830E9
:10E71000AB469DF8502090F8FA91DDE9157105910E
:10E72000032B21D8DFE803F01D2A02044FF0030970
:10E730000F2A06F1040A4B4608BF96F8FD21504601
:10E740000392002211460092CDE90122FAF7CEFC95
:10E750000446B0B10220284A2849FDF767FF204649
:10E7600009E04FF0FF3BE3E70220254A2349FDF78C
:10E770005DFF4FF0FF3009B0BDE8F08F4FF00209A8
:10E78000D6E7059B4FF0FF329DF84C10504607939B
:10E7900007ABCDE900735B46FAF733FD224621460D
:10E7A00083464B465046CDE90244CDE90044FAF792
:10E7B0009DFC04460028CDD1BBF1000F06D00220FD
:10E7C000104A0E49FDF732FF5846D4E796F801315A
:10E7D00063B12B1F53EA080304D13B7843F00A03CB
:10E7E0003B7003E0023D55EA080501D00020C2E776
:10E7F0003B7823F00403F3E7BC9506088C950608E4
:10E8000092950608DA95060838B505461946104669
:10E81000D5F81831013326D105F5847201F01AFDBF
:10E82000431CD5F8604102D12046C11738BD2844A9
:10E8300090F85431D8070AD5002300E00123723341
:10E8400055F82300F1E70223F9E70323F7E79907D7
:10E85000F4D45A07F7D41B07F7D4054A0220054918
:10E86000FDF7E4FEE0E74FF480500021DEE700BF53
:10E87000F89506088C9506080068704730B5039D2A
:10E8800000241C702C708C7814F0200F15D04A7A5C
:10E89000C0F8E02001221A700B7A03F01F0380F801
:10E8A000FD310B7A5B099B0080F8FB31022380F875
:10E8B000F93180F8FE31002030BD102A0FDD0A7CCE
:10E8C000D2060CD5CA7EC0F8E02001221A702A7048
:10E8D0008B7E03F01F0380F8FD318B7EE2E762063A
:10E8E0000FD5CA7AC0F8E02001221A708B7A03F0A3
:10E8F0001F0380F8FD318B7A5B0980F8FB3102231E
:10E90000D7E70B7CDD070ED5CB7DC0F8E0308B7DE3
:10E9100003F01F0380F8FD318B7D5B095B0080F8FD
:10E92000FB310123C3E7E20609D5CB7BC0F8E03019
:10E930008B7B03F01F0380F8FD318B7BEDE7E30752
:10E940000DD54B7BC0F8E0300B7B03F01F0380F844
:10E95000FD310B7B5B0980F8FB310123A9E7032321
:10E96000C0F8E030A7E700002DE9F04385B0064687
:10E970000D461746DDF83880DDF8489000F0C0F805
:10E98000044640B10E4A02200E49FDF74FFE2046D4
:10E9900005B0BDE8F083109B3A462946301DCDF8FE
:10E9A0000890CDE900830C9BFAF78FFC0446002801
:10E9B000EDD02B46044A03490220FDF737FEE6E777
:10E9C000209606088C950608739606082DE9F047F0
:10E9D00000238AB0054642F21074012600274FF04A
:10E9E00000084FF00009DFF864A08DF827300120FF
:10E9F000FFF7F8FC0DF127034FF0FF3205210493D8
:10EA00000023284600934FF0FF33CDE90667CDE998
:10EA10000289FFF7A9FF20B152460A490220FDF7FB
:10EA200005FE9DF82730DA0708D5013CDFD102202A
:10EA3000054A0449FDF7FAFD204600E001200AB02E
:10EA4000BDE8F0878C950608AE9606088F960608F6
:10EA5000F0B500258BB004468DF82750FFF7B6FFC0
:10EA600040B9214A21490220FDF7E0FD4FF0FF3077
:10EA70000BB0F0BD0026002704954FF0FF32009543
:10EA80004FF0FF3306212046CDE90667CDE9026746
:10EA9000FFF76AFF054608B1154AE3E72046FFF78E
:10EAA00095FF08B9134ADDE701220023052120461E
:10EAB0000095CDE906230DF127034FF0FF320493B3
:10EAC0004FF0FF33CDE90267FFF74EFF08B10A4A66
:10EAD000C8E79DF827309A07CAD4084A022003499C
:10EAE000FDF7A4FDC2E700BFD89606088C9506087E
:10EAF000029706081E9706083D9706085E970608C7
:10EB000030B5D0F8F44087B0054601341CD0120E61
:10EB10008DF81720FFF79CFF70B901234FF0FF32EB
:10EB2000CDE901000093281D0DF11703D5F8F4106D
:10EB3000FAF7CBFB07B030BD0C4A02200C49FDF7B9
:10EB400075FD4FF0FF30F5E790F8FA1103290BD06F
:10EB500012F17F426FF0807143F1FF338A4273F10B
:10EB6000FF3301D2034AE8E70020E3E79597060860
:10EB70008C950608A99706082DE9F04387B09046C2
:10EB800005460E46109BDDF8389005934A460F9BCC
:10EB9000FFF7B6FF044640B1224A23490220FDF7A1
:10EBA00045FD204607B0BDE8F08395F8FD312F1DE7
:10EBB00095F8F9210393384695F8FE31029395F8BC
:10EBC000FB31CDE9002395F8FA3195F8F811FAF701
:10EBD0008DFA044608B1154ADFE795F8FB0105AB4D
:10EBE0003146B0FA80F04009CDE9008342424B46FD
:10EBF0003846FAF706FB2246214606463846CDE956
:10EC00000244CDE9004495F8FA31FAF76FFA044668
:10EC10000028E0D126B1064A02200349FDF706FD8F
:10EC20003446BEE7F09706088C950608BC950608A2
:10EC3000389806082DE9FF4100F1BC0804460D464E
:10EC4000174640461E46FFF745FB2046DDE90A23EE
:10EC5000CDE90076CDE902232A46D4F8E010FFF78B
:10EC60008BFF044630B16FF47A64064A06490220ED
:10EC7000FDF7DCFC4046FFF749FB204604B0BDE849
:10EC8000F08100BF499806088C9506082DE9F341EC
:10EC9000DDF820801746099B054642460E46FFF7E1
:10ECA0002FFF044640B10C4A0C490220FDF7BEFC80
:10ECB000204602B0BDE8F0810A9B4FF0FF3231469A
:10ECC000281DCDE900734346FAF7CDFA0446002823
:10ECD000EED0034AE8E700BF5D9806088C95060869
:10ECE000A6980608F0B585B005460E461746FFF70C
:10ECF00007FF044638B10B4A0B490220FDF796FC8A
:10ED0000204605B0F0BD034600903A463146CDE9B5
:10ED10000100281DFAF7D9FA04460028F0D0034A6A
:10ED2000EAE700BFB89806088C950608019906081E
:10ED30002DE9F04F87B00646884614461F4600F17D
:10ED4000BC0ADDE9105955EA090304D10024204624
:10ED500007B0BDE8F08FD6F8F0B100232046394661
:10ED60005A4610F017F8A918504649EB03035945C5
:10ED700073F100034FF000032CBFABEB020BAB466B
:10ED80000593CDF810B0FFF7A5FA3046FFF760FE07
:10ED900048B11D4C02201D4A1D49FDF747FC504655
:10EDA000FFF7B4FAD3E704AB4246022130460293A0
:10EDB000CDE90047FFF76AFF38B1164A022014492F
:10EDC0006FF47A64FDF732FCE9E7DDE90423984249
:10EDD00008BF9345F1D11BEB0404D844304647F1FA
:10EDE0000007B5EB0B0B69F100095D46FFF7EEFD7F
:10EDF00030B9094A02200649084CFDF717FCCEE756
:10EE00005046FFF783FA9EE75CF0FFFF1399060870
:10EE10008C950608AB980608269906085DF0FFFF5A
:10EE20002DE9F04F144689B0054600F58472194665
:10EE300020461E46DDE9127901F00CFA2B1814EB7E
:10EE40000708824693F8543146EB090B0793D5E93E
:10EE50004423424573EB0B0309D25B4A5B4C02200F
:10EE60005B49FDF7E3FB204609B0BDE8F08F2B6856
:10EE700022462846196B3346884702460B462046F1
:10EE800031460FF087FF1A4310D118F1FF322B687B
:10EE90002846196B6BF10003884702460B46404633
:10EEA00059460FF077FF1A4300F08B80494AD5E7A7
:10EEB000D5F81831059301333ED105F590733A46E4
:10EEC0000798CDE902A3CDE900464B4601F0E0F9F1
:10EED000834605EB8003D3F8B821D3F8C8810592A7
:10EEE00042460023204631460FF054FF1A4306D114
:10EEF000E21946EB0903424573F1000308D2364A92
:10EF000002203349CDE9028BCDE90046FDF78EFBA7
:10EF100005F1BC0318460693FFF7DCF92846FFF716
:10EF200097FD60B12D4C02202D4A2949FDF77EFB4B
:10EF30000698FFF7EBF996E74FF48058D0E72246A2
:10EF4000334605992846CDE90079FFF7CBFE38B165
:10EF5000244A02201E496FF47A64FDF767FBE7E755
:10EF600018EB040446F10006B7EB080869F1000944
:10EF7000474658EA090310D00AF12D0355F833200B
:10EF800005EBC301A2424B68B3413FBF0AF1010A3E
:10EF900005EB0A0393F8543107932846FFF716FD53
:10EFA00030B9114A02200A49104CFDF73FFBBFE778
:10EFB0000698FFF7ABF957EA09037FF479AF00240D
:10EFC00051E74FF0000BF6E74B9906085BF0FFFFA7
:10EFD0008C9506086B990608969906085CF0FFFF69
:10EFE000DA990608FF9906081A9A06085DF0FFFFED
:10EFF00030B591F839308BB091F8382004461B01B8
:10F0000003F0100343EA1213082B6ED01DD8022B15
:10F0100005D8002B50D14E4A04204E4960E0042B05
:10F02000F9D10023002400254FF0FF32049335214D
:10F0300000934FF0FF33CDE90645CDE90245FFF7D8
:10F0400093FC00284ED0444A48E0102BE3D1012223
:10F05000002309AD6521CDE9062300220023049594
:10F06000CDE9022300234FF0FF3200934FF0FF332E
:10F07000FFF77AFC20B1394A02203649FDF7D6FA6B
:10F080009DF8243001226121204603F07F0304957E
:10F090008DF824300023CDE9062300220023CDE99A
:10F0A000022300234FF0FF3200934FF0FF33FFF7AE
:10F0B0005BFCB8B12A4A11E00023002400254FF080
:10F0C000FF320493382100934FF0FF33CDE906451A
:10F0D000CDE90245FFF748FC20B1224A1D49022034
:10F0E000FDF7A4FA00200BB030BD0122002309ADCA
:10F0F0006521CDE90623002200230495CDE90223F2
:10F100000023194A00930023FFF72EFC20B1174A71
:10F1100002201049FDF78AFA9DF82430012271215E
:10F12000204643F0400304958DF824300023CDE9B8
:10F13000062300220023CDE9022300230A4A00937C
:10F140000023FFF711FC0028CCD0094AC6E700BF16
:10F15000709B06088C950608759A0608119B060890
:10F16000419B0608459A060803008000A59A0608F8
:10F17000E19A0608D0B503268AB00027002309AA21
:10F180009F21ADF8243004468DF8263004924FF0CC
:10F19000FF3200934FF0FF33CDE9066700260027CA
:10F1A000CDE90267FFF7E0FB40B10220224A234984
:10F1B000FDF73CFA4FF0FF300AB0D0BD9DF8243087
:10F1C0009D2B1ED005D8012B1FD01F2B28D000202F
:10F1D000F2E7BF2B12D0C22BF9D19DF82530202B9E
:10F1E0001FBF012384F800310323C4F8E430152342
:10F1F000C4F8EC30002384F8F030E8E784F8030129
:10F20000E5E70123C4F8E430E1E79DF82520022A70
:10F21000DDD19DF82620202AD9D184F80131D6E706
:10F220009DF82530892BD2D13123C4F8E830012351
:10F2300084F80231CBE700BFAD9B06088C95060829
:10F240003F2A2DE9F04F05468BB040F3B78091F887
:10F250003F3013F0400204D00323002485F8FA3134
:10F260006DE0D90712D50026002704924FF0FF3336
:10F270000092B7214FF0FF32CDE90667CDE9026772
:10F28000FFF772FB0028E7D04D4C58E013F0020264
:10F2900012D0FFF7DDFB00284BD1002200230490A1
:10F2A000B72100902846CDE90623CDE902234FF08F
:10F2B000FF324FF0FF33E3E713F0100158D04FF067
:10F2C00001084FF000090DF127064FF0000A4FF03A
:10F2D000000B8DF8272000924FF0FF334FF0FF32E4
:10F2E000B5210496CDE90689CDE902ABFFF73CFBD9
:10F2F0000028C9D19DF82730284643F001038DF836
:10F300002730FFF7A5FB044698B904904FF0FF3271
:10F310004FF0FF33B12128460096CDE906ABCDE989
:10F320000289FFF721FB0028AED1032385F8FA31CB
:10F3300005E0244C0220244A2449FDF777F995F88A
:10F34000FA31032B10D10022281D1146CDE90222EB
:10F35000CDE90022F9F7CAFE30B16FF47A641C4A95
:10F360001A490220FDF762F920460BB0BDE8F08F84
:10F370001A071AD580230022049117218DF827300F
:10F380000023CDE9062301220023CDE902230DF15C
:10F3900027034FF0FF3200934FF0FF33FFF7E4FAFB
:10F3A000044600287FF470AFBFE713F0040F4FF05E
:10F3B00002031CBFC522C0F8F4204EE70024D3E7A7
:10F3C0005EF0FFFF5CF0FFFF959706088C9506083E
:10F3D000BC950608D0B5044690F8020188B0F0B19B
:10F3E00091F8343013F008021CD0002100284FF0AF
:10F3F00000034FF000004FF0FF32049300934FF0F2
:10F40000FF33CDE90601CDE9020114BF9921F021B6
:10F410002046FFF7A9FA58B31C4808B0D0BD91F8B0
:10F420003D30DFE7DB061DD50026002704924FF0B4
:10F43000FF33009266214FF0FF322046CDE9066788
:10F44000CDE90267FFF790FA0028E5D14FF0FF32CF
:10F450004FF0FF33992104900090CDE90667CDE984
:10F460000267D5E70A4A02200A49FDF7DFF8D3E729
:10F470002046FFF7ABFA30B90220074A0549FDF7ED
:10F48000D5F80648C9E70020C7E700BF5EF0FFFFD8
:10F49000C39B06088C9506084A9C06085DF0FFFF92
:10F4A0002DE97043012288B000234FF000084FF08F
:10F4B000000904910D4605210646CDE906230023E7
:10F4C0004FF0FF3200934FF0FF33CDE90289FFF791
:10F4D0004BFA044640B1114A11490220FDF7A6F843
:10F4E000204608B0BDE87083D6F8E430013BF7D081
:10F4F000013500904FF0FF320495CDE90630CDE99B
:10F5000002894FF0FF33D6F8EC103046FFF72CFAA3
:10F5100004460028E4D0034ADEE700BF3D97060812
:10F520008C950608699C0608D0F8E83001332DE96F
:10F53000F04F054689B00E4628D1FFF789FA50B141
:10F540004FF0FF34334A34490220FDF76FF820466C
:10F5500009B0BDE8F08F0022002304900121CDE91D
:10F560000623D5F8E4304FF0FF320096CDE90230A3
:10F570004FF0FF332846FFF7F7F904460028E6D09E
:10F58000264A02202449FDF751F8E0E7D0F8E4705C
:10F59000022F05D040F25F6221492248FDF75EFD4F
:10F5A000FFF756FA0028CBD14FF0000A4FF0000BBE
:10F5B0004FF001084FF0000904904FF0FF324FF078
:10F5C000FF33012128460096CDE906ABCDE902893B
:10F5D000FFF7CAF9044618B1134A0F493846D2E773
:10F5E0002846FFF735FA0028AAD1013604944FF0D7
:10F5F000FF324FF0FF3300962846CDE906ABCDE948
:10F600000289D5F8E810FFF7AFF9044600289ED02C
:10F61000064AE2E78A9C06088C9506089E9C060826
:10F62000F39C0608089D0608239D0608449D0608CD
:10F63000002373B5ADF8003004468DF80230ADF804
:10F6400004308DF8063090F8023153B991F83A3011
:10F65000C3F30213052B4BD8DFE803F04F033C4103
:10F6600003030123C4F8F830C4F8FC30D4F8F830B0
:10F67000591C09D0D4F8FC104A1C05D008330122CB
:10F680006B448A4003F8082C01A92046FFF708FFC5
:10F690009DF806309DF802202046BDF80010134367
:10F6A000BDF804209DF800500A4301A99DF80160AF
:10F6B000ADF804208DF80630FFF736FF2046FFF73F
:10F6C00085F9E8B9184A02201849FCF7AFFF4FF056
:10F6D000FF3013E00023C0F8F8300623C4E7072307
:10F6E00000203E25C4E93E033F23C4E93A53BDE769
:10F6F0000F4A04200D49FCF799FF002002B070BDAD
:10F70000002301A92046ADF804308DF80630FFF73C
:10F71000C7FE9DF804301D409DF805301E4035435E
:10F72000EBD1044ACFE700BF269906088C9506085E
:10F73000659D0608839D060830B500238BB00546FD
:10F74000ADF824308DF82630FFF740F940B9274A4C
:10F7500002202749FCF76AFF4FF0FF300BB030BDA5
:10F7600095F8034144B1012C20D02846FFF72EF92B
:10F770000028ECD00020F1E72846FFF769F908B12E
:10F780001C4AE5E7002200230490982100902846B7
:10F79000CDE90623CDE902234FF0FF324FF0FF33CE
:10F7A000FFF7E2F80028E0D0134AD1E709A928467C
:10F7B000FFF776FE08B1114ACAE7D5F8F83093B9D9
:10F7C000D5F8FC309C4044F00304E4B29DF82430AA
:10F7D00009A928461C408DF82440FFF7A5FE002803
:10F7E000C3D0074AB4E70324F0E700BFA59D06088D
:10F7F0008C95060895970608D89D0608FE9D060874
:10F80000349E0608D0F8E430032B70B5044686B069
:10F8100005D040F2035225492548FDF71FFC002280
:10F82000022304301146ADF814208DF81620CDE9DE
:10F830000222CDE90022F9F759FC48B11D4A4FF0E8
:10F84000FF351D490220FCF7F1FE284606B070BDC9
:10F8500005A92046FFF724FE08B1184AEFE79DF8F6
:10F860001630204643F002038DF81630FFF7F0F80B
:10F87000054608B1124AE2E705A92046FFF754FE03
:10F88000064608B10F4ADAE72046FFF79FF808B9A5
:10F890000D4AD4E705A92046ADF814608DF816602E
:10F8A000FFF7FEFD0028D0D0084AC8E7F39C060801
:10F8B0006C9E0608BC9506088C950608879E06086F
:10F8C0008A9C0608A69E060826990608D89E060861
:10F8D00010B50446F2F730F8204610BDF8B51848C8
:10F8E0000C46184DF8F7B2FFFEF7F4FC2A68092A17
:10F8F00020DC154B1B68991E184603F1120631F9DE
:10F90000027FA74219D0B142F9D114330146023027
:10F91000B1F9006001360AD10C80013200242A605E
:10F920000748F8F793FFFEF7F1FC2046F8BD984230
:10F93000ECD1F2E76FF00104F2E74FF0FF34EFE7AC
:10F94000E4FD0024E0FD0024DCFD00247FB52F4E03
:10F950000446BDF9285040F8046B0B9ECDE90256D1
:10F96000BDF924600196BDF920600096F9F778FB97
:10F9700004F1BC00A4F8B850FEF7A4FC0C9B294687
:10F980002046C4F8F4310023C4F8003284F804326D
:10F99000FFF7A4FFC4F8B40050B101301C494FF088
:10F9A000020007BF2B461B4A0A231B4AFCF73EFEF8
:10F9B0000020002100224FF0FF33C4E944014FF43E
:10F9C0000030C4F8602184F854210121C4F8F80102
:10F9D000032084F8FD2184F8FE210222C4F81831A6
:10F9E000C4F8E830C4F8FC30C4F8281184F8F010EA
:10F9F000C4E93802C4E93D3335224FF08073204614
:10FA0000C4F8EC20C4F8003104B070BDA4A106080D
:10FA10008C950608F99E0608309F060810B5134815
:10FA20000C46F8F713FFFEF755FC114B1B6803F16A
:10FA300014011A460233B2F90000A0420AD14FF66F
:10FA4000FF7313800B4A1368002B01DD013B136029
:10FA5000002403E08B42ECD14FF0FF340348F8F769
:10FA6000F5FEFEF753FC204610BD00BFE4FD002468
:10FA7000DCFD0024E0FD002470B500F1BC06044666
:10FA800088B03046FEF726FC94F8043243B9C4F837
:10FA9000003200253046FEF739FC284608B070BD1C
:10FAA000D4F80032013BC4F80032002BF1D1002021
:10FAB000002104934FF0FF3200934FF0FF33CDE964
:10FAC0000601CDE9020104212046FEF74DFF05465F
:10FAD00030B16FF47A650A4A0A490220FCF7A6FDA4
:10FAE0000023304684F80432FEF710FCD4F8B4301A
:10FAF000002BD2D1B4F9B8102046FFF78FFFCCE726
:10FB00006E9F06088C9506082DE9F04387B01D7896
:10FB100009680E9B1E780F9B1F78109BD3F800C0BE
:10FB2000D0E9004313F0010F01EB63001EBF4FEA61
:10FB3000630E51F80E301C59119BD3E90089CDE9B1
:10FB4000027CCDE90489CDE90056D2E90023A04723
:10FB500007B0BDE8F0837FB5CDE904230CAB0146C7
:10FB600004AA043003930BAB02930AAB019309ABD5
:10FB7000009308ABFFF7C8FF07B05DF804FB000077
:10FB8000034A0346C26007C983E80700704700BF05
:10FB9000F0A1060870B586B00E46002104466D46F9
:10FBA00085E80C00102212F04BF806AB039695E89E
:10FBB000030003E90300204603A9FFF7E1FF204605
:10FBC00006B070BD37B56C46054684E80C0094E875
:10FBD0000C00FFF7DFFF284603B030BD08B5F7F78C
:10FBE0006DFC0068003818BF012008BD2DE9F04702
:10FBF000044616461D469DF820709DF824809DF809
:10FC00002890FFF7EBFF28B940F202220849094883
:10FC1000FDF724FAE0683246FEF72EFE2B46014639
:10FC200008972046CDE90989BDE8F047084700BF9D
:10FC3000A47F06082D7A060830B587B00D99039188
:10FC40009DF8301002919DF82C10DDE90E450191D0
:10FC50009DF82810CDE904450091FFF7C7FF07B0D4
:10FC600030BD000090F802312DE9F04315469DB0FB
:10FC700004460E461268002B37D0242008AB002122
:10FC80004FF05A084FF0080901270393002300970B
:10FC9000CDE90401CDE901893046FFF7CDFF50B130
:10FCA000404A4FF0FF3640490220FCF7BFFC304687
:10FCB0001DB0BDE8F0830C220023CDE9042314AB72
:10FCC0006022CDE902930023CDE900783046FFF7AA
:10FCD000B3FF0028E4D104F5847708A8394600F082
:10FCE0002FFB00280DDA314ADBE769680820CDE9EF
:10FCF000041308A903915A21CDE9011001210091B3
:10FD0000E4E7394608A800F005FB002801DA284A94
:10FD1000C7E7696808A800F059FA08A9C4F8F00113
:10FD20002046FFF757FB064608B1224AB9E7394695
:10FD300008A800F057FA002801DA1F4AB1E70DF1D0
:10FD40001F0308A9204600930DF11E036A68FEF701
:10FD500095FD9DF81E309BB194F8003113B12046FB
:10FD6000FFF750FD08A92046FFF762FC08B1134ACF
:10FD700097E79DF81F301BB108A92046FFF738F917
:10FD800094F8F0303BB16A6808A92046FFF758FAAA
:10FD900008B10B4A85E72046FEF718FE002886D1F9
:10FDA000084A7EE7839F06088C950608A79F0608E9
:10FDB000C69F0608E69F060817A006084EA006087C
:10FDC0007FA00608B2A006082DE9F04FD0F8B45085
:10FDD0008FB00446B5B16B1C0CD1A5F6A575B0F972
:10FDE000B830574A02205749FCF720FC28460FB08C
:10FDF000BDE8F08F0A23544A52490220534DFCF7C4
:10FE000015FCF3E700F1BC09261D4846FEF762FA2F
:10FE10002A4629463046CDE90255CDE9005594F8E9
:10FE2000FA31F9F763F950B1494A6FF47A654549F7
:10FE30000220FCF7FBFB4846FEF768FAD6E794F889
:10FE400004320BB9C4F80052D4F800720137012F04
:10FE5000C4F80072EFD100233046D4F8F41184F8CE
:10FE6000FB3184F8FD31F9F775F9064608B1394AD6
:10FE7000DBE72046FEF7AAFD30B9374A02203149B8
:10FE8000364DFCF7D3FBD6E72046FFF773F9002881
:10FE900001DA334AC9E7DFF8E0A004F58478334695
:10FEA000214652460AA8C4E94266C4E94866CDE93B
:10FEB00004A6FFF787FE41460AA800F055FA8346DC
:10FEC0000AA8FFF705FDBBF1000F06DA254A1D4918
:10FED0000220254DFCF7AAFBADE7334652462146EA
:10FEE0000AA8CDE906A6FFF76DFE42460AA92046FC
:10FEF000FFF7B8FE83460AA8FFF7EAFCBBF1000F44
:10FF000001DA1A4AE3E73346524621460AA8CDE908
:10FF100008A6FFF757FE41460AA800F089FA0646F0
:10FF20000AA8FFF7D5FC002E01DA114ACFE72046D8
:10FF3000FFF702FC08B10F4AC9E784F804727AE7B8
:10FF4000F99E06088C950608309F060859F0FFFFB9
:10FF5000BC950608CEA00608B2A006085DF0FFFF1B
:10FF6000E8A0060808A106085EF0FFFF29A1060820
:10FF70004FA1060874A1060801E7040830B587B050
:10FF80000C9CD4E90045CDE904450B9C24680394FE
:10FF90000A9C247802941B78019313780093D1E98A
:10FFA0000023FFF7D8FD07B030BD7FB5CDE90423AE
:10FFB0000CAB08AA04A902930BAB01930AAB009304
:10FFC00009ABFFF7DBFF07B05DF804FB10B51420A9
:10FFD000FDF780FF1422FF21044611F031FE014B92
:10FFE0001C6010BDDCFD002408B528B94FF48472F4
:10FFF00003490448FDF732F80078C0F3400008BD1B
:020000040805ED
:1000000021A206082AA2060810B5042209490446BE
:1000100011F0E6FC10B96379012B07D00220064AE3
:100020000449FCF703FB4FF0FF3010BDA07901300D
:10003000FBE700BF40A2060845A2060837B5837853
:1000400004460D46012B08D00220514A5149FCF7C5
:10005000EDFA4FF0FF3003B030BD4268130EFF2BB6
:1000600040F08A8003780C2B28D91F2B76D003F11F
:100070007F02D2B20C2A01D90020ECE7813B0C2B85
:10008000FAD801A252F823F01101050879000508F9
:10009000790005082B010508790005087900050895
:1000A0006101050865010508790005087900050862
:1000B0007900050879000508750105080C2BDBD8C7
:1000C00001A151F823F000BFFD00050879000508E3
:1000D000790005084901050879000508550105085A
:1000E0005901050879000508790005086901050826
:1000F0006D010508790005087101050822F07F42AD
:100100002A60C3789B00502BA8BF50236B60B3E7D5
:10011000214A08201F49FCF789FA636823F07F43CE
:10012000AB61E3789B00EB61A6E71C4A0820194904
:10013000FCF77CFA636823F07F43C5F8D030E3789E
:100140009B00C5F8D43097E7154A12490820FCF700
:100150006DFA91E7134AF8E7134AF6E7134AF4E712
:10016000134AF2E7134AF0E7134AEEE7134AECE7C3
:10017000134AEAE7134AE8E77F2B3FF67DAF009387
:10018000114A037808200349FCF750FA74E700BFCE
:100190006EA2060840A2060899A20608B6A20608A2
:1001A000E3A2060825A306087BA30608D1A3060838
:1001B000DFA306081DA406086EA40608B9A4060855
:1001C00010A5060841A5060897A50608282981BF9D
:1001D00090F8283001201B09984098BF4FF4807098
:1001E00070470000F8B54B681C2B23D9012301F19F
:1001F000AC0401F1BC064FF0FF379C4644F8047F85
:10020000027F0CFA02F2012A22610BD9457F256098
:100210008D6DAA4200D305B98A6591F84C201A4326
:1002200081F84C205B00B44200F10200DBB2E5D162
:100230000020F8BD4378FF2B0B61F9D10220034A5F
:100240000349FCF7F3F94FF0FF30F2E7E7A50608A2
:1002500040A20608034670B5D2E90240A34271EB02
:10026000000007D2146A2CB1012C0ED058320020A5
:10027000844202DC4FF0FF3070BD52F8086F5568C1
:100280009E428D41F8D20130F2E70020F4E70000F1
:100290002DE9F74F99460F9B074603244FF00808B6
:1002A00003F1A80B0192DDE90C5A17EA080F20D0E0
:1002B0005BF8246000232846514632460EF06AFD62
:1002C0001A4316D1019BB34279F1000311D30E9961
:1002D0006A1E0F9801F109014AF1FF33921900EBF0
:1002E000C10650F8310043F1000371689042994112
:1002F00008D2013C4FEA5808D7D2044A02200449E8
:10030000FCF794F9204603B0BDE8F08F11A606086B
:1003100040A2060813B54368002408205A1CD208DE
:10032000C1E90224CDE900240349044AFCF77EF91F
:10033000204602B010BD00BF40A2060841A6060834
:1003400090F90700C017704738B504460D461022D3
:10035000002111F075FC20462946F3F721FF2046C5
:1003600038BD0000000000002DE9F04F2DED028B9C
:1003700089B04FF05A090824002206AB0746884688
:10038000039301239FED248B009300238DED048BB9
:10039000CDE90194FFF750FC00280CDA4FF0FF354F
:1003A0001F4A20490220FCF741F9284609B0BDEC5C
:1003B000028BBDE8F08F06A8FFF726FE051EF4DBD2
:1003C0000026A246B346AE4201D10020EEE706ABBE
:1003D00022463846CDF80490CDE902A301238DEDE5
:1003E000048B00935B46FFF727FC002808DA022005
:1003F000731C0D4A0B49FCF719F94FF0FF30D5E794
:10040000414606A8FFF71AFE0028CFDB083406F1A4
:1004100001064BF1000BD6E70800000000000000C9
:100420006DA6060840A206088BA60608000000007C
:100430008B692DE9F04F05460C462DED028B8DB0F2
:100440000BB1C86988B901234FF000082362D4E9D1
:1004500002326362013B42F1FF32C4E91832404686
:100460000DB0BDEC028BBDE8F08F7F49FDF740FD7C
:10047000074638B97D4A02207D494FF0FF38FCF726
:10048000D5F8ECE7E369002603900820CDE90436AF
:100490005A23CDE901300123284600933346A2694F
:1004A000FFF7CAFBB0420ADA724A71490220FCF730
:1004B000BDF84FF0FF383846FDF73BFDCFE7294642
:1004C00008A8FFF741FF3846FFF78EFD002853D1FB
:1004D000E3693D4606460DF11F0A07EB03089FED51
:1004E000608B2846FFF780FD034600283CD105F1CC
:1004F0000809C84538D319F8061C19F805BC01F0DD
:100500000F006A688909CDF80CA002908DED048B6C
:1005100019F8070C0091019008A8FFF78DFB00283F
:1005200010DAA9464FF0FF38534A02205049FCF731
:100530007DF84D4608A8FFF7CBF9B8F1000F1ED0A3
:100540004E4AB2E79DF81F3076001BEA030FF6B261
:1005500019F8083C18BF46F00106D90701D44D46EA
:10056000BFE74FF00008E4E7454A022040494FF05A
:10057000FF38FCF75BF8DDE73D46B046DAE7E369B4
:1005800007EB03092846FFF72FFDD0B105F108035B
:10059000994516D3A9788B1C05EB8303994506D2A0
:1005A000384A33490220FCF741F8374A7DE76A7838
:1005B000B24208D02A78D20701D5344AF1E71D4665
:1005C000E0E7334AEDE74B1C0A2B236207DD00937B
:1005D00002200A232F4A2649FCF728F869E7043548
:1005E00004F1200C04F14B0604F158004FF0000E0A
:1005F0000F222B68B14615F804AB23F0FF030AF075
:100600000F0A03F5807302EA0A024CF8043F013B2B
:1006100006F801AF73444FEAE37E40F8083FC0F8A4
:1006200004E003F1010EA9F14B031B1B9942E0DC2E
:100630000023D507A36508D5303354F82330A365CC
:1006400039E70123F8E70223F6E79007F9D45107C9
:10065000F9D413077FF52FAF0323EDE7AFF3008045
:100660000100000000000000DCC70608B3A6060871
:1006700040A20608CDA60608F0A6060866A706084A
:1006800023A7060890A7060852A80608D5A70608BB
:1006900024A8060879A806087047000010B50320B2
:1006A00000F052FB04F026FE0F49104A8B69C3F399
:1006B0000323D35C03F01F03D8408B6903F00F03BF
:1006C000D35C0B4A03F01F0320FA03F31360094BBA
:1006D00018600F200AF032F8044618B9FFF7DCFF63
:1006E000204610BD0124FBE7004402583CA906083F
:1006F0008C0E0024900E002438B504460AF024F82D
:100700000546631C1EBF044B1B78E4180AF01CF856
:10071000431BA342FAD338BD840E0024014B186852
:10072000000C70470010005C014BD3F800087047C4
:1007300000E0F11F014BD3F80408704700E0F11FFF
:10074000014BD3F80808704700E0F11F034A5368D3
:1007500023F4600303435360704700BF0004005854
:10076000024A136A43F00103136270470004005801
:1007700030B5CC030DD5430900F01F05012403F16A
:10078000B063AC4008331B011D68A2B925EA04041C
:100790001C608B030ED500F01F01400901230001EE
:1007A0008B4000F1B04042B9D0F8842022EA030324
:1007B000C0F8843030BD2C43EAE7D0F884201343DE
:1007C000F6E730B5CC030DD5430900F01F05012431
:1007D00003F1B063AC400C331B011D68A2B925EADC
:1007E00004041C608B030ED500F01F014009012397
:1007F00000018B4000F1B04042B9D0F8C42022EA99
:100800000303C0F8C43030BD2C43EAE7D0F8C4205D
:100810001343F6E7806800F0010070478068C0F37A
:10082000800070477047026838B5044610469368E8
:10083000FFF7F0FF08B9002038BD9907FBD4936893
:1008400003F00D03012B19D1936823F0004323F02B
:100850003F0343F0020393600323136009F074FF26
:10086000054623689B68DB07E5D509F06DFF401B53
:100870000228F6D923689B68DA07F2D5636D012058
:1008800043F010036365A36D43F00103A365D3E751
:1008900038B5434A05460368934203D002F5807297
:1008A000934224D13F4B9B6813F4403F14BF012374
:1008B0000023F3B94FF4002005F068FF6B6804468D
:1008C000B3F5101F4AD03FD8B3F5E01F44D036D857
:1008D000B3F5801F08D02CD8B3F5002F04D023F433
:1008E0000022B2F5802F16D19B0C5B000FE02E4B3F
:1008F000D9E704F0C7FE6B680446B3F5003F05D0A6
:10090000B3F5403F06D0B3F5803F04D11B0CB4FBD8
:10091000F3F400E08408FFF701FF41F2030398427B
:100920002B6823D8214A94429A681BD942F48072DA
:100930001AE0B3F5A01FD7D0B3F5C01FD3E7B3F5C6
:10094000001FE8D14409E6E7B3F5201F08D0B3F54E
:10095000301FE0D1040ADEE70409DCE78409DAE7A6
:10096000C409D8E722F480729A6038BD104A9442D4
:1009700003D89A6822F44072F6E70E4A944203D8EC
:100980009A6822F44072D1E70B4A94429A6896BF63
:1009900022F4407242F4407242F40072E4E700BF75
:1009A000002002400023024000630258002D310164
:1009B00021BCBE0041787D0181F0FA02002373B5AD
:1009C00004460193002800F0ED80456D25B9FFF73E
:1009D00029FFA56584F8505023689A68900005D5D2
:1009E0009A6822F0204222F03F029A609A68D10071
:1009F00040F19E809A68D20000F1B080626D0125BE
:100A000042F010026265A26D42F00102A265184632
:100A1000FFF704FF626D02F01002024340F0BE8057
:100A2000626D184622F4817242F002026265FFF79D
:100A3000F1FE88B95C4A934204D002F58072934279
:100A400040F08E805848FFF7E5FE03465748FFF711
:100A5000E1FE034300F09280FFF760FE41F20303E2
:100A6000A2689842217F607D236B40F28980102A22
:100A700040F086800A0442EA4032134343F01C03EC
:100A8000012902BF226A02F1FF3243EA4243626A4D
:100A900022B102F47872A16A0A43134322684449DE
:100AA000D068014010461943D160FFF7B7FE936844
:100AB00003F00803034327D1D368217D23F4804347
:100AC00023F0030343EA8133E16A0B43D36094F8D4
:100AD0003830012B5AD1E36B1069591ED4E9103616
:100AE000334343EA0143A16C0B43324901400B43BA
:100AF00043F00103136120461369616B23F07043D7
:100B00000B431361FFF7C4FEE3682268012B41D158
:100B1000116BA36921F00F01013B0B431363636D5C
:100B200023F0030343F001036365284602B070BD60
:100B30009A68214922F0104222F03F0242F080528E
:100B40009A601E4A1268B2FBF1F201320192019AD8
:100B5000002A3FF44FAF019A013AF7E7002556E724
:100B60001748FFF757FE00287FF476AF154A9368C1
:100B7000616823F47C130B4393606DE7124AF6E738
:100B8000134343EA403343EA014379E7136923F00F
:100B90000103AFE7136B23F00F03BFE7636D43F06F
:100BA000100363650125C0E70020024000210240D8
:100BB00003C0F0FF1EF800FC400D0300900E00245F
:100BC000006002580063025800230240806800F071
:100BD000010070478068C0F380007047002373B540
:100BE0000193044690F850300D461646012B3ED036
:100BF000012380F85030FFF716FE636D002833D1D3
:100C000023F48853226806F0804605F4803523F0EB
:100C1000020343F002036365164B91680B403343B4
:100C20002B4343F0004393609368002B12DA019B3F
:100C3000013301930199104B9942F5D3636D012063
:100C400023F0120343F010036365002384F850304F
:100C500002B070BD636D23F0030343F001036365CD
:100C6000002384F85030F3E743F01003F7E7022045
:100C7000EEE700BFC0FFFE3F00F8C32570B590F857
:100C800050209AB00346012A55D001222B4C80F8FF
:100C9000502000201D681690A54217900ED12848BC
:100CA000FFF798FF04462846FFF794FF20430ED035
:100CB000596D104641F02001596524E0596D83F8C3
:100CC0005000104641F0200159651AB070BD0C6803
:100CD0001C4AE4B190684E6820F440403043906074
:100CE0002846FFF773FF05461548FFF76FFF0543DA
:100CF00008D1896890680C4320F4716121F00F01DC
:100D00000C4394600020002283F85020DDE79168B6
:100D1000284621F440419160FFF758FF01460848FA
:100D2000FFF754FF0143EDD1916821F4716121F087
:100D30000F019160E6E70220C7E700BF00200240F4
:100D4000002102400023024007490302CA6803F45D
:100D5000E06322F4E0621204120C134343F0BF6319
:100D600043F40033CB60704700ED00E0164B30B524
:100D7000DC68C4F30224C4F10703251D042B28BF3B
:100D80000423062D4FF0FF358CBF033C002405FAE9
:100D900003F3002805FA04F521EA030322EA050219
:100DA00003FA04F343EA02034FEA0313DBB206DB60
:100DB00000F1604000F5614080F8003330BD00F084
:100DC0000F00024A1354F9E700ED00E014ED00E0D3
:100DD000002807DB0123410900F01F00024A83407D
:100DE00042F82130704700BF00E100E000280CDB32
:100DF0004309012200F01F0004492033824041F8DA
:100E00002320BFF34F8FBFF36F8F704700E100E0E7
:100E1000BFF35F8F044B5A6A22F480325A62002279
:100E2000C3F89420704700BF00ED00E0064B40F08F
:100E30000100C3F894005A6A42F480325A62BFF348
:100E40004F8FBFF36F8F704700ED00E04378144A77
:100E500010B5C2F898300178E9B14368C2F89C3007
:100E6000C37A047B1B0643EA04730B43817A43EA8B
:100E7000C143417B43EA8143817B43EA4143C17BD8
:100E800043EA0143417A43EA0123017A43EA4103F9
:100E9000C2F8A03010BDC2F89C10C2F8A010F9E74B
:100EA00000ED00E0044B1B6803F0F003702B14BF4F
:100EB00001200320704700BF00ED00E008B528B115
:100EC00090F83530022B03D08023436501205DE08C
:100ED00003683F4A934251D0183293424ED01832A1
:100EE00093424BD01832934248D01832934245D0A7
:100EF0001832934242D0183293423FD01832934274
:100F00003CD002F55672934238D01832934235D015
:100F10001832934232D0183293422FD01832934273
:100F20002CD01832934229D01832934226D018324E
:100F3000934223D01A6822F00E021A601A6822F037
:100F400001021A60234A934221D1026E136823F4EE
:100F500080731360D0E9161303F01F02012393403E
:100F60004B60D0E919325A60C36E2BB31A6822F471
:100F700080721A60D0E91C325A601DE0042280F8A9
:100F800035201A6822F001021A60002008BD124ABA
:100F90009342DAD014329342D7D014329342D4D051
:100FA00014329342D1D014329342CED014329342B1
:100FB000CBD014329342C8D0002380F834300123C0
:100FC00080F83530036D002BDFD09847DDE700BF98
:100FD00010000240085402581C54025890F8350082
:100FE000704710B502680C688B68106823434C6921
:100FF00020F07F4023438C6920F47B0023434C6A1C
:1010000020F4FE402343CC6A20F07C0023430343BA
:10101000087943EAC063087B43EAC053487B43EA4C
:101020008053887B43EA4053C87B43EA0053887C63
:1010300043EA0043087F43EA0033487F43EAC02382
:10104000C87F43EA402391F8280043EA0013087C54
:10105000B0FA80F0400943EAC043487CB0FA80F01F
:10106000400943EA4043887FB0FA80F0400943EAF0
:10107000802391F82000B0FA80F0400943EA002371
:10108000C86B1360536823F07C5323F4EF2323F4DD
:10109000FF6323F0070343EA4063486B034391F87F
:1010A000380043EA006391F8300043EA804391F846
:1010B000310043EA404391F83200B0FA80F0400931
:1010C00043EA00435360D368486C23F4877323F0EA
:1010D0000103034391F8400043EA0023886CD36086
:1010E000136F23F0F2031B041B0C43EA0043086D4B
:1010F000034391F8540043EA400391F84C00B0FADE
:1011000080F0400943EAC0131367D2F8900091F8C9
:10111000563020F00300034391F8550043EA4003A2
:10112000886DC2F89030D2F8003D23F0720303437B
:10113000C86DC2F8003DD2F8303D23F07B03034375
:1011400091F8610043EA001391F8620091F8601091
:1011500043EAC003B1FA81F1490943EA8113C2F8B5
:10116000303D10BD0368086803F580531A6822F407
:10117000F04222F00202024310B51A600A7B58685E
:101180000C79D20320F4504042EA04328C6820F0FB
:101190000100224302435A600A6A487BD3F80041A7
:1011A00042EA0042104820400243C3F800214A7F2F
:1011B000087D1203D3F8044142EA00120869024391
:1011C0000A4820400243C3F80421D3F808010C7FE9
:1011D0008A6920F0004142EAC47221F47C110A437A
:1011E000C3F8082110BD00BF00C0FEFFEFEFC0FF35
:1011F0002DE9F74FD0F840E0009200EB8E038F68A6
:101200009A69D468002C57DB5B6C002B54D10D68B5
:1012100015F0040C28D0D4684B6A6FF30F042343F5
:101220000468D360D36843F48033D360236E43F4FF
:10123000801323662B0717D59668CB6AB6B246EAA9
:1012400003439360D36843F40033D360D6680B6BD9
:1012500026F440263343D360636E43F48013636601
:10126000236D43F08063236515F0100A09D094685C
:101270008B696FF30D0423439360D36843F080635D
:10128000D36015F014091BD0D3680EF1010643F0AA
:101290008043092ED36088BFAEF10906D36843F0BE
:1012A0000043D36000EB86039B69DC68002C7CDA8A
:1012B000D36823F00043D360022003B0BDE8F08F71
:1012C000134676463C681C609C6824F47F587C6812
:1012D00028F03F0848EA0404DFF800829C60BC68FC
:1012E000002C65D027685F609F6807EA080B676875
:1012F0004BEA07479F60DF68BAF1000F5FD027F421
:10130000F0080F6A48EAC747DF60DF684FEA97488E
:10131000CF694FEA884848EA0707DF60DF6847F48B
:101320008027DF60BCF1000F06D09F6827F4404C97
:101330008F6A4CEA07079F60DF6847F00057DF605D
:10134000DF6827F08047DF60DF6847F00047DF6035
:10135000AF0706D5DF6827F0607CCF684CEA070747
:10136000DF6005F001050027DFF87081DFF870B15C
:101370000195A568002D3CD1009A002A00F0A980B3
:101380009A6842F000429A60DA6842F08052DA606D
:1013900000EB8603C26E5A64066472B6036F0133B3
:1013A0003B44036762B6002087E74FF0010989E7F5
:1013B0005C609C6804EA08049C603C469BE727F458
:1013C000FF484F6828F07F0848EA0707DF60EF070B
:1013D00006D5DF6827F440384F6948EA0707DF6021
:1013E000AF069FD5DF6827F040680F6948EA070716
:1013F00097E706F1010CDC68BCF1090F24F080547A
:1014000088BFA6F1090CDC6000EB8C06B369DC68D0
:1014100024F00054DC60DC68002C16DA09F10104C9
:1014200000233C449C423FF447AFD168013321F094
:101430000041D1600EF10101092988BFAEF1090117
:1014400000EB81028E469269ECE7746C002CE5D1CA
:101450002C681C609E686C686FF30D062643AC68B0
:101460009E6004B325685D609E68656806EA0806AC
:1014700046EA05469E60DE68BAF1000F1AD0CD69D3
:1014800006EA0B062E43DE60DD6845F48025DD604C
:10149000DD680137664645F00045DD60DD6825F012
:1014A0008045DD6065E75C609C6804EA08049C6038
:1014B0002C46E0E74D686FF30E062E43019DDE607B
:1014C000002DE5D0DE684D6926F440362E43DE60FF
:1014D000DEE79A6822F0004255E700BFFFFF00C038
:1014E0000000FCFF30B5054600EB8100446F0AB1F7
:1014F000032903D90120C5F8A40030BD2260226170
:10150000E26842F08072E2602BB1A3606361E3683D
:1015100043F00073E360E368002043F00043E360BE
:10152000EBE7D0F89C30102B10B544D1232300F109
:101530008004C0F89C3000F1700353F8041FCA689F
:10154000A34242F08042CA60F7D10123C0F8943030
:1015500003681A6842F002021A601A6842F0010237
:101560001A60D3F8002D42F00102C3F8002D03F5F4
:101570008053D3F8042142F00102C3F80421D3F8C8
:10158000082142F00102C3F80821D3F8602142F497
:101590008172C3F86021D3F8342142F4504242F002
:1015A0004102C3F834211023C0F89C302223C0F834
:1015B000A030002010BD0120FCE7D0F89C3033B3F0
:1015C0002323C0F89C30036803F58052D2F804113D
:1015D00021F00101C2F80411D2F8081121F0010133
:1015E000C2F808111A6822F001021A60D3F8002D1F
:1015F00042F00102C3F8002D1A6822F002021A60BC
:101600001023C0F89C30C0F8A030002070470120A3
:101610007047F8B50446154639B9D0F8A43043F000
:101620000103C4F8A4300120F8BDD0F89C30102B81
:10163000F9D10022FFF7DCFD20B1D4F8A43043F04B
:101640000203EEE7226C931D54F82370531C092B00
:1016500088BFA2F1090322682364063302F5805291
:1016600054F82330C2F8203109F06EF80646FB68C2
:10167000002B01DB0020D7E7236803F58053D3F864
:101680006021D2040DD5D4F8A42042F00802C4F899
:10169000A420D3F86031C4F8A830E023C4F89C300B
:1016A000C1E76B1CE3D009F04FF8801BA84206D9B4
:1016B000D4F8A43043F00403C4F8A430EDE7002DBF
:1016C000D5D1F5E7F0B5D0F88C50002D40D1D0F849
:1016D00084102A462C46052700EB81035E6FF368D1
:1016E000002B01DB013F35D17CB300EB8203D0F846
:1016F00094604FF0807704F1FF3C5B6FC0E92112EA
:10170000196919605969DF6021B19960D96841F0A0
:101710000071D960D96841F00041D9601EB1D96823
:1017200041F08041D960AC4507D9511C032988BFDD
:10173000D11E00EB81030A465B6F0135AC42DFD15D
:10174000026802F58052C2F828310023C0F88C30BC
:10175000002023E0D6F80CC04B1C1CF0805F1ED08C
:10176000002C08BF0A46032B04F1010588BFCB1EDD
:1017700000EB8301496FCC68002C0ADBC9684F007D
:1017800007D50121C0F89010591803298CBF033BDD
:101790000B46C0F88C50C0E921320120F0BDF6683C
:1017A000B6000AD5032B4FF0010488BFCB1E00EB17
:1017B0008302566F0A46194691E7032B04F1010490
:1017C00088BFCB1E00EB83014E6FF4E7D0F8882072
:1017D000F8B500EB820305460C465B6F21B9012387
:1017E000C0F8A43001201EE0D0F88C1041B9FFF7FA
:1017F00069FF0028F6D0D5F8882005EB82035B6FDF
:10180000D5F88C10002001F1FF3C07466969BC4502
:101810000AD8DA68C2F30E02121A186991422060DF
:1018200019D362600020F8BD1869C4E90001586945
:1018300018B1A4685869C4E90001561CD868A468A6
:101840000137032EC0F30E0088BFD61E05EB8603BA
:1018500032465B6FDBE758690028C3D0A068521A94
:101860005B69616003604260DCE770B5D0E92253D8
:1018700004460E4673B1D4F88C302B445A1E032A0A
:101880000ED804EB82040020636FDB68C3F30E0301
:10189000336070BDFFF716FF0028ECD10120F8E798
:1018A0005A1FEEE7D0F88C100246F0B5002939D067
:1018B000D0F8903003B10131D2F8884000204FF0C9
:1018C00080764F1E02EB84035B6F814208D1116862
:1018D000002001F58051C1F82831C2E92300F0BD94
:1018E0001D691D60DE605D692DB15D699D60DD680B
:1018F00045F00075DD60DD6845F00045DD60D2F83B
:1019000094501DB1DD6845F08045DD60874207D900
:10191000651C032D88BFE51E02EB85032C465B6F1B
:101920000130D2E70120DAE770477047704770470F
:10193000036803F58053D3F86021520610B50446BE
:101940000CD5D3F83431590608D5F6F761FC236875
:1019500048F2400203F58053C3F86021236803F581
:101960008053D3F86021D2070DD5D3F83431DB078B
:1019700009D52046FFF7D8FF236848F2010203F596
:101980008053C3F86021236803F58053D3F86021A6
:10199000500424D5D3F83421510420D5D4F8A42000
:1019A00042F00802C4F8A420D3F8602112F4805F4A
:1019B000D3F860215CD022F46F6222F00D02D204D1
:1019C000D20CC4F8A820D3F8342122F44042C3F842
:1019D0003421E023C4F89C302046F6F72DFA226823
:1019E000D2F8B03003F4C043B3F5C04F0CD1D2F8F5
:1019F000B8302046C4F8AC30E023C4F89C30F6F789
:101A000027FA0023C4F8AC302368D3F8B020D206FC
:101A10000BD5D3F8C030204603F06003C4F8B030D3
:101A2000FFF783FF0023C4F8B0302368D3F8B02059
:101A300090060BD5D3F8C030204603F00F03C4F84E
:101A4000B430FFF773FF0023C4F8B430FFF72AFA6D
:101A500003284FF0B04314D1D3F8A820510206D583
:101A60004FF48002C3F8A8202046FFF760FF10BDA6
:101A700002F4CD42C4F8A8204FF4CD42C3F860214F
:101A8000AAE7D3F8E8205202F1D54FF48002C3F858
:101A9000E820E9E770B51E4603680546D3F8000262
:101AA000C00701D5012070BDD3F8004224F078743E
:101AB00044EA415121F4F81141EA024242F00D0298
:101AC000C3F8002208F040FE04462A68D2F800025B
:101AD00010F0010004D1D2F804329BB23360E2E787
:101AE00008F032FE001BB0F57A7FEED9DAE700008D
:101AF00038B505460068D0F80042E40701D501205A
:101B000038BDD0F800429BB224F0787444EA4151C9
:101B100021F4F81141EA02420C4922F00C02C1F80A
:101B2000043242F00502C1F8002208F00DFE04461E
:101B30002B68D3F8000210F00100E1D008F004FE99
:101B4000001BB0F57A7FF3D9D9E700BF00800240CF
:101B5000002900F0C180036800201A6802F00C021E
:101B6000CA621A68C2F3001281F828201A6802F0CB
:101B700060024A621A6882F48072C2F3002281F81D
:101B800020201A68C2F34022CA771A6882F4806261
:101B9000C2F380228A771A68C2F3C0224A771A6891
:101BA000C2F300320A771A6802F400528A611A6896
:101BB00002F480424A611A68C2F300428A741A68C9
:101BC00082F40032C2F340424A741A6882F400225E
:101BD000C2F3C0420A741A68C2F30052CA731A6888
:101BE000C2F340528A731A68C2F380524A731A6869
:101BF000C2F3C0520A731A6802F0E0628A601A687F
